Component: ARM Compiler 5.06 update 4 (build 422) Tool: armlink [4d35d2]

==============================================================================

Section Cross References

    main.o(.text) refers to driver.o(.text) for HWSetup
    main.o(.text) refers to typedefine.o(.text) for SystemSWInit
    main.o(.text) refers to coaphandle.o(.text) for ModelRegister
    main.o(.text) refers to regist.o(.text) for DeviceRegist
    main.o(.text) refers to module_wrapper.o(.text) for at_module_low_power
    main.o(.text) refers to lorawan.o(.text) for lorawan_Sleep
    main.o(.text) refers to controlsystem.o(.text) for CntlSysInitWork
    main.o(.text) refers to drawlcdgui.o(.text) for DrawScheduleDisplay
    main.o(.text) refers to systemalarm.o(.text) for SystemAlarmJudge
    main.o(.text) refers to rtcsetup.o(.text) for SystemTimeUpdate
    main.o(.text) refers to adcsetup.o(.text) for BatteryVoltADCGet
    main.o(.text) refers to bubble_adcsetup.o(.text) for OPB350L_ADCGet
    main.o(.text) refers to zigbeedatahandle.o(.text) for ZigbeeRecvHandle
    main.o(.text) refers to remote.o(.text) for remoteHandle
    main.o(.text) refers to hostslavehandle.o(.text) for HostToSlaveHandle
    main.o(.text) refers to typedefine.o(.bss) for EngineeringModeValue
    main.o(.text) refers to programdata.o(.data) for registInfo
    driver.o(.text) refers to stm32f10x_rcc.o(.text) for RCC_APB2PeriphClockCmd
    driver.o(.text) refers to stm32f10x_gpio.o(.text) for GPIO_Init
    driver.o(.text) refers to misc.o(.text) for NVIC_Init
    driver.o(.text) refers to stm32f10x_exti.o(.text) for EXTI_Init
    driver.o(.text) refers to typedefine.o(.text) for Delay_ms
    driver.o(.text) refers to controlsystem.o(.text) for HornWorkStatus
    driver.o(.text) refers to delay.o(.text) for delay_us
    driver.o(.text) refers to system_stm32f10x.o(.text) for SystemInit
    driver.o(.text) refers to usartsetup.o(.text) for USART1_Init
    driver.o(.text) refers to spisetup.o(.text) for SPIInit
    driver.o(.text) refers to iicsetup.o(.text) for IICInit
    driver.o(.text) refers to ads1110setup.o(.text) for ADS1110Config
    driver.o(.text) refers to bubble_adcsetup.o(.text) for OPB350L_ADCInit
    driver.o(.text) refers to typedefine.o(.data) for SysHornToneType
    driver.o(.text) refers to typedefine.o(.bss) for TaskSchedulerFlag
    driver.o(.text) refers to driver.o(.data) for mcu_id
    driver.o(.text) refers to stm32f10x_it.o(.data) for random_cont
    driver.o(.text) refers to lorawan.o(.data) for Recive_lorawanID_flag
    driver.o(.text) refers to system_stm32f10x.o(.data) for SystemCoreClock
    typedefine.o(.text) refers to flashsetup.o(.text) for FlashReadOperate
    typedefine.o(.text) refers to memseta.o(.text) for __aeabi_memclr4
    typedefine.o(.text) refers to lcdsetup.o(.text) for LCDInit
    typedefine.o(.text) refers to fm31256.o(.text) for GetCurDateTimeFromRTC
    typedefine.o(.text) refers to parameterset.o(.text) for ReadParameterRecord
    typedefine.o(.text) refers to programdata.o(.text) for WriteInitProgramData
    typedefine.o(.text) refers to history.o(.text) for ReadHistoryRecordQTY
    typedefine.o(.text) refers to typedefine.o(.bss) for TaskSchedulerTimer
    typedefine.o(.text) refers to parameterset.o(.bss) for paramRecordBuf
    typedefine.o(.text) refers to history.o(.bss) for historyRecordBuf
    typedefine.o(.text) refers to typedefine.o(.data) for KeyScanStatus
    typedefine.o(.text) refers to controlsystem.o(.data) for InfusionStopTimer
    typedefine.o(.text) refers to systemalarm.o(.bss) for AlarmRecord
    typedefine.o(.text) refers to systemalarm.o(.data) for SysAlarmJudge
    typedefine.o(.text) refers to drawlcdgui.o(.data) for emDisplayPicture
    typedefine.o(.text) refers to history.o(.data) for historyRecordQTY
    typedefine.o(.text) refers to programdata.o(.data) for classification
    stm32f10x_it.o(.text) refers to stm32f10x_gpio.o(.text) for GPIO_ReadInputDataBit
    stm32f10x_it.o(.text) refers to typedefine.o(.data) for motorWorkState
    stm32f10x_it.o(.text) refers to typedefine.o(.bss) for TaskSchedulerTimer
    stm32f10x_it.o(.text) refers to controlsystem.o(.data) for emSysWorkStep
    stm32f10x_it.o(.text) refers to stm32f10x_it.o(.data) for lorawan_overtime
    stm32f10x_it.o(.text) refers to lorawan.o(.data) for lorawan_send_data_flag
    stm32f10x_it.o(.text) refers to systemalarm.o(.bss) for sysAlarmFlag
    stm32f10x_it.o(.text) refers to systemalarm.o(.data) for Timer_VoltLowes
    stm32f10x_it.o(.text) refers to bubble_adcsetup.o(.data) for BubbleCheckTime
    stm32f10x_it.o(.text) refers to rand.o(.text) for srand
    stm32f10x_it.o(.text) refers to controlsystem.o(.text) for CntlSystemWorkTimer
    stm32f10x_it.o(.text) refers to zigbeedatahandle.o(.data) for RunToLorawawn_flag
    stm32f10x_it.o(.text) refers to stm32f10x_exti.o(.text) for EXTI_GetITStatus
    stm32f10x_it.o(.text) refers to stm32f10x_usart.o(.text) for USART_GetITStatus
    stm32f10x_it.o(.text) refers to usartsetup.o(.bss) for usart1RecvBuffer
    stm32f10x_it.o(.text) refers to usartsetup.o(.data) for usart1RecvCnt
    stm32f10x_it.o(.text) refers to sys.o(.bss) for uart_recv
    stm32f10x_it.o(.text) refers to usartsetup.o(.text) for USART1Send
    stm32f10x_it.o(.text) refers to printfa.o(i.__0printf) for __2printf
    timersetup.o(.text) refers to stm32f10x_tim.o(.text) for TIM_DeInit
    rtcsetup.o(.text) refers to stm32f10x_rtc.o(.text) for RTC_WaitForLastTask
    rtcsetup.o(.text) refers to stm32f10x_rcc.o(.text) for RCC_APB1PeriphClockCmd
    rtcsetup.o(.text) refers to stm32f10x_pwr.o(.text) for PWR_BackupAccessCmd
    rtcsetup.o(.text) refers to stm32f10x_bkp.o(.text) for BKP_ReadBackupRegister
    rtcsetup.o(.text) refers to fm31256.o(.text) for GetCurDateTimeFromRTC
    rtcsetup.o(.text) refers to misc.o(.text) for NVIC_Init
    rtcsetup.o(.text) refers to stm32f10x_exti.o(.text) for EXTI_ClearITPendingBit
    rtcsetup.o(.text) refers to rtcsetup.o(.constdata) for table_week
    rtcsetup.o(.text) refers to rtcsetup.o(.data) for daycnt
    rtcsetup.o(.text) refers to typedefine.o(.data) for displayTimeBuf
    rtcsetup.o(.text) refers to typedefine.o(.bss) for TaskSchedulerFlag
    rtcsetup.o(.text) refers to drawlcdgui.o(.data) for emCurrentPicture
    spisetup.o(.text) refers to stm32f10x_rcc.o(.text) for RCC_APB2PeriphClockCmd
    spisetup.o(.text) refers to stm32f10x_gpio.o(.text) for GPIO_Init
    ads1110setup.o(.text) refers to iicsetup.o(.text) for TWI_START
    ads1110setup.o(.text) refers to memseta.o(.text) for __aeabi_memclr
    ads1110setup.o(.text) refers to ads1110setup.o(.data) for tempPressure
    ads1110setup.o(.text) refers to typedefine.o(.bss) for TaskSchedulerFlag
    ads1110setup.o(.text) refers to ads1110setup.o(.bss) for pressureF1
    ads1110setup.o(.text) refers to systemalarm.o(.data) for SysAlarmJudge
    ads1110setup.o(.text) refers to controlsystem.o(.data) for start_flag
    iicsetup.o(.text) refers to stm32f10x_rcc.o(.text) for RCC_APB2PeriphClockCmd
    iicsetup.o(.text) refers to stm32f10x_gpio.o(.text) for GPIO_Init
    usartsetup.o(.text) refers to stm32f10x_rcc.o(.text) for RCC_APB2PeriphClockCmd
    usartsetup.o(.text) refers to stm32f10x_gpio.o(.text) for GPIO_Init
    usartsetup.o(.text) refers to stm32f10x_usart.o(.text) for USART_Init
    usartsetup.o(.text) refers to misc.o(.text) for NVIC_Init
    lcdsetup.o(.text) refers to typedefine.o(.text) for Delay_ms
    lcdsetup.o(.text) refers to spisetup.o(.text) for SPIWriteByte
    history.o(.text) refers to usartsetup.o(.text) for USART1Send
    history.o(.text) refers to flashsetup.o(.text) for FlashReadOperate
    history.o(.text) refers to typedefine.o(.bss) for TaskSchedulerFlag
    history.o(.text) refers to usartsetup.o(.bss) for usart1RecvBuffer
    history.o(.text) refers to history.o(.bss) for historyRecord
    history.o(.text) refers to history.o(.data) for historyRecordQTY
    history.o(.text) refers to typedefine.o(.data) for displayTimeBuf
    flashsetup.o(.text) refers to stm32f10x_flash.o(.text) for FLASH_Unlock
    parameterset.o(.text) refers to flashsetup.o(.text) for FlashReadOperate
    parameterset.o(.text) refers to parameterset.o(.bss) for paramRecordBuf
    parameterset.o(.text) refers to typedefine.o(.bss) for setParamInfo
    adcsetup.o(.text) refers to stm32f10x_rcc.o(.text) for RCC_AHBPeriphClockCmd
    adcsetup.o(.text) refers to stm32f10x_dma.o(.text) for DMA_DeInit
    adcsetup.o(.text) refers to stm32f10x_gpio.o(.text) for GPIO_Init
    adcsetup.o(.text) refers to stm32f10x_adc.o(.text) for ADC_Init
    adcsetup.o(.text) refers to adcsetup.o(.data) for ADC_ConvertedValue
    adcsetup.o(.text) refers to typedefine.o(.bss) for TaskSchedulerFlag
    adcsetup.o(.text) refers to typedefine.o(.data) for motorWorkState
    controlsystem.o(.text) refers to stm32f10x_usart.o(.text) for USART_SendData
    controlsystem.o(.text) refers to stm32f10x_gpio.o(.text) for GPIO_SetBits
    controlsystem.o(.text) refers to driver.o(.text) for SpeakerCtl
    controlsystem.o(.text) refers to controlsystem.o(.data) for emSysWorkStep
    controlsystem.o(.text) refers to typedefine.o(.bss) for TaskSchedulerFlag
    controlsystem.o(.text) refers to typedefine.o(.data) for sysPromptToneType
    controlsystem.o(.text) refers to systemalarm.o(.bss) for sysAlarmFlag
    controlsystem.o(.text) refers to drawlcdgui.o(.text) for DrawSilenceDisplay
    controlsystem.o(.text) refers to drawlcdgui.o(.data) for emDisplayPicture
    controlsystem.o(.text) refers to hostslavehandle.o(.text) for HostToSlaveHandle
    controlsystem.o(.text) refers to systemalarm.o(.text) for PECASelfTestHandle
    controlsystem.o(.text) refers to history.o(.text) for ReadHistoryRecord
    controlsystem.o(.text) refers to history.o(.data) for FackhistoryRecordQTY
    controlsystem.o(.text) refers to history.o(.bss) for historyRecord
    controlsystem.o(.text) refers to fm31256.o(.text) for SetDateTimeToRTC
    controlsystem.o(.text) refers to parameterset.o(.text) for WriteParameterRecord
    controlsystem.o(.text) refers to typedefine.o(.text) for RunParamUpdate
    controlsystem.o(.text) refers to bubble_adcsetup.o(.data) for ElectStartCount
    controlsystem.o(.text) refers to ads1110setup.o(.data) for self_adaption_Pressure
    controlsystem.o(.text) refers to zigbeedatahandle.o(.data) for StartToRun_flag
    controlsystem.o(.text) refers to flashsetup.o(.text) for FlashWriteOperate
    controlsystem.o(.text) refers to zigbeedatahandle.o(.text) for RunToLorawawn
    controlsystem.o(.text) refers to systemalarm.o(.data) for SysAlarmJudge
    drawlcdgui.o(.text) refers to lcdsetup.o(.text) for LCDSetXY
    drawlcdgui.o(.text) refers to uldiv.o(.text) for __aeabi_uldivmod
    drawlcdgui.o(.text) refers to drawlcdgui.o(.constdata) for asc8
    drawlcdgui.o(.text) refers to typedefine.o(.bss) for TaskSchedulerFlag
    drawlcdgui.o(.text) refers to systemalarm.o(.bss) for sysAlarmFlag
    drawlcdgui.o(.text) refers to drawlcdgui.o(.data) for modifyStep
    drawlcdgui.o(.text) refers to controlsystem.o(.data) for emSysWorkStep
    drawlcdgui.o(.text) refers to history.o(.bss) for historyRecord
    drawlcdgui.o(.text) refers to history.o(.data) for historyRecordQTY
    drawlcdgui.o(.text) refers to typedefine.o(.data) for emPictureRunState
    drawlcdgui.o(.text) refers to bubble_adcsetup.o(.data) for ElectricityData
    drawlcdgui.o(.text) refers to lorawan.o(.data) for send_cont
    drawlcdgui.o(.text) refers to ads1110setup.o(.data) for self_adaption_Pressure
    drawlcdgui.o(.text) refers to adcsetup.o(.data) for batteryAverage
    systemalarm.o(.text) refers to stm32f10x_gpio.o(.text) for GPIO_SetBits
    systemalarm.o(.text) refers to history.o(.text) for HistoryQtyAdd
    systemalarm.o(.text) refers to typedefine.o(.bss) for TaskSchedulerFlag
    systemalarm.o(.text) refers to typedefine.o(.data) for motorWorkState
    systemalarm.o(.text) refers to controlsystem.o(.data) for G_Led_Time
    systemalarm.o(.text) refers to systemalarm.o(.bss) for sysAlarmFlag
    systemalarm.o(.text) refers to drawlcdgui.o(.data) for emDisplayPicture
    systemalarm.o(.text) refers to history.o(.data) for historyRefreshFlag
    systemalarm.o(.text) refers to systemalarm.o(.data) for SysAlarmJudge
    systemalarm.o(.text) refers to bubble_adcsetup.o(.data) for BubbleData
    systemalarm.o(.text) refers to adcsetup.o(.data) for ADC_Voit_Done
    zigbeedatahandle.o(.text) refers to usartsetup.o(.text) for USART2Send
    zigbeedatahandle.o(.text) refers to crc16.o(.text) for CalCRC16
    zigbeedatahandle.o(.text) refers to lorawan.o(.text) for transparent_send_data
    zigbeedatahandle.o(.text) refers to usartsetup.o(.bss) for usart2XmitBuffer
    zigbeedatahandle.o(.text) refers to typedefine.o(.bss) for setParamInfo
    zigbeedatahandle.o(.text) refers to zigbeedatahandle.o(.data) for FailureSendNumber
    zigbeedatahandle.o(.text) refers to systemalarm.o(.bss) for sysAlarmFlag
    zigbeedatahandle.o(.text) refers to typedefine.o(.data) for displayTimeBuf
    zigbeedatahandle.o(.text) refers to controlsystem.o(.data) for Start_send
    zigbeedatahandle.o(.text) refers to parameterset.o(.text) for WriteParameterRecord
    zigbeedatahandle.o(.text) refers to lorawan.o(.data) for Recive_lorawanID_flag
    zigbeedatahandle.o(.text) refers to driver.o(.data) for mcu_id
    crc16.o(.text) refers to crc16.o(.constdata) for auchCRCHi
    hostslavehandle.o(.text) refers to stm32f10x_rcc.o(.text) for RCC_APB2PeriphClockCmd
    hostslavehandle.o(.text) refers to stm32f10x_gpio.o(.text) for GPIO_Init
    hostslavehandle.o(.text) refers to typedefine.o(.bss) for realTimeData
    hostslavehandle.o(.text) refers to systemalarm.o(.bss) for sysAlarmFlag
    fm31256.o(.text) refers to iicsetup.o(.text) for RTC_START
    fm31256.o(.text) refers to typedefine.o(.data) for displayTimeBuf
    ads1110asetup.o(.text) refers to iic2setup.o(.text) for TWI2_START
    iic2setup.o(.text) refers to stm32f10x_rcc.o(.text) for RCC_APB2PeriphClockCmd
    iic2setup.o(.text) refers to stm32f10x_gpio.o(.text) for GPIO_Init
    lorawan.o(.text) refers to stm32f10x_rcc.o(.text) for RCC_APB2PeriphClockCmd
    lorawan.o(.text) refers to stm32f10x_gpio.o(.text) for GPIO_Init
    lorawan.o(.text) refers to usartsetup.o(.text) for USART2Send
    lorawan.o(.text) refers to lorawan.o(.data) for send_cont
    lorawan.o(.text) refers to stm32f10x_it.o(.data) for lorawan_time_5s
    lorawan.o(.text) refers to zigbeedatahandle.o(.data) for lorawan_to_sleep
    bubble_adcsetup.o(.text) refers to stm32f10x_rcc.o(.text) for RCC_APB2PeriphClockCmd
    bubble_adcsetup.o(.text) refers to stm32f10x_gpio.o(.text) for GPIO_Init
    bubble_adcsetup.o(.text) refers to stm32f10x_adc.o(.text) for ADC_Init
    bubble_adcsetup.o(.text) refers to typedefine.o(.data) for motorWorkState
    bubble_adcsetup.o(.text) refers to typedefine.o(.bss) for TaskSchedulerFlag
    bubble_adcsetup.o(.text) refers to bubble_adcsetup.o(.data) for BubbleCountFlag
    bubble_adcsetup.o(.text) refers to systemalarm.o(.data) for SysAlarmJudge
    bubble_adcsetup.o(.text) refers to bubble_adcsetup.o(.bss) for ElectricityVolt
    bubble_adcsetup.o(.text) refers to systemalarm.o(.bss) for sysAlarmFlag
    bubble_adcsetup.o(.text) refers to zigbeedatahandle.o(.data) for StartToRun_flag
    bubble_adcsetup.o(.text) refers to controlsystem.o(.data) for start_flag
    system_stm32f10x.o(.text) refers to system_stm32f10x.o(.data) for SystemCoreClock
    stm32f10x_gpio.o(.text) refers to stm32f10x_rcc.o(.text) for RCC_APB2PeriphResetCmd
    stm32f10x_rcc.o(.text) refers to stm32f10x_rcc.o(.data) for APBAHBPrescTable
    stm32f10x_usart.o(.text) refers to stm32f10x_rcc.o(.text) for RCC_APB2PeriphResetCmd
    stm32f10x_tim.o(.text) refers to stm32f10x_rcc.o(.text) for RCC_APB2PeriphResetCmd
    stm32f10x_pwr.o(.text) refers to stm32f10x_rcc.o(.text) for RCC_APB1PeriphResetCmd
    stm32f10x_bkp.o(.text) refers to stm32f10x_rcc.o(.text) for RCC_BackupResetCmd
    stm32f10x_adc.o(.text) refers to stm32f10x_rcc.o(.text) for RCC_APB2PeriphResetCmd
    startup_stm32f10x_md.o(RESET) refers to startup_stm32f10x_md.o(STACK) for __initial_sp
    startup_stm32f10x_md.o(RESET) refers to startup_stm32f10x_md.o(.text) for Reset_Handler
    startup_stm32f10x_md.o(RESET) refers to stm32f10x_it.o(.text) for NMI_Handler
    startup_stm32f10x_md.o(.text) refers to system_stm32f10x.o(.text) for SystemInit
    startup_stm32f10x_md.o(.text) refers to entry.o(.ARM.Collect$$$$00000000) for __main
    delay.o(.text) refers to stm32f10x_tim.o(.text) for TIM_Cmd
    delay.o(.text) refers to stm32f10x_rcc.o(.text) for RCC_HCLKConfig
    at.o(.text) refers to sys.o(.text) for uart_recv_clear
    at.o(.text) refers to strlen.o(.text) for strlen
    at.o(.text) refers to memseta.o(.text) for __aeabi_memclr
    at.o(.text) refers to printfa.o(i.__0snprintf) for __2snprintf
    at.o(.text) refers to sys.o(.bss) for uart_recv
    bc26.o(.text) refers to at.o(.text) for at_send_simple_cmd
    bc26.o(.text) refers to memseta.o(.text) for __aeabi_memclr4
    bc26.o(.text) refers to sys.o(.text) for byteToHexStr
    bc26.o(.text) refers to printfa.o(i.__0snprintf) for __2snprintf
    bc26.o(.text) refers to strstr.o(.text) for strstr
    bc26.o(.text) refers to memcpya.o(.text) for __aeabi_memcpy
    bc26.o(.text) refers to stm32f10x_gpio.o(.text) for GPIO_WriteBit
    bc26.o(.text) refers to sys.o(.bss) for uart_recv
    bc26.o(.text) refers to module_wrapper.o(.data) for module_init_status
    bc26.o(.text) refers to module_wrapper.o(.bss) for module_channel
    bc26.o(.text) refers to strlen.o(.text) for strlen
    bc26.o(.text) refers to bc26.o(.data) for event
    bc26.o(.text) refers to module_wrapper.o(.text) for at_module_register
    bc26.o(.data) refers to bc26.o(.conststring) for .conststring
    bc26.o(.data) refers to bc26.o(.text) for bc26_restart_event
    bc26.o(.data) refers to at.o(.text) for at_send_cmd_back
    esp8266.o(.text) refers to memseta.o(.text) for __aeabi_memclr4
    esp8266.o(.text) refers to sys.o(.text) for uart_recv_clear
    esp8266.o(.text) refers to printfa.o(i.__0snprintf) for __2snprintf
    esp8266.o(.text) refers to at.o(.text) for at_send_cmd
    esp8266.o(.text) refers to memcpya.o(.text) for __aeabi_memcpy
    esp8266.o(.text) refers to stm32f10x_rcc.o(.text) for RCC_APB2PeriphClockCmd
    esp8266.o(.text) refers to stm32f10x_gpio.o(.text) for GPIO_Init
    esp8266.o(.text) refers to strstr.o(.text) for strstr
    esp8266.o(.text) refers to sys.o(.bss) for uart_recv
    esp8266.o(.text) refers to module_wrapper.o(.data) for tcp_connect_status
    esp8266.o(.text) refers to module_wrapper.o(.text) for at_module_register
    esp8266.o(.text) refers to esp8266.o(.data) for esp8266_at_event
    esp8266.o(.data) refers to esp8266.o(.conststring) for .conststring
    esp8266.o(.data) refers to esp8266.o(.text) for esp8266_wifi_reconnect_event
    module_wrapper.o(.text) refers to memseta.o(.text) for __aeabi_memclr4
    module_wrapper.o(.text) refers to module_wrapper.o(.bss) for module_channel
    module_wrapper.o(.text) refers to module_wrapper.o(.data) for g_at_module
    cjson.o(.text) refers to scanf_fp.o(.text) for _scanf_real
    cjson.o(.text) refers to printfa.o(i.__0sprintf) for __2sprintf
    cjson.o(.text) refers to tolower.o(.text) for tolower
    cjson.o(.text) refers to strlen.o(.text) for strlen
    cjson.o(.text) refers to memcpya.o(.text) for __aeabi_memcpy
    cjson.o(.text) refers to memseta.o(.text) for __aeabi_memclr4
    cjson.o(.text) refers to strtod.o(i.strtod) for strtod
    cjson.o(.text) refers to cdrcmple.o(.text) for __aeabi_cdrcmple
    cjson.o(.text) refers to cdcmple.o(.text) for __aeabi_cdcmple
    cjson.o(.text) refers to dfixi.o(.text) for __aeabi_d2iz
    cjson.o(.text) refers to strcpy.o(.text) for strcpy
    cjson.o(.text) refers to cjson.o(.data) for global_error
    cjson.o(.text) refers to cjson.o(.bss) for version
    cjson.o(.text) refers to mallocr.o(i.__malloc$realloc) for malloc
    cjson.o(.text) refers to mallocr.o(i.__free$realloc) for free
    cjson.o(.text) refers to mallocr.o(i.realloc) for realloc
    cjson.o(.text) refers to dmul.o(.text) for __aeabi_dmul
    cjson.o(.text) refers to dadd.o(.text) for __aeabi_dsub
    cjson.o(.text) refers to dflti.o(.text) for __aeabi_i2d
    cjson.o(.text) refers to __0sscanf.o(.text) for __0sscanf
    cjson.o(.text) refers to strncmp.o(.text) for strncmp
    cjson.o(.text) refers to strcmp.o(.text) for strcmp
    cjson.o(.text) refers to f2d.o(.text) for __aeabi_f2d
    cjson.o(.data) refers to mallocr.o(i.__malloc$realloc) for malloc
    cjson.o(.data) refers to mallocr.o(i.__free$realloc) for free
    cjson.o(.data) refers to mallocr.o(i.realloc) for realloc
    cjson_utils.o(.text) refers to strlen.o(.text) for strlen
    cjson_utils.o(.text) refers to cjson.o(.text) for cJSON_malloc
    cjson_utils.o(.text) refers to memcpya.o(.text) for __aeabi_memcpy
    cjson_utils.o(.text) refers to strcmp.o(.text) for strcmp
    cjson_utils.o(.text) refers to tolower.o(.text) for tolower
    cjson_utils.o(.text) refers to cdrcmple.o(.text) for __aeabi_cdrcmple
    cjson_utils.o(.text) refers to dmul.o(.text) for __aeabi_dmul
    cjson_utils.o(.text) refers to dadd.o(.text) for __aeabi_dsub
    cjson_utils.o(.text) refers to cdcmple.o(.text) for __aeabi_cdcmple
    cjson_utils.o(.text) refers to printfa.o(i.__0sprintf) for __2sprintf
    cjson_utils.o(.text) refers to strcat.o(.text) for strcat
    cjson_utils.o(.text) refers to strrchr.o(.text) for strrchr
    cjson_utils.o(.text) refers to cjson_utils.o(.constdata) for invalid
    programdata.o(.text) refers to flashsetup.o(.text) for FlashReadOperate
    programdata.o(.text) refers to memseta.o(.text) for __aeabi_memclr
    programdata.o(.text) refers to programdata.o(.bss) for PROGRAM_INFO_DATA
    programdata.o(.data) refers to programdata.o(.bss) for PROGRAM_INFO_DATA
    sys.o(.text) refers to memcpya.o(.text) for __aeabi_memcpy4
    sys.o(.text) refers to strlen.o(.text) for strlen
    sys.o(.text) refers to strtok.o(.text) for strtok
    sys.o(.text) refers to stm32f10x_usart.o(.text) for USART_SendData
    sys.o(.text) refers to printfa.o(i.__0vsnprintf) for vsnprintf
    sys.o(.text) refers to memseta.o(.text) for __aeabi_memclr4
    sys.o(.text) refers to strstr.o(.text) for strstr
    sys.o(.text) refers to sys.o(.bss) for uart_recv
    aes.o(.text) refers to strlen.o(.text) for strlen
    aes.o(.text) refers to memseta.o(.text) for __aeabi_memset
    aes.o(.text) refers to aes.o(.constdata) for sbox
    mbedtls_util.o(.text) refers to strlen.o(.text) for strlen
    mbedtls_util.o(.text) refers to memseta.o(.text) for __aeabi_memset
    mbedtls_util.o(.text) refers to memcpya.o(.text) for __aeabi_memcpy
    mbedtls_util.o(.text) refers to sha1.o(.text) for mbedtls_sha1_init
    mbedtls_util.o(.text) refers to sys.o(.text) for byteToHexStr
    mbedtls_util.o(.text) refers to sha256.o(.text) for mbedtls_sha256_init
    mbedtls_util.o(.text) refers to aes_1.o(.text) for mbedtls_aes_init
    mbedtls_util.o(.text) refers to base64.o(.text) for mbedtls_base64_encode
    mbedtls_util.o(.text) refers to printfa.o(i.__0printf) for __2printf
    coap.o(.text) refers to memcpya.o(.text) for __aeabi_memcpy
    coap.o(.text) refers to strlen.o(.text) for strlen
    coap.o(.text) refers to memcmp.o(.text) for memcmp
    coap.o(.text) refers to coaphandle.o(.bss) for endpoints
    coaphandle.o(.text) refers to memcpya.o(.text) for __aeabi_memcpy
    coaphandle.o(.text) refers to memseta.o(.text) for __aeabi_memclr4
    coaphandle.o(.text) refers to printfa.o(i.__0snprintf) for __2snprintf
    coaphandle.o(.text) refers to strlen.o(.text) for strlen
    coaphandle.o(.text) refers to mbedtls_util.o(.text) for utils_sha256
    coaphandle.o(.text) refers to sys.o(.text) for my_atoi
    coaphandle.o(.text) refers to coap.o(.text) for coap_build
    coaphandle.o(.text) refers to module_wrapper.o(.text) for at_module_send_rai
    coaphandle.o(.text) refers to coaphandle.o(.bss) for auth_token
    coaphandle.o(.text) refers to programdata.o(.data) for registInfo
    coaphandle.o(.text) refers to coaphandle.o(.constdata) for .constdata
    coaphandle.o(.text) refers to coaphandle.o(.data) for send_num
    coaphandle.o(.text) refers to lorawan.o(.data) for send_cont
    coaphandle.o(.text) refers to typedefine.o(.bss) for EngineeringModeValue
    coaphandle.o(.text) refers to module_wrapper.o(.data) for tcp_connect_status
    coaphandle.o(.text) refers to crc.o(.text) for CRC16_CCITT
    coaphandle.o(.text) refers to systemalarm.o(.bss) for sysAlarmFlag
    coaphandle.o(.text) refers to zigbeedatahandle.o(.data) for StartToRun_flag
    coaphandle.o(.text) refers to strstr.o(.text) for strstr
    coaphandle.o(.text) refers to drawlcdgui.o(.text) for DrawSignalDisplay
    coaphandle.o(.text) refers to controlsystem.o(.data) for emSysWorkStep
    coaphandle.o(.text) refers to cjson.o(.text) for cJSON_Parse
    coaphandle.o(.text) refers to driver.o(.text) for SpeakerCtl
    coaphandle.o(.text) refers to stm32f10x_rcc.o(.text) for RCC_APB2PeriphClockCmd
    coaphandle.o(.text) refers to stm32f10x_gpio.o(.text) for GPIO_Init
    coaphandle.o(.text) refers to bc26.o(.text) for bc26_sal_register
    coaphandle.o(.text) refers to sys.o(.bss) for valid_data
    coaphandle.o(.text) refers to typedefine.o(.data) for motorWorkState
    coaphandle.o(.constdata) refers to coaphandle.o(.conststring) for .conststring
    coaphandle.o(.data) refers to coaphandle.o(.conststring) for .conststring
    regist.o(.text) refers to module_wrapper.o(.text) for at_module_start
    regist.o(.text) refers to memseta.o(.text) for __aeabi_memclr4
    regist.o(.text) refers to sys.o(.text) for byteToHexStr
    regist.o(.text) refers to strlen.o(.text) for strlen
    regist.o(.text) refers to strstr.o(.text) for strstr
    regist.o(.text) refers to memcpya.o(.text) for __aeabi_memcpy
    regist.o(.text) refers to printfa.o(i.__0snprintf) for __2snprintf
    regist.o(.text) refers to aes.o(.text) for ECBAesEncrypt
    regist.o(.text) refers to cjson.o(.text) for cJSON_Parse
    regist.o(.text) refers to programdata.o(.text) for WriteProgramData
    regist.o(.text) refers to drawlcdgui.o(.text) for DrawRegistingPicture
    regist.o(.text) refers to typedefine.o(.text) for Delay_ms
    regist.o(.text) refers to typedefine.o(.bss) for TaskSchedulerFlag
    regist.o(.text) refers to regist.o(.data) for registModuleStartCou
    regist.o(.text) refers to module_wrapper.o(.data) for module_start_status
    regist.o(.text) refers to regist.o(.bss) for registData
    regist.o(.text) refers to driver.o(.data) for mcu_id
    regist.o(.text) refers to drawlcdgui.o(.data) for Version_data
    regist.o(.text) refers to sys.o(.bss) for valid_data
    regist.o(.text) refers to programdata.o(.data) for registInfo
    remote.o(.text) refers to module_wrapper.o(.text) for at_module_channel_open
    remote.o(.text) refers to memseta.o(.text) for __aeabi_memclr
    remote.o(.text) refers to strlen.o(.text) for strlen
    remote.o(.text) refers to memcpya.o(.text) for __aeabi_memcpy
    remote.o(.text) refers to sys.o(.text) for byteToHexStr
    remote.o(.text) refers to aes.o(.text) for ECBAesEncrypt
    remote.o(.text) refers to cjson.o(.text) for cJSON_CreateObject
    remote.o(.text) refers to mallocr.o(i.__free$realloc) for free
    remote.o(.text) refers to module_wrapper.o(.data) for module_start_status
    remote.o(.text) refers to module_wrapper.o(.bss) for module_channel
    remote.o(.text) refers to remote.o(.bss) for remoteData
    remote.o(.text) refers to driver.o(.data) for mcu_id
    remote.o(.text) refers to regist.o(.bss) for expansionkey
    remote.o(.text) refers to typedefine.o(.bss) for verifyInfo
    remote.o(.text) refers to remote.o(.data) for remote_flag
    remote.o(.text) refers to regist.o(.data) for key
    aes_1.o(.text) refers to memseta.o(.text) for __aeabi_memclr4
    aes_1.o(.text) refers to platform_util.o(.text) for mbedtls_platform_zeroize
    aes_1.o(.text) refers to aes_1.o(.constdata) for RCON
    aes_1.o(.text) refers to memcpya.o(.text) for __aeabi_memcpy
    base64.o(.text) refers to constant_time.o(.text) for mbedtls_ct_base64_enc_char
    cipher.o(.text) refers to strcmp.o(.text) for strcmp
    cipher.o(.text) refers to memseta.o(.text) for __aeabi_memclr4
    cipher.o(.text) refers to platform_util.o(.text) for mbedtls_platform_zeroize
    cipher.o(.text) refers to memcpya.o(.text) for __aeabi_memcpy
    cipher.o(.text) refers to cipher.o(.data) for supported_init
    cipher.o(.text) refers to cipher_wrap.o(.constdata) for mbedtls_cipher_definitions
    cipher.o(.text) refers to cipher_wrap.o(.bss) for mbedtls_cipher_supported
    cipher_wrap.o(.text) refers to aes_1.o(.text) for mbedtls_aes_crypt_ecb
    cipher_wrap.o(.text) refers to calloc.o(.text) for calloc
    cipher_wrap.o(.text) refers to mallocr.o(i.__free$realloc) for free
    cipher_wrap.o(.constdata) refers to cipher_wrap.o(.text) for aes_crypt_ecb_wrap
    cipher_wrap.o(.constdata) refers to cipher_wrap.o(.conststring) for .conststring
    platform_util.o(.text) refers to platform_util.o(.data) for memset_func
    platform_util.o(.data) refers to memseta.o(.text) for memset
    sha1.o(.text) refers to memseta.o(.text) for __aeabi_memclr4
    sha1.o(.text) refers to platform_util.o(.text) for mbedtls_platform_zeroize
    sha1.o(.text) refers to memcpya.o(.text) for __aeabi_memcpy4
    sha256.o(.text) refers to memseta.o(.text) for __aeabi_memclr4
    sha256.o(.text) refers to platform_util.o(.text) for mbedtls_platform_zeroize
    sha256.o(.text) refers to memcpya.o(.text) for __aeabi_memcpy4
    sha256.o(.text) refers to sha256.o(.constdata) for K
    strtod.o(i.__softfp_strtod) refers (Special) to iusefp.o(.text) for __I$use$fp
    strtod.o(i.__softfp_strtod) refers to strtod.o(.text) for __strtod_int
    strtod.o(i.strtod) refers (Special) to iusefp.o(.text) for __I$use$fp
    strtod.o(i.strtod) refers to strtod.o(.text) for __strtod_int
    entry.o(.ARM.Collect$$$$00000000) refers (Special) to entry10a.o(.ARM.Collect$$$$0000000D) for __rt_final_cpp
    entry.o(.ARM.Collect$$$$00000000) refers (Special) to entry11a.o(.ARM.Collect$$$$0000000F) for __rt_final_exit
    entry.o(.ARM.Collect$$$$00000000) refers (Special) to entry7b.o(.ARM.Collect$$$$00000008) for _main_clock
    entry.o(.ARM.Collect$$$$00000000) refers (Special) to entry8b.o(.ARM.Collect$$$$0000000A) for _main_cpp_init
    entry.o(.ARM.Collect$$$$00000000) refers (Special) to entry9a.o(.ARM.Collect$$$$0000000B) for _main_init
    entry.o(.ARM.Collect$$$$00000000) refers (Special) to entry5.o(.ARM.Collect$$$$00000004) for _main_scatterload
    entry.o(.ARM.Collect$$$$00000000) refers (Special) to entry2.o(.ARM.Collect$$$$00000001) for _main_stk
    uldiv.o(.text) refers to llushr.o(.text) for __aeabi_llsr
    uldiv.o(.text) refers to llshl.o(.text) for __aeabi_llsl
    rand.o(.text) refers to rand.o(.data) for .data
    strtok.o(.text) refers to strtok.o(.data) for .data
    strtok_r.o(.text) refers to strtok_r.o(.data) for .data
    printfb.o(i.__0fprintf$bare) refers to printfb.o(i._printf_core) for _printf_core
    printfb.o(i.__0fprintf$bare) refers to controlsystem.o(.text) for fputc
    printfb.o(i.__0printf$bare) refers to printfb.o(i._printf_core) for _printf_core
    printfb.o(i.__0printf$bare) refers to controlsystem.o(.text) for fputc
    printfb.o(i.__0printf$bare) refers to stdout.o(.data) for __stdout
    printfb.o(i.__0snprintf$bare) refers to printfb.o(i._printf_core) for _printf_core
    printfb.o(i.__0snprintf$bare) refers to printfb.o(i._snputc) for _snputc
    printfb.o(i.__0sprintf$bare) refers to printfb.o(i._printf_core) for _printf_core
    printfb.o(i.__0sprintf$bare) refers to printfb.o(i._sputc) for _sputc
    printfb.o(i.__0vfprintf$bare) refers to printfb.o(i._printf_core) for _printf_core
    printfb.o(i.__0vfprintf$bare) refers to controlsystem.o(.text) for fputc
    printfb.o(i.__0vprintf$bare) refers to printfb.o(i._printf_core) for _printf_core
    printfb.o(i.__0vprintf$bare) refers to controlsystem.o(.text) for fputc
    printfb.o(i.__0vprintf$bare) refers to stdout.o(.data) for __stdout
    printfb.o(i.__0vsnprintf$bare) refers to printfb.o(i._printf_core) for _printf_core
    printfb.o(i.__0vsnprintf$bare) refers to printfb.o(i._snputc) for _snputc
    printfb.o(i.__0vsprintf$bare) refers to printfb.o(i._printf_core) for _printf_core
    printfb.o(i.__0vsprintf$bare) refers to printfb.o(i._sputc) for _sputc
    printf0.o(i.__0fprintf$0) refers to printf0.o(i._printf_core) for _printf_core
    printf0.o(i.__0fprintf$0) refers to controlsystem.o(.text) for fputc
    printf0.o(i.__0printf$0) refers to printf0.o(i._printf_core) for _printf_core
    printf0.o(i.__0printf$0) refers to controlsystem.o(.text) for fputc
    printf0.o(i.__0printf$0) refers to stdout.o(.data) for __stdout
    printf0.o(i.__0snprintf$0) refers to printf0.o(i._printf_core) for _printf_core
    printf0.o(i.__0snprintf$0) refers to printf0.o(i._snputc) for _snputc
    printf0.o(i.__0sprintf$0) refers to printf0.o(i._printf_core) for _printf_core
    printf0.o(i.__0sprintf$0) refers to printf0.o(i._sputc) for _sputc
    printf0.o(i.__0vfprintf$0) refers to printf0.o(i._printf_core) for _printf_core
    printf0.o(i.__0vfprintf$0) refers to controlsystem.o(.text) for fputc
    printf0.o(i.__0vprintf$0) refers to printf0.o(i._printf_core) for _printf_core
    printf0.o(i.__0vprintf$0) refers to controlsystem.o(.text) for fputc
    printf0.o(i.__0vprintf$0) refers to stdout.o(.data) for __stdout
    printf0.o(i.__0vsnprintf$0) refers to printf0.o(i._printf_core) for _printf_core
    printf0.o(i.__0vsnprintf$0) refers to printf0.o(i._snputc) for _snputc
    printf0.o(i.__0vsprintf$0) refers to printf0.o(i._printf_core) for _printf_core
    printf0.o(i.__0vsprintf$0) refers to printf0.o(i._sputc) for _sputc
    printf1.o(i.__0fprintf$1) refers to printf1.o(i._printf_core) for _printf_core
    printf1.o(i.__0fprintf$1) refers to controlsystem.o(.text) for fputc
    printf1.o(i.__0printf$1) refers to printf1.o(i._printf_core) for _printf_core
    printf1.o(i.__0printf$1) refers to controlsystem.o(.text) for fputc
    printf1.o(i.__0printf$1) refers to stdout.o(.data) for __stdout
    printf1.o(i.__0snprintf$1) refers to printf1.o(i._printf_core) for _printf_core
    printf1.o(i.__0snprintf$1) refers to printf1.o(i._snputc) for _snputc
    printf1.o(i.__0sprintf$1) refers to printf1.o(i._printf_core) for _printf_core
    printf1.o(i.__0sprintf$1) refers to printf1.o(i._sputc) for _sputc
    printf1.o(i.__0vfprintf$1) refers to printf1.o(i._printf_core) for _printf_core
    printf1.o(i.__0vfprintf$1) refers to controlsystem.o(.text) for fputc
    printf1.o(i.__0vprintf$1) refers to printf1.o(i._printf_core) for _printf_core
    printf1.o(i.__0vprintf$1) refers to controlsystem.o(.text) for fputc
    printf1.o(i.__0vprintf$1) refers to stdout.o(.data) for __stdout
    printf1.o(i.__0vsnprintf$1) refers to printf1.o(i._printf_core) for _printf_core
    printf1.o(i.__0vsnprintf$1) refers to printf1.o(i._snputc) for _snputc
    printf1.o(i.__0vsprintf$1) refers to printf1.o(i._printf_core) for _printf_core
    printf1.o(i.__0vsprintf$1) refers to printf1.o(i._sputc) for _sputc
    printf1.o(i._printf_core) refers to uidiv.o(.text) for __aeabi_uidivmod
    printf2.o(i.__0fprintf$2) refers to printf2.o(i._printf_core) for _printf_core
    printf2.o(i.__0fprintf$2) refers to controlsystem.o(.text) for fputc
    printf2.o(i.__0printf$2) refers to printf2.o(i._printf_core) for _printf_core
    printf2.o(i.__0printf$2) refers to controlsystem.o(.text) for fputc
    printf2.o(i.__0printf$2) refers to stdout.o(.data) for __stdout
    printf2.o(i.__0snprintf$2) refers to printf2.o(i._printf_core) for _printf_core
    printf2.o(i.__0snprintf$2) refers to printf2.o(i._snputc) for _snputc
    printf2.o(i.__0sprintf$2) refers to printf2.o(i._printf_core) for _printf_core
    printf2.o(i.__0sprintf$2) refers to printf2.o(i._sputc) for _sputc
    printf2.o(i.__0vfprintf$2) refers to printf2.o(i._printf_core) for _printf_core
    printf2.o(i.__0vfprintf$2) refers to controlsystem.o(.text) for fputc
    printf2.o(i.__0vprintf$2) refers to printf2.o(i._printf_core) for _printf_core
    printf2.o(i.__0vprintf$2) refers to controlsystem.o(.text) for fputc
    printf2.o(i.__0vprintf$2) refers to stdout.o(.data) for __stdout
    printf2.o(i.__0vsnprintf$2) refers to printf2.o(i._printf_core) for _printf_core
    printf2.o(i.__0vsnprintf$2) refers to printf2.o(i._snputc) for _snputc
    printf2.o(i.__0vsprintf$2) refers to printf2.o(i._printf_core) for _printf_core
    printf2.o(i.__0vsprintf$2) refers to printf2.o(i._sputc) for _sputc
    printf3.o(i.__0fprintf$3) refers to printf3.o(i._printf_core) for _printf_core
    printf3.o(i.__0fprintf$3) refers to controlsystem.o(.text) for fputc
    printf3.o(i.__0printf$3) refers to printf3.o(i._printf_core) for _printf_core
    printf3.o(i.__0printf$3) refers to controlsystem.o(.text) for fputc
    printf3.o(i.__0printf$3) refers to stdout.o(.data) for __stdout
    printf3.o(i.__0snprintf$3) refers to printf3.o(i._printf_core) for _printf_core
    printf3.o(i.__0snprintf$3) refers to printf3.o(i._snputc) for _snputc
    printf3.o(i.__0sprintf$3) refers to printf3.o(i._printf_core) for _printf_core
    printf3.o(i.__0sprintf$3) refers to printf3.o(i._sputc) for _sputc
    printf3.o(i.__0vfprintf$3) refers to printf3.o(i._printf_core) for _printf_core
    printf3.o(i.__0vfprintf$3) refers to controlsystem.o(.text) for fputc
    printf3.o(i.__0vprintf$3) refers to printf3.o(i._printf_core) for _printf_core
    printf3.o(i.__0vprintf$3) refers to controlsystem.o(.text) for fputc
    printf3.o(i.__0vprintf$3) refers to stdout.o(.data) for __stdout
    printf3.o(i.__0vsnprintf$3) refers to printf3.o(i._printf_core) for _printf_core
    printf3.o(i.__0vsnprintf$3) refers to printf3.o(i._snputc) for _snputc
    printf3.o(i.__0vsprintf$3) refers to printf3.o(i._printf_core) for _printf_core
    printf3.o(i.__0vsprintf$3) refers to printf3.o(i._sputc) for _sputc
    printf3.o(i._printf_core) refers to uidiv.o(.text) for __aeabi_uidivmod
    printf4.o(i.__0fprintf$4) refers to printf4.o(i._printf_core) for _printf_core
    printf4.o(i.__0fprintf$4) refers to controlsystem.o(.text) for fputc
    printf4.o(i.__0printf$4) refers to printf4.o(i._printf_core) for _printf_core
    printf4.o(i.__0printf$4) refers to controlsystem.o(.text) for fputc
    printf4.o(i.__0printf$4) refers to stdout.o(.data) for __stdout
    printf4.o(i.__0snprintf$4) refers to printf4.o(i._printf_core) for _printf_core
    printf4.o(i.__0snprintf$4) refers to printf4.o(i._snputc) for _snputc
    printf4.o(i.__0sprintf$4) refers to printf4.o(i._printf_core) for _printf_core
    printf4.o(i.__0sprintf$4) refers to printf4.o(i._sputc) for _sputc
    printf4.o(i.__0vfprintf$4) refers to printf4.o(i._printf_core) for _printf_core
    printf4.o(i.__0vfprintf$4) refers to controlsystem.o(.text) for fputc
    printf4.o(i.__0vprintf$4) refers to printf4.o(i._printf_core) for _printf_core
    printf4.o(i.__0vprintf$4) refers to controlsystem.o(.text) for fputc
    printf4.o(i.__0vprintf$4) refers to stdout.o(.data) for __stdout
    printf4.o(i.__0vsnprintf$4) refers to printf4.o(i._printf_core) for _printf_core
    printf4.o(i.__0vsnprintf$4) refers to printf4.o(i._snputc) for _snputc
    printf4.o(i.__0vsprintf$4) refers to printf4.o(i._printf_core) for _printf_core
    printf4.o(i.__0vsprintf$4) refers to printf4.o(i._sputc) for _sputc
    printf4.o(i._printf_core) refers to uldiv.o(.text) for __aeabi_uldivmod
    printf5.o(i.__0fprintf$5) refers to printf5.o(i._printf_core) for _printf_core
    printf5.o(i.__0fprintf$5) refers to controlsystem.o(.text) for fputc
    printf5.o(i.__0printf$5) refers to printf5.o(i._printf_core) for _printf_core
    printf5.o(i.__0printf$5) refers to controlsystem.o(.text) for fputc
    printf5.o(i.__0printf$5) refers to stdout.o(.data) for __stdout
    printf5.o(i.__0snprintf$5) refers to printf5.o(i._printf_core) for _printf_core
    printf5.o(i.__0snprintf$5) refers to printf5.o(i._snputc) for _snputc
    printf5.o(i.__0sprintf$5) refers to printf5.o(i._printf_core) for _printf_core
    printf5.o(i.__0sprintf$5) refers to printf5.o(i._sputc) for _sputc
    printf5.o(i.__0vfprintf$5) refers to printf5.o(i._printf_core) for _printf_core
    printf5.o(i.__0vfprintf$5) refers to controlsystem.o(.text) for fputc
    printf5.o(i.__0vprintf$5) refers to printf5.o(i._printf_core) for _printf_core
    printf5.o(i.__0vprintf$5) refers to controlsystem.o(.text) for fputc
    printf5.o(i.__0vprintf$5) refers to stdout.o(.data) for __stdout
    printf5.o(i.__0vsnprintf$5) refers to printf5.o(i._printf_core) for _printf_core
    printf5.o(i.__0vsnprintf$5) refers to printf5.o(i._snputc) for _snputc
    printf5.o(i.__0vsprintf$5) refers to printf5.o(i._printf_core) for _printf_core
    printf5.o(i.__0vsprintf$5) refers to printf5.o(i._sputc) for _sputc
    printf5.o(i._printf_core) refers to uldiv.o(.text) for __aeabi_uldivmod
    printf6.o(i.__0fprintf$6) refers to printf6.o(i._printf_core) for _printf_core
    printf6.o(i.__0fprintf$6) refers to controlsystem.o(.text) for fputc
    printf6.o(i.__0printf$6) refers to printf6.o(i._printf_core) for _printf_core
    printf6.o(i.__0printf$6) refers to controlsystem.o(.text) for fputc
    printf6.o(i.__0printf$6) refers to stdout.o(.data) for __stdout
    printf6.o(i.__0snprintf$6) refers to printf6.o(i._printf_core) for _printf_core
    printf6.o(i.__0snprintf$6) refers to printf6.o(i._snputc) for _snputc
    printf6.o(i.__0sprintf$6) refers to printf6.o(i._printf_core) for _printf_core
    printf6.o(i.__0sprintf$6) refers to printf6.o(i._sputc) for _sputc
    printf6.o(i.__0vfprintf$6) refers to printf6.o(i._printf_core) for _printf_core
    printf6.o(i.__0vfprintf$6) refers to controlsystem.o(.text) for fputc
    printf6.o(i.__0vprintf$6) refers to printf6.o(i._printf_core) for _printf_core
    printf6.o(i.__0vprintf$6) refers to controlsystem.o(.text) for fputc
    printf6.o(i.__0vprintf$6) refers to stdout.o(.data) for __stdout
    printf6.o(i.__0vsnprintf$6) refers to printf6.o(i._printf_core) for _printf_core
    printf6.o(i.__0vsnprintf$6) refers to printf6.o(i._snputc) for _snputc
    printf6.o(i.__0vsprintf$6) refers to printf6.o(i._printf_core) for _printf_core
    printf6.o(i.__0vsprintf$6) refers to printf6.o(i._sputc) for _sputc
    printf6.o(i._printf_core) refers to printf6.o(i._printf_pre_padding) for _printf_pre_padding
    printf6.o(i._printf_core) refers to uidiv.o(.text) for __aeabi_uidivmod
    printf6.o(i._printf_core) refers to printf6.o(i._printf_post_padding) for _printf_post_padding
    printf7.o(i.__0fprintf$7) refers to printf7.o(i._printf_core) for _printf_core
    printf7.o(i.__0fprintf$7) refers to controlsystem.o(.text) for fputc
    printf7.o(i.__0printf$7) refers to printf7.o(i._printf_core) for _printf_core
    printf7.o(i.__0printf$7) refers to controlsystem.o(.text) for fputc
    printf7.o(i.__0printf$7) refers to stdout.o(.data) for __stdout
    printf7.o(i.__0snprintf$7) refers to printf7.o(i._printf_core) for _printf_core
    printf7.o(i.__0snprintf$7) refers to printf7.o(i._snputc) for _snputc
    printf7.o(i.__0sprintf$7) refers to printf7.o(i._printf_core) for _printf_core
    printf7.o(i.__0sprintf$7) refers to printf7.o(i._sputc) for _sputc
    printf7.o(i.__0vfprintf$7) refers to printf7.o(i._printf_core) for _printf_core
    printf7.o(i.__0vfprintf$7) refers to controlsystem.o(.text) for fputc
    printf7.o(i.__0vprintf$7) refers to printf7.o(i._printf_core) for _printf_core
    printf7.o(i.__0vprintf$7) refers to controlsystem.o(.text) for fputc
    printf7.o(i.__0vprintf$7) refers to stdout.o(.data) for __stdout
    printf7.o(i.__0vsnprintf$7) refers to printf7.o(i._printf_core) for _printf_core
    printf7.o(i.__0vsnprintf$7) refers to printf7.o(i._snputc) for _snputc
    printf7.o(i.__0vsprintf$7) refers to printf7.o(i._printf_core) for _printf_core
    printf7.o(i.__0vsprintf$7) refers to printf7.o(i._sputc) for _sputc
    printf7.o(i._printf_core) refers to printf7.o(i._printf_pre_padding) for _printf_pre_padding
    printf7.o(i._printf_core) refers to uldiv.o(.text) for __aeabi_uldivmod
    printf7.o(i._printf_core) refers to printf7.o(i._printf_post_padding) for _printf_post_padding
    printf8.o(i.__0fprintf$8) refers to printf8.o(i._printf_core) for _printf_core
    printf8.o(i.__0fprintf$8) refers to controlsystem.o(.text) for fputc
    printf8.o(i.__0printf$8) refers to printf8.o(i._printf_core) for _printf_core
    printf8.o(i.__0printf$8) refers to controlsystem.o(.text) for fputc
    printf8.o(i.__0printf$8) refers to stdout.o(.data) for __stdout
    printf8.o(i.__0snprintf$8) refers to printf8.o(i._printf_core) for _printf_core
    printf8.o(i.__0snprintf$8) refers to printf8.o(i._snputc) for _snputc
    printf8.o(i.__0sprintf$8) refers to printf8.o(i._printf_core) for _printf_core
    printf8.o(i.__0sprintf$8) refers to printf8.o(i._sputc) for _sputc
    printf8.o(i.__0vfprintf$8) refers to printf8.o(i._printf_core) for _printf_core
    printf8.o(i.__0vfprintf$8) refers to controlsystem.o(.text) for fputc
    printf8.o(i.__0vprintf$8) refers to printf8.o(i._printf_core) for _printf_core
    printf8.o(i.__0vprintf$8) refers to controlsystem.o(.text) for fputc
    printf8.o(i.__0vprintf$8) refers to stdout.o(.data) for __stdout
    printf8.o(i.__0vsnprintf$8) refers to printf8.o(i._printf_core) for _printf_core
    printf8.o(i.__0vsnprintf$8) refers to printf8.o(i._snputc) for _snputc
    printf8.o(i.__0vsprintf$8) refers to printf8.o(i._printf_core) for _printf_core
    printf8.o(i.__0vsprintf$8) refers to printf8.o(i._sputc) for _sputc
    printf8.o(i._printf_core) refers to printf8.o(i._printf_pre_padding) for _printf_pre_padding
    printf8.o(i._printf_core) refers to uldiv.o(.text) for __aeabi_uldivmod
    printf8.o(i._printf_core) refers to printf8.o(i._printf_post_padding) for _printf_post_padding
    printfa.o(i.__0fprintf) refers (Special) to iusefp.o(.text) for __I$use$fp
    printfa.o(i.__0fprintf) refers to printfa.o(i._printf_core) for _printf_core
    printfa.o(i.__0fprintf) refers to controlsystem.o(.text) for fputc
    printfa.o(i.__0printf) refers (Special) to iusefp.o(.text) for __I$use$fp
    printfa.o(i.__0printf) refers to printfa.o(i._printf_core) for _printf_core
    printfa.o(i.__0printf) refers to controlsystem.o(.text) for fputc
    printfa.o(i.__0printf) refers to stdout.o(.data) for __stdout
    printfa.o(i.__0snprintf) refers (Special) to iusefp.o(.text) for __I$use$fp
    printfa.o(i.__0snprintf) refers to printfa.o(i._printf_core) for _printf_core
    printfa.o(i.__0snprintf) refers to printfa.o(i._snputc) for _snputc
    printfa.o(i.__0sprintf) refers (Special) to iusefp.o(.text) for __I$use$fp
    printfa.o(i.__0sprintf) refers to printfa.o(i._printf_core) for _printf_core
    printfa.o(i.__0sprintf) refers to printfa.o(i._sputc) for _sputc
    printfa.o(i.__0vfprintf) refers (Special) to iusefp.o(.text) for __I$use$fp
    printfa.o(i.__0vfprintf) refers to printfa.o(i._printf_core) for _printf_core
    printfa.o(i.__0vfprintf) refers to controlsystem.o(.text) for fputc
    printfa.o(i.__0vprintf) refers (Special) to iusefp.o(.text) for __I$use$fp
    printfa.o(i.__0vprintf) refers to printfa.o(i._printf_core) for _printf_core
    printfa.o(i.__0vprintf) refers to controlsystem.o(.text) for fputc
    printfa.o(i.__0vprintf) refers to stdout.o(.data) for __stdout
    printfa.o(i.__0vsnprintf) refers (Special) to iusefp.o(.text) for __I$use$fp
    printfa.o(i.__0vsnprintf) refers to printfa.o(i._printf_core) for _printf_core
    printfa.o(i.__0vsnprintf) refers to printfa.o(i._snputc) for _snputc
    printfa.o(i.__0vsprintf) refers (Special) to iusefp.o(.text) for __I$use$fp
    printfa.o(i.__0vsprintf) refers to printfa.o(i._printf_core) for _printf_core
    printfa.o(i.__0vsprintf) refers to printfa.o(i._sputc) for _sputc
    printfa.o(i._fp_digits) refers (Special) to iusefp.o(.text) for __I$use$fp
    printfa.o(i._fp_digits) refers to dmul.o(.text) for __aeabi_dmul
    printfa.o(i._fp_digits) refers to ddiv.o(.text) for __aeabi_ddiv
    printfa.o(i._fp_digits) refers to cdrcmple.o(.text) for __aeabi_cdrcmple
    printfa.o(i._fp_digits) refers to dadd.o(.text) for __aeabi_dadd
    printfa.o(i._fp_digits) refers to dfixul.o(.text) for __aeabi_d2ulz
    printfa.o(i._fp_digits) refers to uldiv.o(.text) for __aeabi_uldivmod
    printfa.o(i._printf_core) refers (Special) to iusefp.o(.text) for __I$use$fp
    printfa.o(i._printf_core) refers to printfa.o(i._printf_pre_padding) for _printf_pre_padding
    printfa.o(i._printf_core) refers to uldiv.o(.text) for __aeabi_uldivmod
    printfa.o(i._printf_core) refers to printfa.o(i._printf_post_padding) for _printf_post_padding
    printfa.o(i._printf_core) refers to printfa.o(i._fp_digits) for _fp_digits
    printfa.o(i._printf_core) refers to uidiv.o(.text) for __aeabi_uidivmod
    printfa.o(i._printf_post_padding) refers (Special) to iusefp.o(.text) for __I$use$fp
    printfa.o(i._printf_pre_padding) refers (Special) to iusefp.o(.text) for __I$use$fp
    printfa.o(i._snputc) refers (Special) to iusefp.o(.text) for __I$use$fp
    printfa.o(i._sputc) refers (Special) to iusefp.o(.text) for __I$use$fp
    malloc.o(i.free) refers to mvars.o(.data) for __microlib_freelist
    malloc.o(i.malloc) refers to mvars.o(.data) for __microlib_freelist_initialised
    malloc.o(i.malloc) refers to mvars.o(.data) for __microlib_freelist
    malloc.o(i.malloc) refers to startup_stm32f10x_md.o(HEAP) for __heap_base
    mallocr.o(i.__free$realloc) refers to mvars.o(.data) for __microlib_freelist
    mallocr.o(i.__malloc$realloc) refers to mallocr.o(i.internal_alloc) for internal_alloc
    mallocr.o(i.__malloc$realloc) refers to mvars.o(.data) for __microlib_freelist_initialised
    mallocr.o(i.__malloc$realloc) refers to startup_stm32f10x_md.o(HEAP) for __heap_base
    mallocr.o(i.__malloc$realloc) refers to mvars.o(.data) for __microlib_freelist
    mallocr.o(i.internal_alloc) refers to memcpya.o(.text) for __aeabi_memcpy
    mallocr.o(i.internal_alloc) refers to mvars.o(.data) for __microlib_freelist
    mallocr.o(i.realloc) refers to mallocr.o(i.__free$realloc) for free
    mallocr.o(i.realloc) refers to mallocr.o(i.internal_alloc) for internal_alloc
    mallocr.o(i.realloc) refers to mallocr.o(i.__malloc$realloc) for malloc
    mallocr.o(i.realloc) refers to mvars.o(.data) for __microlib_freelist
    malloca.o(i.__aligned_malloc) refers to mvars.o(.data) for __microlib_freelist_initialised
    malloca.o(i.__aligned_malloc) refers to mvars.o(.data) for __microlib_freelist
    malloca.o(i.__aligned_malloc) refers to startup_stm32f10x_md.o(HEAP) for __heap_base
    malloca.o(i.__free$memalign) refers to mvars.o(.data) for __microlib_freelist
    malloca.o(i.__malloc$memalign) refers to malloca.o(i.__aligned_malloc) for __aligned_malloc
    mallocra.o(i.__aligned_malloc$realloc) refers to mallocra.o(i.internal_alloc) for internal_alloc
    mallocra.o(i.__aligned_malloc$realloc) refers to mvars.o(.data) for __microlib_freelist_initialised
    mallocra.o(i.__aligned_malloc$realloc) refers to startup_stm32f10x_md.o(HEAP) for __heap_base
    mallocra.o(i.__aligned_malloc$realloc) refers to mvars.o(.data) for __microlib_freelist
    mallocra.o(i.__free$realloc$memalign) refers to mvars.o(.data) for __microlib_freelist
    mallocra.o(i.__malloc$realloc$memalign) refers to mallocra.o(i.__aligned_malloc$realloc) for __aligned_malloc$realloc
    mallocra.o(i.__realloc$memalign) refers to mallocra.o(i.__free$realloc$memalign) for __free$realloc$memalign
    mallocra.o(i.__realloc$memalign) refers to mallocra.o(i.internal_alloc) for internal_alloc
    mallocra.o(i.__realloc$memalign) refers to mallocra.o(i.__malloc$realloc$memalign) for __malloc$realloc$memalign
    mallocra.o(i.__realloc$memalign) refers to mvars.o(.data) for __microlib_freelist
    mallocra.o(i.internal_alloc) refers to memcpya.o(.text) for __aeabi_memcpy
    mallocra.o(i.internal_alloc) refers to mvars.o(.data) for __microlib_freelist
    calloc.o(.text) refers to mallocr.o(i.__malloc$realloc) for malloc
    __0sscanf.o(.text) refers to scanf_char.o(.text) for __vfscanf_char
    __0sscanf.o(.text) refers to _sgetc.o(.text) for _sgetc
    scanf_fp.o(.text) refers (Special) to iusefp.o(.text) for __I$use$fp
    scanf_fp.o(.text) refers to dfltul.o(.text) for __aeabi_ul2d
    scanf_fp.o(.text) refers to dmul.o(.text) for __aeabi_dmul
    scanf_fp.o(.text) refers to ddiv.o(.text) for __aeabi_ddiv
    scanf_fp.o(.text) refers to scanf_fp.o(i._is_digit) for _is_digit
    scanf_fp.o(.text) refers to d2f.o(.text) for __aeabi_d2f
    dadd.o(.text) refers (Special) to iusefp.o(.text) for __I$use$fp
    dadd.o(.text) refers to llshl.o(.text) for __aeabi_llsl
    dadd.o(.text) refers to llsshr.o(.text) for __aeabi_lasr
    dadd.o(.text) refers to depilogue.o(.text) for _double_epilogue
    dmul.o(.text) refers (Special) to iusefp.o(.text) for __I$use$fp
    dmul.o(.text) refers to depilogue.o(.text) for _double_epilogue
    dflti.o(.text) refers (Special) to iusefp.o(.text) for __I$use$fp
    dflti.o(.text) refers to depilogue.o(.text) for _double_epilogue
    dfixi.o(.text) refers (Special) to iusefp.o(.text) for __I$use$fp
    dfixi.o(.text) refers to llushr.o(.text) for __aeabi_llsr
    f2d.o(.text) refers (Special) to iusefp.o(.text) for __I$use$fp
    cdcmple.o(.text) refers (Special) to iusefp.o(.text) for __I$use$fp
    cdrcmple.o(.text) refers (Special) to iusefp.o(.text) for __I$use$fp
    entry2.o(.ARM.Collect$$$$00000001) refers to entry2.o(.ARM.Collect$$$$00002712) for __lit__00000000
    entry2.o(.ARM.Collect$$$$00002712) refers to startup_stm32f10x_md.o(STACK) for __initial_sp
    entry2.o(__vectab_stack_and_reset_area) refers to startup_stm32f10x_md.o(STACK) for __initial_sp
    entry2.o(__vectab_stack_and_reset_area) refers to entry.o(.ARM.Collect$$$$00000000) for __main
    entry5.o(.ARM.Collect$$$$00000004) refers to init.o(.text) for __scatterload
    entry9a.o(.ARM.Collect$$$$0000000B) refers to main.o(.text) for main
    entry9b.o(.ARM.Collect$$$$0000000C) refers to main.o(.text) for main
    scanf_char.o(.text) refers to _scanf.o(.text) for __vfscanf
    scanf_char.o(.text) refers to isspace_c.o(.text) for isspace
    strtod.o(.text) refers to scanf_fp.o(.text) for _scanf_real
    strtod.o(.text) refers to _sgetc.o(.text) for _sgetc
    strtod.o(.text) refers to isspace_c.o(.text) for isspace
    depilogue.o(.text) refers to llshl.o(.text) for __aeabi_llsl
    depilogue.o(.text) refers to llushr.o(.text) for __aeabi_llsr
    ddiv.o(.text) refers to depilogue.o(.text) for _double_round
    dfltul.o(.text) refers to depilogue.o(.text) for _double_epilogue
    dfixul.o(.text) refers to llushr.o(.text) for __aeabi_llsr
    dfixul.o(.text) refers to llshl.o(.text) for __aeabi_llsl
    d2f.o(.text) refers to fepilogue.o(.text) for _float_round
    init.o(.text) refers to entry5.o(.ARM.Collect$$$$00000004) for __main_after_scatterload
    isspace_c.o(.text) refers to ctype_c.o(.text) for __ctype_lookup
    _scanf.o(.text) refers (Weak) to scanf_fp.o(.text) for _scanf_real
    ctype_c.o(.text) refers to ctype_c.o(.constdata) for .constdata
    scanf_fp.o(i._is_digit) refers (Special) to iusefp.o(.text) for __I$use$fp


==============================================================================

Removing Unused input sections from the image.

    Removing main.o(.data), (50 bytes).
    Removing timersetup.o(.text), (140 bytes).
    Removing ads1110asetup.o(.text), (116 bytes).
    Removing iic2setup.o(.text), (616 bytes).
    Removing core_cm3.o(.emb_text), (32 bytes).
    Removing esp8266.o(.text), (1780 bytes).
    Removing esp8266.o(.conststring), (70 bytes).
    Removing esp8266.o(.data), (128 bytes).
    Removing cjson_utils.o(.text), (4244 bytes).
    Removing cjson_utils.o(.constdata), (40 bytes).
    Removing cipher.o(.text), (1484 bytes).
    Removing cipher.o(.data), (4 bytes).
    Removing cipher_wrap.o(.text), (152 bytes).
    Removing cipher_wrap.o(.bss), (28 bytes).
    Removing cipher_wrap.o(.constdata), (252 bytes).
    Removing cipher_wrap.o(.conststring), (72 bytes).

16 unused section(s) (total 9208 bytes) removed from the image.

==============================================================================

Image Symbol Table

    Local Symbols

    Symbol Name                              Value     Ov Type        Size  Object(Section)

    ../clib/../cmprslib/zerorunl2.c          0x00000000   Number         0  __dczerorl2.o ABSOLUTE
    ../clib/microlib/ctype/ctype.c           0x00000000   Number         0  isspace_c.o ABSOLUTE
    ../clib/microlib/ctype/ctype.c           0x00000000   Number         0  ctype_c.o ABSOLUTE
    ../clib/microlib/ctype/tolower.c         0x00000000   Number         0  tolower.o ABSOLUTE
    ../clib/microlib/division.c              0x00000000   Number         0  uidiv.o ABSOLUTE
    ../clib/microlib/division.c              0x00000000   Number         0  uldiv.o ABSOLUTE
    ../clib/microlib/init/entry.s            0x00000000   Number         0  entry11b.o ABSOLUTE
    ../clib/microlib/init/entry.s            0x00000000   Number         0  entry.o ABSOLUTE
    ../clib/microlib/init/entry.s            0x00000000   Number         0  entry11a.o ABSOLUTE
    ../clib/microlib/init/entry.s            0x00000000   Number         0  entry10b.o ABSOLUTE
    ../clib/microlib/init/entry.s            0x00000000   Number         0  entry10a.o ABSOLUTE
    ../clib/microlib/init/entry.s            0x00000000   Number         0  entry9b.o ABSOLUTE
    ../clib/microlib/init/entry.s            0x00000000   Number         0  entry2.o ABSOLUTE
    ../clib/microlib/init/entry.s            0x00000000   Number         0  entry9a.o ABSOLUTE
    ../clib/microlib/init/entry.s            0x00000000   Number         0  entry8b.o ABSOLUTE
    ../clib/microlib/init/entry.s            0x00000000   Number         0  entry8a.o ABSOLUTE
    ../clib/microlib/init/entry.s            0x00000000   Number         0  entry7b.o ABSOLUTE
    ../clib/microlib/init/entry.s            0x00000000   Number         0  entry7a.o ABSOLUTE
    ../clib/microlib/init/entry.s            0x00000000   Number         0  entry5.o ABSOLUTE
    ../clib/microlib/longlong.c              0x00000000   Number         0  llushr.o ABSOLUTE
    ../clib/microlib/longlong.c              0x00000000   Number         0  llsshr.o ABSOLUTE
    ../clib/microlib/longlong.c              0x00000000   Number         0  llshl.o ABSOLUTE
    ../clib/microlib/malloc/calloc.c         0x00000000   Number         0  calloc.o ABSOLUTE
    ../clib/microlib/malloc/malloc.c         0x00000000   Number         0  malloc.o ABSOLUTE
    ../clib/microlib/malloc/malloc.c         0x00000000   Number         0  mallocr.o ABSOLUTE
    ../clib/microlib/malloc/malloc.c         0x00000000   Number         0  malloca.o ABSOLUTE
    ../clib/microlib/malloc/malloc.c         0x00000000   Number         0  mallocra.o ABSOLUTE
    ../clib/microlib/malloc/mvars.c          0x00000000   Number         0  mvars.o ABSOLUTE
    ../clib/microlib/printf/printf.c         0x00000000   Number         0  printf6.o ABSOLUTE
    ../clib/microlib/printf/printf.c         0x00000000   Number         0  printf3.o ABSOLUTE
    ../clib/microlib/printf/printf.c         0x00000000   Number         0  printf2.o ABSOLUTE
    ../clib/microlib/printf/printf.c         0x00000000   Number         0  printf1.o ABSOLUTE
    ../clib/microlib/printf/printf.c         0x00000000   Number         0  printf0.o ABSOLUTE
    ../clib/microlib/printf/printf.c         0x00000000   Number         0  printfb.o ABSOLUTE
    ../clib/microlib/printf/printf.c         0x00000000   Number         0  printf8.o ABSOLUTE
    ../clib/microlib/printf/printf.c         0x00000000   Number         0  printfa.o ABSOLUTE
    ../clib/microlib/printf/printf.c         0x00000000   Number         0  printf7.o ABSOLUTE
    ../clib/microlib/printf/printf.c         0x00000000   Number         0  printf5.o ABSOLUTE
    ../clib/microlib/printf/printf.c         0x00000000   Number         0  printf4.o ABSOLUTE
    ../clib/microlib/printf/stubs.s          0x00000000   Number         0  stubs.o ABSOLUTE
    ../clib/microlib/stdio/streams.c         0x00000000   Number         0  stdout.o ABSOLUTE
    ../clib/microlib/stdlib/rand.c           0x00000000   Number         0  rand.o ABSOLUTE
    ../clib/microlib/string/memcmp.c         0x00000000   Number         0  memcmp.o ABSOLUTE
    ../clib/microlib/string/memcpy.c         0x00000000   Number         0  memcpyb.o ABSOLUTE
    ../clib/microlib/string/memcpy.c         0x00000000   Number         0  memcpya.o ABSOLUTE
    ../clib/microlib/string/memset.c         0x00000000   Number         0  memset.o ABSOLUTE
    ../clib/microlib/string/memset.c         0x00000000   Number         0  memseta.o ABSOLUTE
    ../clib/microlib/string/strcat.c         0x00000000   Number         0  strcat.o ABSOLUTE
    ../clib/microlib/string/strcmp.c         0x00000000   Number         0  strcmp.o ABSOLUTE
    ../clib/microlib/string/strcpy.c         0x00000000   Number         0  strcpy.o ABSOLUTE
    ../clib/microlib/string/strlen.c         0x00000000   Number         0  strlen.o ABSOLUTE
    ../clib/microlib/string/strncmp.c        0x00000000   Number         0  strncmp.o ABSOLUTE
    ../clib/microlib/string/strrchr.c        0x00000000   Number         0  strrchr.o ABSOLUTE
    ../clib/microlib/string/strstr.c         0x00000000   Number         0  strstr.o ABSOLUTE
    ../clib/microlib/string/strtok.c         0x00000000   Number         0  strtok.o ABSOLUTE
    ../clib/microlib/string/strtok.c         0x00000000   Number         0  strtok_r.o ABSOLUTE
    ../clib/microlib/stubs.s                 0x00000000   Number         0  iusefp.o ABSOLUTE
    ../clib/scanf.c                          0x00000000   Number         0  __0sscanf.o ABSOLUTE
    ../clib/scanf.c                          0x00000000   Number         0  strtod.o ABSOLUTE
    ../clib/scanf.c                          0x00000000   Number         0  _sgetc.o ABSOLUTE
    ../clib/scanf.c                          0x00000000   Number         0  scanf_char.o ABSOLUTE
    ../clib/scanf.c                          0x00000000   Number         0  scanf_fp.o ABSOLUTE
    ../clib/scanf.c                          0x00000000   Number         0  _scanf.o ABSOLUTE
    ../fplib/microlib/d2f.c                  0x00000000   Number         0  d2f.o ABSOLUTE
    ../fplib/microlib/f2d.c                  0x00000000   Number         0  f2d.o ABSOLUTE
    ../fplib/microlib/fpadd.c                0x00000000   Number         0  dadd.o ABSOLUTE
    ../fplib/microlib/fpdiv.c                0x00000000   Number         0  ddiv.o ABSOLUTE
    ../fplib/microlib/fpepilogue.c           0x00000000   Number         0  fepilogue.o ABSOLUTE
    ../fplib/microlib/fpepilogue.c           0x00000000   Number         0  depilogue.o ABSOLUTE
    ../fplib/microlib/fpfix.c                0x00000000   Number         0  dfixi.o ABSOLUTE
    ../fplib/microlib/fpfix.c                0x00000000   Number         0  dfixul.o ABSOLUTE
    ../fplib/microlib/fpflt.c                0x00000000   Number         0  dflti.o ABSOLUTE
    ../fplib/microlib/fpflt.c                0x00000000   Number         0  dfltul.o ABSOLUTE
    ../fplib/microlib/fpmul.c                0x00000000   Number         0  dmul.o ABSOLUTE
    ../mathlib/strtod.c                      0x00000000   Number         0  strtod.o ABSOLUTE
    ..\CMSIS\CM3\CoreSupport\core_cm3.c      0x00000000   Number         0  core_cm3.o ABSOLUTE
    ..\CMSIS\CM3\DeviceSupport\ST\STM32F10x\system_stm32f10x.c 0x00000000   Number         0  system_stm32f10x.o ABSOLUTE
    ..\Libraries\src\misc.c                  0x00000000   Number         0  misc.o ABSOLUTE
    ..\Libraries\src\stm32f10x_adc.c         0x00000000   Number         0  stm32f10x_adc.o ABSOLUTE
    ..\Libraries\src\stm32f10x_bkp.c         0x00000000   Number         0  stm32f10x_bkp.o ABSOLUTE
    ..\Libraries\src\stm32f10x_dma.c         0x00000000   Number         0  stm32f10x_dma.o ABSOLUTE
    ..\Libraries\src\stm32f10x_exti.c        0x00000000   Number         0  stm32f10x_exti.o ABSOLUTE
    ..\Libraries\src\stm32f10x_flash.c       0x00000000   Number         0  stm32f10x_flash.o ABSOLUTE
    ..\Libraries\src\stm32f10x_gpio.c        0x00000000   Number         0  stm32f10x_gpio.o ABSOLUTE
    ..\Libraries\src\stm32f10x_pwr.c         0x00000000   Number         0  stm32f10x_pwr.o ABSOLUTE
    ..\Libraries\src\stm32f10x_rcc.c         0x00000000   Number         0  stm32f10x_rcc.o ABSOLUTE
    ..\Libraries\src\stm32f10x_rtc.c         0x00000000   Number         0  stm32f10x_rtc.o ABSOLUTE
    ..\Libraries\src\stm32f10x_tim.c         0x00000000   Number         0  stm32f10x_tim.o ABSOLUTE
    ..\Libraries\src\stm32f10x_usart.c       0x00000000   Number         0  stm32f10x_usart.o ABSOLUTE
    ..\NET\COAP\COAPHandle.c                 0x00000000   Number         0  coaphandle.o ABSOLUTE
    ..\NET\COAP\coap.c                       0x00000000   Number         0  coap.o ABSOLUTE
    ..\NET\COAP\regist.c                     0x00000000   Number         0  regist.o ABSOLUTE
    ..\NET\COAP\remote.c                     0x00000000   Number         0  remote.o ABSOLUTE
    ..\NET\Module\at.c                       0x00000000   Number         0  at.o ABSOLUTE
    ..\NET\Module\bc26.c                     0x00000000   Number         0  bc26.o ABSOLUTE
    ..\NET\Module\esp8266.c                  0x00000000   Number         0  esp8266.o ABSOLUTE
    ..\NET\Module\module_wrapper.c           0x00000000   Number         0  module_wrapper.o ABSOLUTE
    ..\NET\Util\AES.c                        0x00000000   Number         0  aes.o ABSOLUTE
    ..\NET\Util\ProgramData.c                0x00000000   Number         0  programdata.o ABSOLUTE
    ..\NET\Util\cJSON.c                      0x00000000   Number         0  cjson.o ABSOLUTE
    ..\NET\Util\cJSON_Utils.c                0x00000000   Number         0  cjson_utils.o ABSOLUTE
    ..\NET\Util\crc.c                        0x00000000   Number         0  crc.o ABSOLUTE
    ..\NET\Util\mbedtls_util.c               0x00000000   Number         0  mbedtls_util.o ABSOLUTE
    ..\NET\Util\sys.c                        0x00000000   Number         0  sys.o ABSOLUTE
    ..\Startup\startup_stm32f10x_md.s        0x00000000   Number         0  startup_stm32f10x_md.o ABSOLUTE
    ..\System\delay.c                        0x00000000   Number         0  delay.o ABSOLUTE
    ..\USER\ADCSetup.c                       0x00000000   Number         0  adcsetup.o ABSOLUTE
    ..\USER\ADS1110ASetup.c                  0x00000000   Number         0  ads1110asetup.o ABSOLUTE
    ..\USER\ADS1110Setup.c                   0x00000000   Number         0  ads1110setup.o ABSOLUTE
    ..\USER\Bubble_ADCSetup.c                0x00000000   Number         0  bubble_adcsetup.o ABSOLUTE
    ..\USER\CRC16.C                          0x00000000   Number         0  crc16.o ABSOLUTE
    ..\USER\ControlSystem.c                  0x00000000   Number         0  controlsystem.o ABSOLUTE
    ..\USER\DrawLCDGUI.c                     0x00000000   Number         0  drawlcdgui.o ABSOLUTE
    ..\USER\Driver.c                         0x00000000   Number         0  driver.o ABSOLUTE
    ..\USER\FM31256.c                        0x00000000   Number         0  fm31256.o ABSOLUTE
    ..\USER\FlashSetup.c                     0x00000000   Number         0  flashsetup.o ABSOLUTE
    ..\USER\History.c                        0x00000000   Number         0  history.o ABSOLUTE
    ..\USER\HostSlaveHandle.c                0x00000000   Number         0  hostslavehandle.o ABSOLUTE
    ..\USER\IIC2Setup.c                      0x00000000   Number         0  iic2setup.o ABSOLUTE
    ..\USER\IICSetup.c                       0x00000000   Number         0  iicsetup.o ABSOLUTE
    ..\USER\LCDSetup.c                       0x00000000   Number         0  lcdsetup.o ABSOLUTE
    ..\USER\Lorawan.c                        0x00000000   Number         0  lorawan.o ABSOLUTE
    ..\USER\ParameterSet.c                   0x00000000   Number         0  parameterset.o ABSOLUTE
    ..\USER\RTCSetup.c                       0x00000000   Number         0  rtcsetup.o ABSOLUTE
    ..\USER\SPISetup.c                       0x00000000   Number         0  spisetup.o ABSOLUTE
    ..\USER\SystemAlarm.c                    0x00000000   Number         0  systemalarm.o ABSOLUTE
    ..\USER\TimerSetup.c                     0x00000000   Number         0  timersetup.o ABSOLUTE
    ..\USER\TypeDefine.c                     0x00000000   Number         0  typedefine.o ABSOLUTE
    ..\USER\USARTSetup.c                     0x00000000   Number         0  usartsetup.o ABSOLUTE
    ..\USER\ZigbeeDataHandle.c               0x00000000   Number         0  zigbeedatahandle.o ABSOLUTE
    ..\USER\main.c                           0x00000000   Number         0  main.o ABSOLUTE
    ..\USER\stm32f10x_it.c                   0x00000000   Number         0  stm32f10x_it.o ABSOLUTE
    ..\\CMSIS\\CM3\\CoreSupport\\core_cm3.c  0x00000000   Number         0  core_cm3.o ABSOLUTE
    C:\Users\wulianwei\AppData\Local\Arm\Packs\ARM\mbedTLS\1.8.0\library\aes.c 0x00000000   Number         0  aes_1.o ABSOLUTE
    C:\Users\wulianwei\AppData\Local\Arm\Packs\ARM\mbedTLS\1.8.0\library\arc4.c 0x00000000   Number         0  arc4.o ABSOLUTE
    C:\Users\wulianwei\AppData\Local\Arm\Packs\ARM\mbedTLS\1.8.0\library\aria.c 0x00000000   Number         0  aria.o ABSOLUTE
    C:\Users\wulianwei\AppData\Local\Arm\Packs\ARM\mbedTLS\1.8.0\library\asn1parse.c 0x00000000   Number         0  asn1parse.o ABSOLUTE
    C:\Users\wulianwei\AppData\Local\Arm\Packs\ARM\mbedTLS\1.8.0\library\asn1write.c 0x00000000   Number         0  asn1write.o ABSOLUTE
    C:\Users\wulianwei\AppData\Local\Arm\Packs\ARM\mbedTLS\1.8.0\library\base64.c 0x00000000   Number         0  base64.o ABSOLUTE
    C:\Users\wulianwei\AppData\Local\Arm\Packs\ARM\mbedTLS\1.8.0\library\bignum.c 0x00000000   Number         0  bignum.o ABSOLUTE
    C:\Users\wulianwei\AppData\Local\Arm\Packs\ARM\mbedTLS\1.8.0\library\blowfish.c 0x00000000   Number         0  blowfish.o ABSOLUTE
    C:\Users\wulianwei\AppData\Local\Arm\Packs\ARM\mbedTLS\1.8.0\library\camellia.c 0x00000000   Number         0  camellia.o ABSOLUTE
    C:\Users\wulianwei\AppData\Local\Arm\Packs\ARM\mbedTLS\1.8.0\library\ccm.c 0x00000000   Number         0  ccm.o ABSOLUTE
    C:\Users\wulianwei\AppData\Local\Arm\Packs\ARM\mbedTLS\1.8.0\library\certs.c 0x00000000   Number         0  certs.o ABSOLUTE
    C:\Users\wulianwei\AppData\Local\Arm\Packs\ARM\mbedTLS\1.8.0\library\chacha20.c 0x00000000   Number         0  chacha20.o ABSOLUTE
    C:\Users\wulianwei\AppData\Local\Arm\Packs\ARM\mbedTLS\1.8.0\library\chachapoly.c 0x00000000   Number         0  chachapoly.o ABSOLUTE
    C:\Users\wulianwei\AppData\Local\Arm\Packs\ARM\mbedTLS\1.8.0\library\cipher.c 0x00000000   Number         0  cipher.o ABSOLUTE
    C:\Users\wulianwei\AppData\Local\Arm\Packs\ARM\mbedTLS\1.8.0\library\cipher_wrap.c 0x00000000   Number         0  cipher_wrap.o ABSOLUTE
    C:\Users\wulianwei\AppData\Local\Arm\Packs\ARM\mbedTLS\1.8.0\library\cmac.c 0x00000000   Number         0  cmac.o ABSOLUTE
    C:\Users\wulianwei\AppData\Local\Arm\Packs\ARM\mbedTLS\1.8.0\library\constant_time.c 0x00000000   Number         0  constant_time.o ABSOLUTE
    C:\Users\wulianwei\AppData\Local\Arm\Packs\ARM\mbedTLS\1.8.0\library\ctr_drbg.c 0x00000000   Number         0  ctr_drbg.o ABSOLUTE
    C:\Users\wulianwei\AppData\Local\Arm\Packs\ARM\mbedTLS\1.8.0\library\debug.c 0x00000000   Number         0  debug.o ABSOLUTE
    C:\Users\wulianwei\AppData\Local\Arm\Packs\ARM\mbedTLS\1.8.0\library\des.c 0x00000000   Number         0  des.o ABSOLUTE
    C:\Users\wulianwei\AppData\Local\Arm\Packs\ARM\mbedTLS\1.8.0\library\dhm.c 0x00000000   Number         0  dhm.o ABSOLUTE
    C:\Users\wulianwei\AppData\Local\Arm\Packs\ARM\mbedTLS\1.8.0\library\ecdh.c 0x00000000   Number         0  ecdh.o ABSOLUTE
    C:\Users\wulianwei\AppData\Local\Arm\Packs\ARM\mbedTLS\1.8.0\library\ecdsa.c 0x00000000   Number         0  ecdsa.o ABSOLUTE
    C:\Users\wulianwei\AppData\Local\Arm\Packs\ARM\mbedTLS\1.8.0\library\ecjpake.c 0x00000000   Number         0  ecjpake.o ABSOLUTE
    C:\Users\wulianwei\AppData\Local\Arm\Packs\ARM\mbedTLS\1.8.0\library\ecp.c 0x00000000   Number         0  ecp.o ABSOLUTE
    C:\Users\wulianwei\AppData\Local\Arm\Packs\ARM\mbedTLS\1.8.0\library\ecp_curves.c 0x00000000   Number         0  ecp_curves.o ABSOLUTE
    C:\Users\wulianwei\AppData\Local\Arm\Packs\ARM\mbedTLS\1.8.0\library\entropy.c 0x00000000   Number         0  entropy.o ABSOLUTE
    C:\Users\wulianwei\AppData\Local\Arm\Packs\ARM\mbedTLS\1.8.0\library\entropy_poll.c 0x00000000   Number         0  entropy_poll.o ABSOLUTE
    C:\Users\wulianwei\AppData\Local\Arm\Packs\ARM\mbedTLS\1.8.0\library\error.c 0x00000000   Number         0  error.o ABSOLUTE
    C:\Users\wulianwei\AppData\Local\Arm\Packs\ARM\mbedTLS\1.8.0\library\gcm.c 0x00000000   Number         0  gcm.o ABSOLUTE
    C:\Users\wulianwei\AppData\Local\Arm\Packs\ARM\mbedTLS\1.8.0\library\havege.c 0x00000000   Number         0  havege.o ABSOLUTE
    C:\Users\wulianwei\AppData\Local\Arm\Packs\ARM\mbedTLS\1.8.0\library\hkdf.c 0x00000000   Number         0  hkdf.o ABSOLUTE
    C:\Users\wulianwei\AppData\Local\Arm\Packs\ARM\mbedTLS\1.8.0\library\hmac_drbg.c 0x00000000   Number         0  hmac_drbg.o ABSOLUTE
    C:\Users\wulianwei\AppData\Local\Arm\Packs\ARM\mbedTLS\1.8.0\library\md.c 0x00000000   Number         0  md.o ABSOLUTE
    C:\Users\wulianwei\AppData\Local\Arm\Packs\ARM\mbedTLS\1.8.0\library\md2.c 0x00000000   Number         0  md2.o ABSOLUTE
    C:\Users\wulianwei\AppData\Local\Arm\Packs\ARM\mbedTLS\1.8.0\library\md4.c 0x00000000   Number         0  md4.o ABSOLUTE
    C:\Users\wulianwei\AppData\Local\Arm\Packs\ARM\mbedTLS\1.8.0\library\md5.c 0x00000000   Number         0  md5.o ABSOLUTE
    C:\Users\wulianwei\AppData\Local\Arm\Packs\ARM\mbedTLS\1.8.0\library\memory_buffer_alloc.c 0x00000000   Number         0  memory_buffer_alloc.o ABSOLUTE
    C:\Users\wulianwei\AppData\Local\Arm\Packs\ARM\mbedTLS\1.8.0\library\mps_reader.c 0x00000000   Number         0  mps_reader.o ABSOLUTE
    C:\Users\wulianwei\AppData\Local\Arm\Packs\ARM\mbedTLS\1.8.0\library\mps_trace.c 0x00000000   Number         0  mps_trace.o ABSOLUTE
    C:\Users\wulianwei\AppData\Local\Arm\Packs\ARM\mbedTLS\1.8.0\library\net_sockets.c 0x00000000   Number         0  net_sockets.o ABSOLUTE
    C:\Users\wulianwei\AppData\Local\Arm\Packs\ARM\mbedTLS\1.8.0\library\nist_kw.c 0x00000000   Number         0  nist_kw.o ABSOLUTE
    C:\Users\wulianwei\AppData\Local\Arm\Packs\ARM\mbedTLS\1.8.0\library\oid.c 0x00000000   Number         0  oid.o ABSOLUTE
    C:\Users\wulianwei\AppData\Local\Arm\Packs\ARM\mbedTLS\1.8.0\library\pem.c 0x00000000   Number         0  pem.o ABSOLUTE
    C:\Users\wulianwei\AppData\Local\Arm\Packs\ARM\mbedTLS\1.8.0\library\pk.c 0x00000000   Number         0  pk.o ABSOLUTE
    C:\Users\wulianwei\AppData\Local\Arm\Packs\ARM\mbedTLS\1.8.0\library\pk_wrap.c 0x00000000   Number         0  pk_wrap.o ABSOLUTE
    C:\Users\wulianwei\AppData\Local\Arm\Packs\ARM\mbedTLS\1.8.0\library\pkcs11.c 0x00000000   Number         0  pkcs11.o ABSOLUTE
    C:\Users\wulianwei\AppData\Local\Arm\Packs\ARM\mbedTLS\1.8.0\library\pkcs12.c 0x00000000   Number         0  pkcs12.o ABSOLUTE
    C:\Users\wulianwei\AppData\Local\Arm\Packs\ARM\mbedTLS\1.8.0\library\pkcs5.c 0x00000000   Number         0  pkcs5.o ABSOLUTE
    C:\Users\wulianwei\AppData\Local\Arm\Packs\ARM\mbedTLS\1.8.0\library\pkparse.c 0x00000000   Number         0  pkparse.o ABSOLUTE
    C:\Users\wulianwei\AppData\Local\Arm\Packs\ARM\mbedTLS\1.8.0\library\pkwrite.c 0x00000000   Number         0  pkwrite.o ABSOLUTE
    C:\Users\wulianwei\AppData\Local\Arm\Packs\ARM\mbedTLS\1.8.0\library\platform.c 0x00000000   Number         0  platform.o ABSOLUTE
    C:\Users\wulianwei\AppData\Local\Arm\Packs\ARM\mbedTLS\1.8.0\library\platform_util.c 0x00000000   Number         0  platform_util.o ABSOLUTE
    C:\Users\wulianwei\AppData\Local\Arm\Packs\ARM\mbedTLS\1.8.0\library\poly1305.c 0x00000000   Number         0  poly1305.o ABSOLUTE
    C:\Users\wulianwei\AppData\Local\Arm\Packs\ARM\mbedTLS\1.8.0\library\psa_crypto.c 0x00000000   Number         0  psa_crypto.o ABSOLUTE
    C:\Users\wulianwei\AppData\Local\Arm\Packs\ARM\mbedTLS\1.8.0\library\psa_crypto_aead.c 0x00000000   Number         0  psa_crypto_aead.o ABSOLUTE
    C:\Users\wulianwei\AppData\Local\Arm\Packs\ARM\mbedTLS\1.8.0\library\psa_crypto_cipher.c 0x00000000   Number         0  psa_crypto_cipher.o ABSOLUTE
    C:\Users\wulianwei\AppData\Local\Arm\Packs\ARM\mbedTLS\1.8.0\library\psa_crypto_client.c 0x00000000   Number         0  psa_crypto_client.o ABSOLUTE
    C:\Users\wulianwei\AppData\Local\Arm\Packs\ARM\mbedTLS\1.8.0\library\psa_crypto_driver_wrappers.c 0x00000000   Number         0  psa_crypto_driver_wrappers.o ABSOLUTE
    C:\Users\wulianwei\AppData\Local\Arm\Packs\ARM\mbedTLS\1.8.0\library\psa_crypto_ecp.c 0x00000000   Number         0  psa_crypto_ecp.o ABSOLUTE
    C:\Users\wulianwei\AppData\Local\Arm\Packs\ARM\mbedTLS\1.8.0\library\psa_crypto_hash.c 0x00000000   Number         0  psa_crypto_hash.o ABSOLUTE
    C:\Users\wulianwei\AppData\Local\Arm\Packs\ARM\mbedTLS\1.8.0\library\psa_crypto_mac.c 0x00000000   Number         0  psa_crypto_mac.o ABSOLUTE
    C:\Users\wulianwei\AppData\Local\Arm\Packs\ARM\mbedTLS\1.8.0\library\psa_crypto_rsa.c 0x00000000   Number         0  psa_crypto_rsa.o ABSOLUTE
    C:\Users\wulianwei\AppData\Local\Arm\Packs\ARM\mbedTLS\1.8.0\library\psa_crypto_se.c 0x00000000   Number         0  psa_crypto_se.o ABSOLUTE
    C:\Users\wulianwei\AppData\Local\Arm\Packs\ARM\mbedTLS\1.8.0\library\psa_crypto_slot_management.c 0x00000000   Number         0  psa_crypto_slot_management.o ABSOLUTE
    C:\Users\wulianwei\AppData\Local\Arm\Packs\ARM\mbedTLS\1.8.0\library\psa_crypto_storage.c 0x00000000   Number         0  psa_crypto_storage.o ABSOLUTE
    C:\Users\wulianwei\AppData\Local\Arm\Packs\ARM\mbedTLS\1.8.0\library\psa_its_file.c 0x00000000   Number         0  psa_its_file.o ABSOLUTE
    C:\Users\wulianwei\AppData\Local\Arm\Packs\ARM\mbedTLS\1.8.0\library\ripemd160.c 0x00000000   Number         0  ripemd160.o ABSOLUTE
    C:\Users\wulianwei\AppData\Local\Arm\Packs\ARM\mbedTLS\1.8.0\library\rsa.c 0x00000000   Number         0  rsa.o ABSOLUTE
    C:\Users\wulianwei\AppData\Local\Arm\Packs\ARM\mbedTLS\1.8.0\library\rsa_internal.c 0x00000000   Number         0  rsa_internal.o ABSOLUTE
    C:\Users\wulianwei\AppData\Local\Arm\Packs\ARM\mbedTLS\1.8.0\library\sha1.c 0x00000000   Number         0  sha1.o ABSOLUTE
    C:\Users\wulianwei\AppData\Local\Arm\Packs\ARM\mbedTLS\1.8.0\library\sha256.c 0x00000000   Number         0  sha256.o ABSOLUTE
    C:\Users\wulianwei\AppData\Local\Arm\Packs\ARM\mbedTLS\1.8.0\library\sha512.c 0x00000000   Number         0  sha512.o ABSOLUTE
    C:\Users\wulianwei\AppData\Local\Arm\Packs\ARM\mbedTLS\1.8.0\library\ssl_cache.c 0x00000000   Number         0  ssl_cache.o ABSOLUTE
    C:\Users\wulianwei\AppData\Local\Arm\Packs\ARM\mbedTLS\1.8.0\library\ssl_ciphersuites.c 0x00000000   Number         0  ssl_ciphersuites.o ABSOLUTE
    C:\Users\wulianwei\AppData\Local\Arm\Packs\ARM\mbedTLS\1.8.0\library\ssl_cli.c 0x00000000   Number         0  ssl_cli.o ABSOLUTE
    C:\Users\wulianwei\AppData\Local\Arm\Packs\ARM\mbedTLS\1.8.0\library\ssl_cookie.c 0x00000000   Number         0  ssl_cookie.o ABSOLUTE
    C:\Users\wulianwei\AppData\Local\Arm\Packs\ARM\mbedTLS\1.8.0\library\ssl_msg.c 0x00000000   Number         0  ssl_msg.o ABSOLUTE
    C:\Users\wulianwei\AppData\Local\Arm\Packs\ARM\mbedTLS\1.8.0\library\ssl_srv.c 0x00000000   Number         0  ssl_srv.o ABSOLUTE
    C:\Users\wulianwei\AppData\Local\Arm\Packs\ARM\mbedTLS\1.8.0\library\ssl_ticket.c 0x00000000   Number         0  ssl_ticket.o ABSOLUTE
    C:\Users\wulianwei\AppData\Local\Arm\Packs\ARM\mbedTLS\1.8.0\library\ssl_tls.c 0x00000000   Number         0  ssl_tls.o ABSOLUTE
    C:\Users\wulianwei\AppData\Local\Arm\Packs\ARM\mbedTLS\1.8.0\library\ssl_tls13_keys.c 0x00000000   Number         0  ssl_tls13_keys.o ABSOLUTE
    C:\Users\wulianwei\AppData\Local\Arm\Packs\ARM\mbedTLS\1.8.0\library\threading.c 0x00000000   Number         0  threading.o ABSOLUTE
    C:\Users\wulianwei\AppData\Local\Arm\Packs\ARM\mbedTLS\1.8.0\library\timing.c 0x00000000   Number         0  timing.o ABSOLUTE
    C:\Users\wulianwei\AppData\Local\Arm\Packs\ARM\mbedTLS\1.8.0\library\version.c 0x00000000   Number         0  version.o ABSOLUTE
    C:\Users\wulianwei\AppData\Local\Arm\Packs\ARM\mbedTLS\1.8.0\library\version_features.c 0x00000000   Number         0  version_features.o ABSOLUTE
    C:\Users\wulianwei\AppData\Local\Arm\Packs\ARM\mbedTLS\1.8.0\library\x509.c 0x00000000   Number         0  x509.o ABSOLUTE
    C:\Users\wulianwei\AppData\Local\Arm\Packs\ARM\mbedTLS\1.8.0\library\x509_create.c 0x00000000   Number         0  x509_create.o ABSOLUTE
    C:\Users\wulianwei\AppData\Local\Arm\Packs\ARM\mbedTLS\1.8.0\library\x509_crl.c 0x00000000   Number         0  x509_crl.o ABSOLUTE
    C:\Users\wulianwei\AppData\Local\Arm\Packs\ARM\mbedTLS\1.8.0\library\x509_crt.c 0x00000000   Number         0  x509_crt.o ABSOLUTE
    C:\Users\wulianwei\AppData\Local\Arm\Packs\ARM\mbedTLS\1.8.0\library\x509_csr.c 0x00000000   Number         0  x509_csr.o ABSOLUTE
    C:\Users\wulianwei\AppData\Local\Arm\Packs\ARM\mbedTLS\1.8.0\library\x509write_crt.c 0x00000000   Number         0  x509write_crt.o ABSOLUTE
    C:\Users\wulianwei\AppData\Local\Arm\Packs\ARM\mbedTLS\1.8.0\library\x509write_csr.c 0x00000000   Number         0  x509write_csr.o ABSOLUTE
    C:\Users\wulianwei\AppData\Local\Arm\Packs\ARM\mbedTLS\1.8.0\library\xtea.c 0x00000000   Number         0  xtea.o ABSOLUTE
    cdcmple.s                                0x00000000   Number         0  cdcmple.o ABSOLUTE
    cdrcmple.s                               0x00000000   Number         0  cdrcmple.o ABSOLUTE
    dc.s                                     0x00000000   Number         0  dc.o ABSOLUTE
    handlers.s                               0x00000000   Number         0  handlers.o ABSOLUTE
    init.s                                   0x00000000   Number         0  init.o ABSOLUTE
    RESET                                    0x08000000   Section      236  startup_stm32f10x_md.o(RESET)
    .ARM.Collect$$$$00000000                 0x080000ec   Section        0  entry.o(.ARM.Collect$$$$00000000)
    .ARM.Collect$$$$00000001                 0x080000ec   Section        4  entry2.o(.ARM.Collect$$$$00000001)
    .ARM.Collect$$$$00000004                 0x080000f0   Section        4  entry5.o(.ARM.Collect$$$$00000004)
    .ARM.Collect$$$$00000008                 0x080000f4   Section        0  entry7b.o(.ARM.Collect$$$$00000008)
    .ARM.Collect$$$$0000000A                 0x080000f4   Section        0  entry8b.o(.ARM.Collect$$$$0000000A)
    .ARM.Collect$$$$0000000B                 0x080000f4   Section        8  entry9a.o(.ARM.Collect$$$$0000000B)
    .ARM.Collect$$$$0000000D                 0x080000fc   Section        0  entry10a.o(.ARM.Collect$$$$0000000D)
    .ARM.Collect$$$$0000000F                 0x080000fc   Section        0  entry11a.o(.ARM.Collect$$$$0000000F)
    .ARM.Collect$$$$00002712                 0x080000fc   Section        4  entry2.o(.ARM.Collect$$$$00002712)
    __lit__00000000                          0x080000fc   Data           4  entry2.o(.ARM.Collect$$$$00002712)
    .text                                    0x08000100   Section        0  main.o(.text)
    .text                                    0x080001c8   Section        0  driver.o(.text)
    .text                                    0x080008f0   Section        0  typedefine.o(.text)
    .text                                    0x08000d84   Section        0  stm32f10x_it.o(.text)
    .text                                    0x08001b54   Section        0  rtcsetup.o(.text)
    .text                                    0x0800201c   Section        0  spisetup.o(.text)
    .text                                    0x08002090   Section        0  ads1110setup.o(.text)
    .text                                    0x080022f0   Section        0  iicsetup.o(.text)
    .text                                    0x08002724   Section        0  usartsetup.o(.text)
    .text                                    0x080029f4   Section        0  lcdsetup.o(.text)
    .text                                    0x08002e78   Section        0  history.o(.text)
    .text                                    0x080039a8   Section        0  flashsetup.o(.text)
    .text                                    0x08003a48   Section        0  parameterset.o(.text)
    .text                                    0x0800477c   Section        0  adcsetup.o(.text)
    .text                                    0x08004a04   Section        0  controlsystem.o(.text)
    .text                                    0x0800a07c   Section        0  drawlcdgui.o(.text)
    .text                                    0x0801213c   Section        0  systemalarm.o(.text)
    .text                                    0x08012978   Section        0  zigbeedatahandle.o(.text)
    .text                                    0x080135d0   Section        0  crc16.o(.text)
    .text                                    0x08013608   Section        0  hostslavehandle.o(.text)
    .text                                    0x08013684   Section        0  fm31256.o(.text)
    .text                                    0x08013bb8   Section        0  lorawan.o(.text)
    LoraNode_Reset                           0x08013c59   Thumb Code    32  lorawan.o(.text)
    .text                                    0x08013d74   Section        0  bubble_adcsetup.o(.text)
    .text                                    0x08014510   Section        0  system_stm32f10x.o(.text)
    SetSysClockToHSE                         0x08014511   Thumb Code   160  system_stm32f10x.o(.text)
    SetSysClock                              0x080145b1   Thumb Code     8  system_stm32f10x.o(.text)
    .text                                    0x080146b8   Section        0  misc.o(.text)
    .text                                    0x08014794   Section        0  stm32f10x_exti.o(.text)
    .text                                    0x080148b0   Section        0  stm32f10x_gpio.o(.text)
    .text                                    0x08014c0c   Section        0  stm32f10x_rcc.o(.text)
    .text                                    0x08014fb0   Section        0  stm32f10x_usart.o(.text)
    .text                                    0x080153b8   Section        0  stm32f10x_rtc.o(.text)
    .text                                    0x08015500   Section        0  stm32f10x_tim.o(.text)
    TI4_Config                               0x080159a7   Thumb Code   130  stm32f10x_tim.o(.text)
    TI3_Config                               0x08015a3b   Thumb Code   122  stm32f10x_tim.o(.text)
    TI2_Config                               0x08015acf   Thumb Code   130  stm32f10x_tim.o(.text)
    TI1_Config                               0x08015b63   Thumb Code   108  stm32f10x_tim.o(.text)
    .text                                    0x0801631c   Section        0  stm32f10x_pwr.o(.text)
    .text                                    0x080163e8   Section        0  stm32f10x_bkp.o(.text)
    .text                                    0x080164ac   Section        0  stm32f10x_flash.o(.text)
    .text                                    0x08016a68   Section        0  stm32f10x_adc.o(.text)
    .text                                    0x08016eb8   Section        0  stm32f10x_dma.o(.text)
    .text                                    0x0801710c   Section       36  startup_stm32f10x_md.o(.text)
    .text                                    0x08017130   Section        0  delay.o(.text)
    .text                                    0x080171b4   Section        0  at.o(.text)
    .text                                    0x0801733c   Section        0  bc26.o(.text)
    bc26_wake                                0x0801733d   Thumb Code    10  bc26.o(.text)
    bc26_send_data                           0x08017347   Thumb Code    96  bc26.o(.text)
    bc26_send_data_rai                       0x080173a7   Thumb Code   122  bc26.o(.text)
    bc26_send_data_ch                        0x08017421   Thumb Code   126  bc26.o(.text)
    bc26_get_data                            0x0801749f   Thumb Code   184  bc26.o(.text)
    bc26_restart                             0x08017557   Thumb Code    42  bc26.o(.text)
    bc26_config                              0x08017581   Thumb Code   172  bc26.o(.text)
    bc26_init                                0x0801762d   Thumb Code     8  bc26.o(.text)
    bc26_ue_down                             0x08017635   Thumb Code    54  bc26.o(.text)
    bc26_tcp_connect                         0x0801766b   Thumb Code    58  bc26.o(.text)
    bc26_channel_open                        0x080176a5   Thumb Code   604  bc26.o(.text)
    bc26_udp_open                            0x08017901   Thumb Code    54  bc26.o(.text)
    bc26_tcp_close                           0x08017937   Thumb Code    46  bc26.o(.text)
    bc26_channel_close                       0x08017965   Thumb Code    82  bc26.o(.text)
    bc26_tcp_state                           0x080179b7   Thumb Code   128  bc26.o(.text)
    bc26_channel_state                       0x08017a37   Thumb Code   178  bc26.o(.text)
    bc26_tcp_reconnect                       0x08017ae9   Thumb Code    38  bc26.o(.text)
    bc26_udp_reopen                          0x08017b0f   Thumb Code    38  bc26.o(.text)
    bc26_channel_reopen                      0x08017b35   Thumb Code    54  bc26.o(.text)
    bc26_online_event                        0x08017b6b   Thumb Code   102  bc26.o(.text)
    bc26_close_event                         0x08017bd1   Thumb Code    84  bc26.o(.text)
    bc26_recv_event                          0x08017c25   Thumb Code   572  bc26.o(.text)
    bc26_restart_event                       0x08017e93   Thumb Code    60  bc26.o(.text)
    bc26_handle_event                        0x08017ecf   Thumb Code   108  bc26.o(.text)
    .text                                    0x08017fdc   Section        0  module_wrapper.o(.text)
    .text                                    0x080182f8   Section        0  cjson.o(.text)
    case_insensitive_strcmp                  0x08018373   Thumb Code    72  cjson.o(.text)
    cJSON_strdup                             0x080183bb   Thumb Code    56  cjson.o(.text)
    cJSON_New_Item                           0x08018445   Thumb Code    26  cjson.o(.text)
    get_decimal_point                        0x080184b3   Thumb Code     4  cjson.o(.text)
    parse_number                             0x080184b7   Thumb Code   298  cjson.o(.text)
    ensure                                   0x08018695   Thumb Code   238  cjson.o(.text)
    update_offset                            0x08018783   Thumb Code    36  cjson.o(.text)
    compare_double                           0x080187a7   Thumb Code   112  cjson.o(.text)
    print_number                             0x08018817   Thumb Code   304  cjson.o(.text)
    parse_hex4                               0x08018947   Thumb Code    90  cjson.o(.text)
    utf16_literal_to_utf8                    0x080189a1   Thumb Code   300  cjson.o(.text)
    parse_string                             0x08018acd   Thumb Code   436  cjson.o(.text)
    print_string_ptr                         0x08018c81   Thumb Code   360  cjson.o(.text)
    print_string                             0x08018de9   Thumb Code    16  cjson.o(.text)
    buffer_skip_whitespace                   0x08018df9   Thumb Code    72  cjson.o(.text)
    skip_utf8_bom                            0x08018e41   Thumb Code    56  cjson.o(.text)
    parse_object                             0x08018e79   Thumb Code   318  cjson.o(.text)
    parse_array                              0x08018fb7   Thumb Code   266  cjson.o(.text)
    parse_value                              0x080190c1   Thumb Code   292  cjson.o(.text)
    print_object                             0x080192fd   Thumb Code   372  cjson.o(.text)
    print_array                              0x08019471   Thumb Code   204  cjson.o(.text)
    print_value                              0x0801953d   Thumb Code   242  cjson.o(.text)
    print                                    0x0801962f   Thumb Code   178  cjson.o(.text)
    get_array_item                           0x080197b7   Thumb Code    30  cjson.o(.text)
    get_object_item                          0x080197ed   Thumb Code    82  cjson.o(.text)
    suffix_object                            0x0801987b   Thumb Code     6  cjson.o(.text)
    create_reference                         0x08019881   Thumb Code    60  cjson.o(.text)
    add_item_to_array                        0x080198bd   Thumb Code    54  cjson.o(.text)
    cast_away_const                          0x08019903   Thumb Code     2  cjson.o(.text)
    add_item_to_object                       0x08019905   Thumb Code   122  cjson.o(.text)
    replace_item_in_object                   0x08019e7f   Thumb Code    98  cjson.o(.text)
    skip_oneline_comment                     0x0801a1d3   Thumb Code    42  cjson.o(.text)
    skip_multiline_comment                   0x0801a1fd   Thumb Code    50  cjson.o(.text)
    minify_string                            0x0801a22f   Thumb Code   116  cjson.o(.text)
    .text                                    0x0801a584   Section        0  crc.o(.text)
    .text                                    0x0801a674   Section        0  programdata.o(.text)
    .text                                    0x0801a6b8   Section        0  sys.o(.text)
    .text                                    0x0801ab38   Section        0  aes.o(.text)
    x2time                                   0x0801ab39   Thumb Code    24  aes.o(.text)
    x3time                                   0x0801ab51   Thumb Code    14  aes.o(.text)
    x4time                                   0x0801ab5f   Thumb Code    18  aes.o(.text)
    x8time                                   0x0801ab71   Thumb Code    24  aes.o(.text)
    x9time                                   0x0801ab89   Thumb Code    14  aes.o(.text)
    xBtime                                   0x0801ab97   Thumb Code    26  aes.o(.text)
    xDtime                                   0x0801abb1   Thumb Code    26  aes.o(.text)
    xEtime                                   0x0801abcb   Thumb Code    30  aes.o(.text)
    MixColumns                               0x0801abe9   Thumb Code   154  aes.o(.text)
    Contrary_MixColumns                      0x0801ac83   Thumb Code   186  aes.o(.text)
    ShiftRows                                0x0801ad3d   Thumb Code    50  aes.o(.text)
    Contrary_ShiftRows                       0x0801ad6f   Thumb Code    50  aes.o(.text)
    SubBytes                                 0x0801ada1   Thumb Code    22  aes.o(.text)
    Contrary_SubBytes                        0x0801adb7   Thumb Code    22  aes.o(.text)
    AddRoundKey                              0x0801adcd   Thumb Code    28  aes.o(.text)
    .text                                    0x0801b044   Section        0  mbedtls_util.o(.text)
    fillAESPKCS7Data                         0x0801b045   Thumb Code    74  mbedtls_util.o(.text)
    cutAESPKCS7Data                          0x0801b08f   Thumb Code    38  mbedtls_util.o(.text)
    .text                                    0x0801b3fc   Section        0  coap.o(.text)
    .text                                    0x0801b9ec   Section        0  coaphandle.o(.text)
    setValue                                 0x0801b9ef   Thumb Code    26  coaphandle.o(.text)
    generateCoapKey                          0x0801ba09   Thumb Code    96  coaphandle.o(.text)
    packPumbDataCoapSend                     0x0801bcc5   Thumb Code   934  coaphandle.o(.text)
    IntePumpStateCoap                        0x0801c06b   Thumb Code   322  coaphandle.o(.text)
    DecideSendFlagCoap                       0x0801c1ad   Thumb Code   296  coaphandle.o(.text)
    ModuleKeepOnLine                         0x0801c523   Thumb Code   712  coaphandle.o(.text)
    AuthHandle                               0x0801c7eb   Thumb Code   206  coaphandle.o(.text)
    HandleCoapValidData                      0x0801c8b9   Thumb Code   216  coaphandle.o(.text)
    SendCoapPumpData                         0x0801c9a7   Thumb Code   146  coaphandle.o(.text)
    .text                                    0x0801ce04   Section        0  regist.o(.text)
    packRegistDataAndSend                    0x0801ce53   Thumb Code   212  regist.o(.text)
    handleRegistInfo                         0x0801cf27   Thumb Code   278  regist.o(.text)
    .text                                    0x0801d268   Section        0  remote.o(.text)
    remoteModuleKeepLine                     0x0801d269   Thumb Code    48  remote.o(.text)
    packRemotetDataAndSend                   0x0801d299   Thumb Code   108  remote.o(.text)
    packRemotetDataJSONAndSend               0x0801d305   Thumb Code   162  remote.o(.text)
    handleRemoteInfo                         0x0801d3a7   Thumb Code   350  remote.o(.text)
    .text                                    0x0801d73c   Section        0  aes_1.o(.text)
    .text                                    0x0801e4bc   Section        0  base64.o(.text)
    .text                                    0x0801e764   Section        0  constant_time.o(.text)
    mbedtls_ct_uchar_mask_of_range           0x0801e7a7   Thumb Code    22  constant_time.o(.text)
    .text                                    0x0801e8b0   Section        0  platform_util.o(.text)
    .text                                    0x0801e8d0   Section        0  sha1.o(.text)
    .text                                    0x08020598   Section        0  sha256.o(.text)
    .text                                    0x0802180e   Section        0  uldiv.o(.text)
    .text                                    0x08021870   Section        0  tolower.o(.text)
    .text                                    0x0802187c   Section        0  rand.o(.text)
    .text                                    0x080218a0   Section        0  memcpya.o(.text)
    .text                                    0x080218c4   Section        0  memseta.o(.text)
    .text                                    0x080218e8   Section        0  strstr.o(.text)
    .text                                    0x0802190c   Section        0  strlen.o(.text)
    .text                                    0x0802191a   Section        0  strcmp.o(.text)
    .text                                    0x08021936   Section        0  memcmp.o(.text)
    .text                                    0x08021950   Section        0  strcpy.o(.text)
    .text                                    0x08021962   Section        0  strncmp.o(.text)
    .text                                    0x08021980   Section        0  strtok.o(.text)
    .text                                    0x080219c4   Section        0  __0sscanf.o(.text)
    .text                                    0x080219fc   Section        0  scanf_fp.o(.text)
    _fp_value                                0x080219fd   Thumb Code   256  scanf_fp.o(.text)
    .text                                    0x08021d34   Section        0  dadd.o(.text)
    .text                                    0x08021e82   Section        0  dmul.o(.text)
    .text                                    0x08021f66   Section        0  dflti.o(.text)
    .text                                    0x08021f88   Section        0  dfixi.o(.text)
    .text                                    0x08021fc6   Section        0  f2d.o(.text)
    .text                                    0x08021fec   Section       48  cdcmple.o(.text)
    .text                                    0x0802201c   Section       48  cdrcmple.o(.text)
    .text                                    0x0802204c   Section        0  uidiv.o(.text)
    .text                                    0x08022078   Section        0  llshl.o(.text)
    .text                                    0x08022096   Section        0  llushr.o(.text)
    .text                                    0x080220b6   Section        0  llsshr.o(.text)
    .text                                    0x080220dc   Section        0  scanf_char.o(.text)
    _scanf_char_input                        0x080220dd   Thumb Code    12  scanf_char.o(.text)
    .text                                    0x08022104   Section        0  _sgetc.o(.text)
    .text                                    0x08022144   Section        0  strtod.o(.text)
    _local_sscanf                            0x08022145   Thumb Code    54  strtod.o(.text)
    .text                                    0x080221e0   Section        0  iusefp.o(.text)
    .text                                    0x080221e0   Section        0  depilogue.o(.text)
    .text                                    0x0802229a   Section        0  ddiv.o(.text)
    .text                                    0x08022378   Section        0  dfltul.o(.text)
    .text                                    0x08022390   Section        0  dfixul.o(.text)
    .text                                    0x080223c0   Section        0  d2f.o(.text)
    .text                                    0x080223f8   Section       36  init.o(.text)
    .text                                    0x0802241c   Section        0  isspace_c.o(.text)
    .text                                    0x08022428   Section        0  _scanf.o(.text)
    .text                                    0x08022754   Section        0  fepilogue.o(.text)
    .text                                    0x080227c4   Section        0  ctype_c.o(.text)
    .text                                    0x080227ec   Section        0  __dczerorl2.o(.text)
    i.__0printf                              0x08022844   Section        0  printfa.o(i.__0printf)
    i.__0snprintf                            0x08022864   Section        0  printfa.o(i.__0snprintf)
    i.__0sprintf                             0x08022894   Section        0  printfa.o(i.__0sprintf)
    i.__0vsnprintf                           0x080228bc   Section        0  printfa.o(i.__0vsnprintf)
    i.__free$realloc                         0x080228e8   Section        0  mallocr.o(i.__free$realloc)
    i.__malloc$realloc                       0x08022944   Section        0  mallocr.o(i.__malloc$realloc)
    i.__scatterload_copy                     0x08022994   Section       14  handlers.o(i.__scatterload_copy)
    i.__scatterload_null                     0x080229a2   Section        2  handlers.o(i.__scatterload_null)
    i.__scatterload_zeroinit                 0x080229a4   Section       14  handlers.o(i.__scatterload_zeroinit)
    i._fp_digits                             0x080229b4   Section        0  printfa.o(i._fp_digits)
    _fp_digits                               0x080229b5   Thumb Code   366  printfa.o(i._fp_digits)
    i._is_digit                              0x08022b38   Section        0  scanf_fp.o(i._is_digit)
    i._printf_core                           0x08022b48   Section        0  printfa.o(i._printf_core)
    _printf_core                             0x08022b49   Thumb Code  1744  printfa.o(i._printf_core)
    i._printf_post_padding                   0x08023224   Section        0  printfa.o(i._printf_post_padding)
    _printf_post_padding                     0x08023225   Thumb Code    36  printfa.o(i._printf_post_padding)
    i._printf_pre_padding                    0x08023248   Section        0  printfa.o(i._printf_pre_padding)
    _printf_pre_padding                      0x08023249   Thumb Code    46  printfa.o(i._printf_pre_padding)
    i._snputc                                0x08023276   Section        0  printfa.o(i._snputc)
    _snputc                                  0x08023277   Thumb Code    22  printfa.o(i._snputc)
    i._sputc                                 0x0802328c   Section        0  printfa.o(i._sputc)
    _sputc                                   0x0802328d   Thumb Code    10  printfa.o(i._sputc)
    i.internal_alloc                         0x08023298   Section        0  mallocr.o(i.internal_alloc)
    internal_alloc                           0x08023299   Thumb Code    76  mallocr.o(i.internal_alloc)
    i.realloc                                0x080232e8   Section        0  mallocr.o(i.realloc)
    i.strtod                                 0x08023354   Section        0  strtod.o(i.strtod)
    .constdata                               0x08023370   Section       24  rtcsetup.o(.constdata)
    .constdata                               0x08023388   Section     9534  drawlcdgui.o(.constdata)
    .constdata                               0x080258c6   Section      512  crc16.o(.constdata)
    .constdata                               0x08025ac6   Section      522  aes.o(.constdata)
    sbox                                     0x08025ac6   Data         256  aes.o(.constdata)
    contrary_sbox                            0x08025bc6   Data         256  aes.o(.constdata)
    Rcon                                     0x08025cc6   Data          10  aes.o(.constdata)
    .constdata                               0x08025cd0   Section       32  coaphandle.o(.constdata)
    coap_content_json                        0x08025cd0   Data           1  coaphandle.o(.constdata)
    .constdata                               0x08025cf0   Section     8744  aes_1.o(.constdata)
    FSb                                      0x08025cf0   Data         256  aes_1.o(.constdata)
    FT0                                      0x08025df0   Data        1024  aes_1.o(.constdata)
    FT1                                      0x080261f0   Data        1024  aes_1.o(.constdata)
    FT2                                      0x080265f0   Data        1024  aes_1.o(.constdata)
    FT3                                      0x080269f0   Data        1024  aes_1.o(.constdata)
    RSb                                      0x08026df0   Data         256  aes_1.o(.constdata)
    RT0                                      0x08026ef0   Data        1024  aes_1.o(.constdata)
    RT1                                      0x080272f0   Data        1024  aes_1.o(.constdata)
    RT2                                      0x080276f0   Data        1024  aes_1.o(.constdata)
    RT3                                      0x08027af0   Data        1024  aes_1.o(.constdata)
    RCON                                     0x08027ef0   Data          40  aes_1.o(.constdata)
    .constdata                               0x08027f18   Section      256  sha256.o(.constdata)
    K                                        0x08027f18   Data         256  sha256.o(.constdata)
    .constdata                               0x08028018   Section       64  ctype_c.o(.constdata)
    .conststring                             0x08028058   Section       94  bc26.o(.conststring)
    .conststring                             0x080280b8   Section      184  coaphandle.o(.conststring)
    .data                                    0x20000000   Section        8  driver.o(.data)
    .data                                    0x20000008   Section       76  typedefine.o(.data)
    .data                                    0x20000054   Section       41  stm32f10x_it.o(.data)
    .data                                    0x2000007e   Section        4  rtcsetup.o(.data)
    HSEStartUpStatus                         0x2000007e   Data           1  rtcsetup.o(.data)
    daycnt                                   0x20000080   Data           2  rtcsetup.o(.data)
    .data                                    0x20000082   Section       23  ads1110setup.o(.data)
    .data                                    0x20000099   Section        3  usartsetup.o(.data)
    .data                                    0x2000009c   Section        8  history.o(.data)
    .data                                    0x200000a4   Section       26  adcsetup.o(.data)
    .data                                    0x200000c0   Section       44  controlsystem.o(.data)
    .data                                    0x200000ec   Section       10  drawlcdgui.o(.data)
    .data                                    0x200000f8   Section       22  systemalarm.o(.data)
    .data                                    0x2000010e   Section       11  zigbeedatahandle.o(.data)
    .data                                    0x2000011a   Section        7  lorawan.o(.data)
    .data                                    0x20000122   Section       84  bubble_adcsetup.o(.data)
    .data                                    0x20000178   Section       20  system_stm32f10x.o(.data)
    .data                                    0x2000018c   Section       20  stm32f10x_rcc.o(.data)
    APBAHBPrescTable                         0x2000018c   Data          16  stm32f10x_rcc.o(.data)
    ADCPrescTable                            0x2000019c   Data           4  stm32f10x_rcc.o(.data)
    .data                                    0x200001a0   Section      136  bc26.o(.data)
    event                                    0x200001a4   Data           4  bc26.o(.data)
    .data                                    0x20000228   Section        7  module_wrapper.o(.data)
    g_at_module                              0x20000228   Data           4  module_wrapper.o(.data)
    .data                                    0x20000230   Section       20  cjson.o(.data)
    global_error                             0x20000230   Data           8  cjson.o(.data)
    global_hooks                             0x20000238   Data          12  cjson.o(.data)
    .data                                    0x20000244   Section        8  programdata.o(.data)
    .data                                    0x2000024c   Section      315  coaphandle.o(.data)
    iv                                       0x2000024c   Data          17  coaphandle.o(.data)
    coap_con_path                            0x20000260   Data           4  coaphandle.o(.data)
    sign_format                              0x20000264   Data           4  coaphandle.o(.data)
    payload_format                           0x20000268   Data           4  coaphandle.o(.data)
    coap_auth_id                             0x20000270   Data           2  coaphandle.o(.data)
    send_num                                 0x20000352   Data           2  coaphandle.o(.data)
    send_suc_num                             0x20000354   Data           2  coaphandle.o(.data)
    repeat_send_count                        0x20000358   Data           1  coaphandle.o(.data)
    pre_send_num                             0x2000035a   Data           2  coaphandle.o(.data)
    firstSendFlag                            0x20000360   Data           4  coaphandle.o(.data)
    moduleInitCou                            0x20000364   Data           4  coaphandle.o(.data)
    pumpState                                0x20000368   Data           1  coaphandle.o(.data)
    pumpAlarm                                0x2000036a   Data           2  coaphandle.o(.data)
    pumpPreAlarm                             0x2000036c   Data           1  coaphandle.o(.data)
    pumpStateLast                            0x2000036d   Data           1  coaphandle.o(.data)
    pumpAlarmLast                            0x2000036e   Data           2  coaphandle.o(.data)
    pumpPreAlarmLast                         0x20000370   Data           1  coaphandle.o(.data)
    signData                                 0x20000371   Data           4  coaphandle.o(.data)
    addition_active                          0x20000378   Data           4  coaphandle.o(.data)
    first_dose_active                        0x2000037c   Data           4  coaphandle.o(.data)
    seq                                      0x20000380   Data           4  coaphandle.o(.data)
    last_send_num                            0x20000384   Data           2  coaphandle.o(.data)
    send_flag                                0x20000386   Data           1  coaphandle.o(.data)
    .data                                    0x20000388   Section       21  regist.o(.data)
    .data                                    0x200003a0   Section       10  remote.o(.data)
    remoteModuleStartCou                     0x200003a4   Data           4  remote.o(.data)
    send_flag                                0x200003a8   Data           1  remote.o(.data)
    remote_flag                              0x200003a9   Data           1  remote.o(.data)
    .data                                    0x200003ac   Section        4  platform_util.o(.data)
    memset_func                              0x200003ac   Data           4  platform_util.o(.data)
    .data                                    0x200003b0   Section        4  rand.o(.data)
    _rand_state                              0x200003b0   Data           4  rand.o(.data)
    .data                                    0x200003b4   Section        4  strtok.o(.data)
    state                                    0x200003b4   Data           4  strtok.o(.data)
    .data                                    0x200003b8   Section        4  stdout.o(.data)
    .data                                    0x200003bc   Section        4  mvars.o(.data)
    .data                                    0x200003c0   Section        4  mvars.o(.data)
    .bss                                     0x200003c8   Section      368  typedefine.o(.bss)
    .bss                                     0x20000538   Section      850  ads1110setup.o(.bss)
    .bss                                     0x2000088a   Section      306  usartsetup.o(.bss)
    .bss                                     0x200009bc   Section     2076  history.o(.bss)
    .bss                                     0x200011d8   Section      256  parameterset.o(.bss)
    .bss                                     0x200012d8   Section       30  systemalarm.o(.bss)
    .bss                                     0x200012f6   Section      170  bubble_adcsetup.o(.bss)
    .bss                                     0x200013a0   Section     2464  module_wrapper.o(.bss)
    .bss                                     0x20001d40   Section       15  cjson.o(.bss)
    version                                  0x20001d40   Data          15  cjson.o(.bss)
    .bss                                     0x20001d4f   Section      600  programdata.o(.bss)
    .bss                                     0x20001fa8   Section     2264  sys.o(.bss)
    .bss                                     0x20002880   Section     1396  coaphandle.o(.bss)
    buf                                      0x20002890   Data        1024  coaphandle.o(.bss)
    auth_token                               0x20002c90   Data          88  coaphandle.o(.bss)
    pumpData                                 0x20002dc4   Data          48  coaphandle.o(.bss)
    .bss                                     0x20002df4   Section      440  regist.o(.bss)
    .bss                                     0x20002fac   Section      200  remote.o(.bss)
    remoteData                               0x20002fac   Data         200  remote.o(.bss)
    HEAP                                     0x20003078   Section     2048  startup_stm32f10x_md.o(HEAP)
    STACK                                    0x20003878   Section     9216  startup_stm32f10x_md.o(STACK)

    Global Symbols

    Symbol Name                              Value     Ov Type        Size  Object(Section)

    BuildAttributes$$THM_ISAv4$P$D$K$B$S$PE$A:L22UL41UL21$X:L11$S22US41US21$IEEE1$IW$USESV6$~STKCKD$USESV7$~SHL$OTIME$ROPI$IEEEJ$EBA8$MICROLIB$REQ8$PRES8$EABIv2 0x00000000   Number         0  anon$$obj.o ABSOLUTE
    __ARM_use_no_argv                        0x00000000   Number         0  main.o ABSOLUTE
    _printf_a                                0x00000000   Number         0  stubs.o ABSOLUTE
    _printf_c                                0x00000000   Number         0  stubs.o ABSOLUTE
    _printf_charcount                        0x00000000   Number         0  stubs.o ABSOLUTE
    _printf_d                                0x00000000   Number         0  stubs.o ABSOLUTE
    _printf_e                                0x00000000   Number         0  stubs.o ABSOLUTE
    _printf_f                                0x00000000   Number         0  stubs.o ABSOLUTE
    _printf_flags                            0x00000000   Number         0  stubs.o ABSOLUTE
    _printf_fp_dec                           0x00000000   Number         0  stubs.o ABSOLUTE
    _printf_fp_hex                           0x00000000   Number         0  stubs.o ABSOLUTE
    _printf_g                                0x00000000   Number         0  stubs.o ABSOLUTE
    _printf_i                                0x00000000   Number         0  stubs.o ABSOLUTE
    _printf_int_dec                          0x00000000   Number         0  stubs.o ABSOLUTE
    _printf_l                                0x00000000   Number         0  stubs.o ABSOLUTE
    _printf_lc                               0x00000000   Number         0  stubs.o ABSOLUTE
    _printf_ll                               0x00000000   Number         0  stubs.o ABSOLUTE
    _printf_lld                              0x00000000   Number         0  stubs.o ABSOLUTE
    _printf_lli                              0x00000000   Number         0  stubs.o ABSOLUTE
    _printf_llo                              0x00000000   Number         0  stubs.o ABSOLUTE
    _printf_llu                              0x00000000   Number         0  stubs.o ABSOLUTE
    _printf_llx                              0x00000000   Number         0  stubs.o ABSOLUTE
    _printf_longlong_dec                     0x00000000   Number         0  stubs.o ABSOLUTE
    _printf_longlong_hex                     0x00000000   Number         0  stubs.o ABSOLUTE
    _printf_longlong_oct                     0x00000000   Number         0  stubs.o ABSOLUTE
    _printf_ls                               0x00000000   Number         0  stubs.o ABSOLUTE
    _printf_mbtowc                           0x00000000   Number         0  stubs.o ABSOLUTE
    _printf_n                                0x00000000   Number         0  stubs.o ABSOLUTE
    _printf_o                                0x00000000   Number         0  stubs.o ABSOLUTE
    _printf_p                                0x00000000   Number         0  stubs.o ABSOLUTE
    _printf_percent                          0x00000000   Number         0  stubs.o ABSOLUTE
    _printf_pre_padding                      0x00000000   Number         0  stubs.o ABSOLUTE
    _printf_return_value                     0x00000000   Number         0  stubs.o ABSOLUTE
    _printf_s                                0x00000000   Number         0  stubs.o ABSOLUTE
    _printf_sizespec                         0x00000000   Number         0  stubs.o ABSOLUTE
    _printf_str                              0x00000000   Number         0  stubs.o ABSOLUTE
    _printf_truncate_signed                  0x00000000   Number         0  stubs.o ABSOLUTE
    _printf_truncate_unsigned                0x00000000   Number         0  stubs.o ABSOLUTE
    _printf_u                                0x00000000   Number         0  stubs.o ABSOLUTE
    _printf_wc                               0x00000000   Number         0  stubs.o ABSOLUTE
    _printf_wctomb                           0x00000000   Number         0  stubs.o ABSOLUTE
    _printf_widthprec                        0x00000000   Number         0  stubs.o ABSOLUTE
    _printf_x                                0x00000000   Number         0  stubs.o ABSOLUTE
    __cpp_initialize__aeabi_                  - Undefined Weak Reference
    __cxa_finalize                            - Undefined Weak Reference
    _clock_init                               - Undefined Weak Reference
    _microlib_exit                            - Undefined Weak Reference
    _scanf_int                                - Undefined Weak Reference
    _scanf_longlong                           - Undefined Weak Reference
    _scanf_string                             - Undefined Weak Reference
    __Vectors_Size                           0x000000ec   Number         0  startup_stm32f10x_md.o ABSOLUTE
    __Vectors                                0x08000000   Data           4  startup_stm32f10x_md.o(RESET)
    __Vectors_End                            0x080000ec   Data           0  startup_stm32f10x_md.o(RESET)
    __main                                   0x080000ed   Thumb Code     0  entry.o(.ARM.Collect$$$$00000000)
    _main_stk                                0x080000ed   Thumb Code     0  entry2.o(.ARM.Collect$$$$00000001)
    _main_scatterload                        0x080000f1   Thumb Code     0  entry5.o(.ARM.Collect$$$$00000004)
    __main_after_scatterload                 0x080000f5   Thumb Code     0  entry5.o(.ARM.Collect$$$$00000004)
    _main_clock                              0x080000f5   Thumb Code     0  entry7b.o(.ARM.Collect$$$$00000008)
    _main_cpp_init                           0x080000f5   Thumb Code     0  entry8b.o(.ARM.Collect$$$$0000000A)
    _main_init                               0x080000f5   Thumb Code     0  entry9a.o(.ARM.Collect$$$$0000000B)
    __rt_final_cpp                           0x080000fd   Thumb Code     0  entry10a.o(.ARM.Collect$$$$0000000D)
    __rt_final_exit                          0x080000fd   Thumb Code     0  entry11a.o(.ARM.Collect$$$$0000000F)
    main                                     0x08000101   Thumb Code   182  main.o(.text)
    DriverSpeakerInit                        0x080001c9   Thumb Code    40  driver.o(.text)
    DriverLCDPWRInit                         0x080001f1   Thumb Code    82  driver.o(.text)
    DriverZigbeePWRInit                      0x08000243   Thumb Code    50  driver.o(.text)
    DriverKeyInit                            0x08000275   Thumb Code   424  driver.o(.text)
    PowerKeySave                             0x0800041d   Thumb Code    26  driver.o(.text)
    DriverMotorInit                          0x08000437   Thumb Code    40  driver.o(.text)
    DriverHallInit                           0x0800045f   Thumb Code   128  driver.o(.text)
    DriverSavePinInit                        0x080004df   Thumb Code     2  driver.o(.text)
    SpeakerCtl                               0x080004e1   Thumb Code    30  driver.o(.text)
    SensorPWRCtl                             0x080004ff   Thumb Code    44  driver.o(.text)
    Power_GPIOInit                           0x0800052b   Thumb Code    92  driver.o(.text)
    LedInit                                  0x08000587   Thumb Code    50  driver.o(.text)
    WatchDogInit                             0x080005b9   Thumb Code    60  driver.o(.text)
    LCDBLACtl                                0x080005f5   Thumb Code    30  driver.o(.text)
    ZigbeePWRCtl                             0x08000613   Thumb Code    18  driver.o(.text)
    MotorPWRCtl                              0x08000625   Thumb Code    30  driver.o(.text)
    SpeakerInit                              0x08000643   Thumb Code    80  driver.o(.text)
    SpeakerResetInit                         0x08000693   Thumb Code    46  driver.o(.text)
    CntAlarmSpeaker                          0x080006c1   Thumb Code   126  driver.o(.text)
    CntOpenHornInit                          0x0800073f   Thumb Code    64  driver.o(.text)
    MCU_ID                                   0x0800077f   Thumb Code   130  driver.o(.text)
    HWSetup                                  0x08000801   Thumb Code   194  driver.o(.text)
    Delay_ms                                 0x080008f1   Thumb Code    16  typedefine.o(.text)
    ReadInputTotalDose                       0x08000901   Thumb Code    52  typedefine.o(.text)
    SystemSWInit                             0x08000935   Thumb Code   824  typedefine.o(.text)
    RunParamUpdate                           0x08000c6d   Thumb Code   280  typedefine.o(.text)
    NMI_Handler                              0x08000d85   Thumb Code     2  stm32f10x_it.o(.text)
    HardFault_Handler                        0x08000d87   Thumb Code     4  stm32f10x_it.o(.text)
    MemManage_Handler                        0x08000d8b   Thumb Code     4  stm32f10x_it.o(.text)
    BusFault_Handler                         0x08000d8f   Thumb Code     4  stm32f10x_it.o(.text)
    UsageFault_Handler                       0x08000d93   Thumb Code     4  stm32f10x_it.o(.text)
    SVC_Handler                              0x08000d97   Thumb Code     2  stm32f10x_it.o(.text)
    DebugMon_Handler                         0x08000d99   Thumb Code     2  stm32f10x_it.o(.text)
    PendSV_Handler                           0x08000d9b   Thumb Code     2  stm32f10x_it.o(.text)
    SysTick_Handler                          0x08000d9d   Thumb Code  2428  stm32f10x_it.o(.text)
    EXTI1_IRQHandler                         0x08001719   Thumb Code     2  stm32f10x_it.o(.text)
    EXTI9_5_IRQHandler                       0x0800171b   Thumb Code   288  stm32f10x_it.o(.text)
    EXTI15_10_IRQHandler                     0x0800183b   Thumb Code   260  stm32f10x_it.o(.text)
    USART1_IRQHandler                        0x0800193f   Thumb Code    98  stm32f10x_it.o(.text)
    USART2_IRQHandler                        0x080019a1   Thumb Code    76  stm32f10x_it.o(.text)
    USART2_IRQHandler1                       0x080019ed   Thumb Code   236  stm32f10x_it.o(.text)
    USART3_IRQHandler                        0x08001ad9   Thumb Code    92  stm32f10x_it.o(.text)
    Is_Leap_Year                             0x08001b55   Thumb Code    58  rtcsetup.o(.text)
    RTC_Get_Week                             0x08001b8f   Thumb Code   116  rtcsetup.o(.text)
    RTC_Set                                  0x08001c03   Thumb Code   194  rtcsetup.o(.text)
    RTC_Get                                  0x08001cc5   Thumb Code   210  rtcsetup.o(.text)
    RTCInit                                  0x08001d97   Thumb Code   194  rtcsetup.o(.text)
    SystemTimeUpdate                         0x08001e59   Thumb Code    54  rtcsetup.o(.text)
    RTC_NVIC_Config                          0x08001e8f   Thumb Code    32  rtcsetup.o(.text)
    RTC_Alarm_Configuration                  0x08001eaf   Thumb Code   108  rtcsetup.o(.text)
    StopMode_Configuration                   0x08001f1b   Thumb Code   112  rtcsetup.o(.text)
    StopMode_SYSCLKConfig_STOP               0x08001f8b   Thumb Code    60  rtcsetup.o(.text)
    StopMode_EnterStopMode                   0x08001fc7   Thumb Code    34  rtcsetup.o(.text)
    SPIInit                                  0x0800201d   Thumb Code    40  spisetup.o(.text)
    SPIWriteByte                             0x08002045   Thumb Code    72  spisetup.o(.text)
    ADS1110Config                            0x08002091   Thumb Code    60  ads1110setup.o(.text)
    RD_ADS                                   0x080020cd   Thumb Code    56  ads1110setup.o(.text)
    ContactForceUpdate                       0x08002105   Thumb Code   430  ads1110setup.o(.text)
    TWI_Delay                                0x080022f1   Thumb Code    16  iicsetup.o(.text)
    RTC_Delay                                0x08002301   Thumb Code    18  iicsetup.o(.text)
    IICInit                                  0x08002313   Thumb Code    96  iicsetup.o(.text)
    TWI_START                                0x08002373   Thumb Code    82  iicsetup.o(.text)
    TWI_STOP                                 0x080023c5   Thumb Code    48  iicsetup.o(.text)
    TWI_SendACK                              0x080023f5   Thumb Code    50  iicsetup.o(.text)
    TWI_SendNACK                             0x08002427   Thumb Code    48  iicsetup.o(.text)
    TWI_WaitAck                              0x08002457   Thumb Code    70  iicsetup.o(.text)
    TWI_SendByte                             0x0800249d   Thumb Code   104  iicsetup.o(.text)
    TWI_ReceiveByte                          0x08002505   Thumb Code    78  iicsetup.o(.text)
    RTC_START                                0x08002553   Thumb Code    76  iicsetup.o(.text)
    RTC_STOP                                 0x0800259f   Thumb Code    48  iicsetup.o(.text)
    RTC_SendACK                              0x080025cf   Thumb Code    50  iicsetup.o(.text)
    RTC_SendNACK                             0x08002601   Thumb Code    48  iicsetup.o(.text)
    RTC_WaitAck                              0x08002631   Thumb Code    70  iicsetup.o(.text)
    RTC_SendByte                             0x08002677   Thumb Code    90  iicsetup.o(.text)
    RTC_ReceiveByte                          0x080026d1   Thumb Code    84  iicsetup.o(.text)
    USART2_DMAinit                           0x08002725   Thumb Code     2  usartsetup.o(.text)
    USART1_Init                              0x08002727   Thumb Code   176  usartsetup.o(.text)
    USART2_Init                              0x080027d7   Thumb Code   172  usartsetup.o(.text)
    USART3_Init                              0x08002883   Thumb Code   176  usartsetup.o(.text)
    USART1Send                               0x08002933   Thumb Code    58  usartsetup.o(.text)
    USART2Send                               0x0800296d   Thumb Code    58  usartsetup.o(.text)
    USART3Send                               0x080029a7   Thumb Code    58  usartsetup.o(.text)
    LCDReset                                 0x080029f5   Thumb Code    30  lcdsetup.o(.text)
    LCDWriteIndex                            0x08002a13   Thumb Code    22  lcdsetup.o(.text)
    LCDWriteData                             0x08002a29   Thumb Code    32  lcdsetup.o(.text)
    LCDWriteData16Bit                        0x08002a49   Thumb Code    20  lcdsetup.o(.text)
    LCDSetRegion                             0x08002a5d   Thumb Code    90  lcdsetup.o(.text)
    LCDInit                                  0x08002ab7   Thumb Code   110  lcdsetup.o(.text)
    LCDClear                                 0x08002b25   Thumb Code    74  lcdsetup.o(.text)
    LCDPartClear                             0x08002b6f   Thumb Code    84  lcdsetup.o(.text)
    LCDSetXY                                 0x08002bc3   Thumb Code    44  lcdsetup.o(.text)
    DisplayHeader                            0x08002bef   Thumb Code    70  lcdsetup.o(.text)
    DisplayGraphicsGBK24                     0x08002c35   Thumb Code    88  lcdsetup.o(.text)
    DisplayGraphicsGBK16                     0x08002c8d   Thumb Code    92  lcdsetup.o(.text)
    DisplayGraphicsGBK12                     0x08002ce9   Thumb Code    92  lcdsetup.o(.text)
    DisplayGraphicsGBK8_8                    0x08002d45   Thumb Code   100  lcdsetup.o(.text)
    DisplayGraphicsGBK8_12                   0x08002da9   Thumb Code   106  lcdsetup.o(.text)
    DisplayGraphicsGBK8_16                   0x08002e13   Thumb Code   100  lcdsetup.o(.text)
    HistorySendToPC                          0x08002e79   Thumb Code   820  history.o(.text)
    ReadHistoryRecordQTY                     0x080031ad   Thumb Code   170  history.o(.text)
    ReadHistoryRecord                        0x08003257   Thumb Code   888  history.o(.text)
    WriteHistoryRecordQTY                    0x080035cf   Thumb Code   234  history.o(.text)
    WriteHistoryRecord                       0x080036b9   Thumb Code   676  history.o(.text)
    HistoryQtyAdd                            0x0800395d   Thumb Code    34  history.o(.text)
    FlashWriteOperate                        0x080039a9   Thumb Code    88  flashsetup.o(.text)
    FlashReadOperate                         0x08003a01   Thumb Code    70  flashsetup.o(.text)
    ReadParameterRecord                      0x08003a49   Thumb Code  1604  parameterset.o(.text)
    WriteParameterRecord                     0x0800408d   Thumb Code   962  parameterset.o(.text)
    WriteInitParameterRecord                 0x0800444f   Thumb Code   806  parameterset.o(.text)
    AdcDmaInit                               0x0800477d   Thumb Code    82  adcsetup.o(.text)
    DriverADCInit                            0x080047cf   Thumb Code   176  adcsetup.o(.text)
    BatteryVoltADCGet                        0x0800487f   Thumb Code   336  adcsetup.o(.text)
    fputc                                    0x08004a05   Thumb Code    32  controlsystem.o(.text)
    CntlSysInitWork                          0x08004a25   Thumb Code    28  controlsystem.o(.text)
    CntlMotorWork                            0x08004a41   Thumb Code    50  controlsystem.o(.text)
    CntlSpeakerWork                          0x08004a73   Thumb Code   196  controlsystem.o(.text)
    HornWorkStatus                           0x08004b37   Thumb Code    62  controlsystem.o(.text)
    CntlHornWork                             0x08004b75   Thumb Code   350  controlsystem.o(.text)
    CntlSensorPWWork                         0x08004cd3   Thumb Code    38  controlsystem.o(.text)
    CntlLCDBlackWork                         0x08004cf9   Thumb Code   170  controlsystem.o(.text)
    ScanKeyWorkType                          0x08004da3   Thumb Code  1934  controlsystem.o(.text)
    CntlPowerOFFWork                         0x08005531   Thumb Code   100  controlsystem.o(.text)
    CntlPowerONWork                          0x08005595   Thumb Code    36  controlsystem.o(.text)
    CntlAutoPowerOff                         0x080055b9   Thumb Code    64  controlsystem.o(.text)
    CntlNoActionHint                         0x080055f9   Thumb Code    46  controlsystem.o(.text)
    InfusionControl                          0x08005627   Thumb Code   240  controlsystem.o(.text)
    CntlSystemStandby                        0x08005717   Thumb Code    54  controlsystem.o(.text)
    CntlStartupPicture                       0x0800574d   Thumb Code   132  controlsystem.o(.text)
    CntlHistoryPicture                       0x080057d1   Thumb Code   410  controlsystem.o(.text)
    CntlDeviceIDPicture                      0x0800596b   Thumb Code    60  controlsystem.o(.text)
    CntlDispTimePicture                      0x080059a7   Thumb Code   350  controlsystem.o(.text)
    CntlSetTimePicture                       0x08005b05   Thumb Code  1350  controlsystem.o(.text)
    CntlSetPasswordPicture                   0x0800604b   Thumb Code   630  controlsystem.o(.text)
    CntlVerifyInfoPicture                    0x080062c1   Thumb Code   370  controlsystem.o(.text)
    CntlSetVerifyInfoPicture                 0x08006433   Thumb Code  1568  controlsystem.o(.text)
    CntlInpatienPicture                      0x08006a53   Thumb Code   106  controlsystem.o(.text)
    CntlSetParamPicture                      0x08006abd   Thumb Code  1746  controlsystem.o(.text)
    CntlAiroutPicture                        0x0800718f   Thumb Code   274  controlsystem.o(.text)
    CntlLockPasswordPicture                  0x080072a1   Thumb Code   666  controlsystem.o(.text)
    CntlRunFirstDosePicture                  0x0800753b   Thumb Code  1004  controlsystem.o(.text)
    CntlRunMainPicture                       0x08007927   Thumb Code  1872  controlsystem.o(.text)
    CntlTransfuseOverPicture                 0x08008077   Thumb Code   424  controlsystem.o(.text)
    CntlEvaluateTransfusePicture             0x0800821f   Thumb Code   612  controlsystem.o(.text)
    CntlEvaluatePainPicture                  0x08008483   Thumb Code   546  controlsystem.o(.text)
    CntlLimbMyodynamiaPicture                0x080086a5   Thumb Code   592  controlsystem.o(.text)
    CntlEvaluateVerifyPicture                0x080088f5   Thumb Code   448  controlsystem.o(.text)
    CntlAlarmPicture                         0x08008ab5   Thumb Code  1218  controlsystem.o(.text)
    CntMechanicalFaultPicture                0x08008f77   Thumb Code   194  controlsystem.o(.text)
    CntlEngineeringMode1Picture              0x08009039   Thumb Code  1650  controlsystem.o(.text)
    CntlSystemWorkStep                       0x080096ab   Thumb Code   246  controlsystem.o(.text)
    CntlSystemWorkTimer                      0x080097a1   Thumb Code  1350  controlsystem.o(.text)
    RealTimeStateUpdate                      0x08009ce7   Thumb Code   906  controlsystem.o(.text)
    Gui_DrawPoint                            0x0800a07d   Thumb Code    24  drawlcdgui.o(.text)
    Gui_DrawLine                             0x0800a095   Thumb Code   186  drawlcdgui.o(.text)
    Gui_DrawFont_GBK8                        0x0800a14f   Thumb Code   102  drawlcdgui.o(.text)
    Gui_DrawFont_GBK8Number                  0x0800a1b5   Thumb Code   102  drawlcdgui.o(.text)
    Gui_DrawFont_GBK12                       0x0800a21b   Thumb Code   192  drawlcdgui.o(.text)
    Gui_DrawFont_GBK16                       0x0800a2db   Thumb Code   192  drawlcdgui.o(.text)
    Gui_DrawFont_GBK24                       0x0800a39b   Thumb Code   138  drawlcdgui.o(.text)
    HexToASCII                               0x0800a425   Thumb Code    86  drawlcdgui.o(.text)
    DecimalToASCII                           0x0800a47b   Thumb Code  1816  drawlcdgui.o(.text)
    DrawPhoneDisplay                         0x0800ab93   Thumb Code    36  drawlcdgui.o(.text)
    DrawPauseDisplay                         0x0800abb7   Thumb Code    36  drawlcdgui.o(.text)
    DrawLockDisplay                          0x0800abdb   Thumb Code    34  drawlcdgui.o(.text)
    DrawSignalDisplay                        0x0800abfd   Thumb Code    42  drawlcdgui.o(.text)
    DrawSilenceDisplay                       0x0800ac27   Thumb Code    60  drawlcdgui.o(.text)
    DrawBatteryDisplay                       0x0800ac63   Thumb Code   150  drawlcdgui.o(.text)
    DrawScheduleDisplay                      0x0800acf9   Thumb Code   808  drawlcdgui.o(.text)
    DrawStartupPicture                       0x0800b021   Thumb Code    48  drawlcdgui.o(.text)
    DrawHistoryFirstPicture                  0x0800b051   Thumb Code   996  drawlcdgui.o(.text)
    DrawHistorySecondPicture                 0x0800b435   Thumb Code   750  drawlcdgui.o(.text)
    DrawDeviceIDPicture                      0x0800b723   Thumb Code  1248  drawlcdgui.o(.text)
    DrawTimeDispPicture                      0x0800bc03   Thumb Code   528  drawlcdgui.o(.text)
    DrawTimeSetPicture                       0x0800be13   Thumb Code  1144  drawlcdgui.o(.text)
    DrawPasswordSetPicture                   0x0800c28b   Thumb Code  1112  drawlcdgui.o(.text)
    DrawVerifyInfoPicture                    0x0800c6e3   Thumb Code   488  drawlcdgui.o(.text)
    DrawSetVerifyInfoPicture                 0x0800c8cb   Thumb Code  1224  drawlcdgui.o(.text)
    DrawNoInpatientPicture                   0x0800cd93   Thumb Code    30  drawlcdgui.o(.text)
    DrawAiroutPicture                        0x0800cdb1   Thumb Code   450  drawlcdgui.o(.text)
    DrawSetParameterPicture                  0x0800cf73   Thumb Code  3352  drawlcdgui.o(.text)
    DrawRunFirstDosePicture                  0x0800dc8b   Thumb Code   740  drawlcdgui.o(.text)
    DrawRunMainPicture                       0x0800df6f   Thumb Code  1770  drawlcdgui.o(.text)
    DrawRunPressurePicture                   0x0800e659   Thumb Code   534  drawlcdgui.o(.text)
    DrawPauseMainPicture                     0x0800e86f   Thumb Code   434  drawlcdgui.o(.text)
    DrawPCAPicture                           0x0800ea21   Thumb Code  1212  drawlcdgui.o(.text)
    DrawLockPasswordPicture                  0x0800eedd   Thumb Code   392  drawlcdgui.o(.text)
    DrawTransfuseOverPicture                 0x0800f065   Thumb Code   688  drawlcdgui.o(.text)
    DrawAlarmDevicePicture                   0x0800f315   Thumb Code   250  drawlcdgui.o(.text)
    DrawAlarmJamPicture                      0x0800f40f   Thumb Code   304  drawlcdgui.o(.text)
    DrawAlarmMaxPicture                      0x0800f53f   Thumb Code   256  drawlcdgui.o(.text)
    DrawAlarmBubblePicture                   0x0800f63f   Thumb Code   256  drawlcdgui.o(.text)
    DrawAlarmNonePillCasePicture             0x0800f73f   Thumb Code   256  drawlcdgui.o(.text)
    DrawAlarmLowVoltPicture                  0x0800f83f   Thumb Code   306  drawlcdgui.o(.text)
    DrawAlarmLineLostPicture                 0x0800f971   Thumb Code    52  drawlcdgui.o(.text)
    InputTotalPicture                        0x0800f9a5   Thumb Code   256  drawlcdgui.o(.text)
    DrawEngineeringMode1Picture              0x0800faa5   Thumb Code  1442  drawlcdgui.o(.text)
    DrawEngineeringMode2Picture              0x08010047   Thumb Code  2102  drawlcdgui.o(.text)
    DrawTest1Picture                         0x0801087d   Thumb Code  1036  drawlcdgui.o(.text)
    DrawEvaluateTransfusePicture             0x08010c89   Thumb Code  1442  drawlcdgui.o(.text)
    DrawEvaluatePainPicture                  0x0801122b   Thumb Code   922  drawlcdgui.o(.text)
    DrawLimbMyodynamiaPicture                0x080115c5   Thumb Code   902  drawlcdgui.o(.text)
    DrawEvaluateUploadEnterPicture           0x0801194b   Thumb Code   512  drawlcdgui.o(.text)
    DrawEvaluateUploadingPicture             0x08011b4b   Thumb Code   270  drawlcdgui.o(.text)
    DrawEvaluateUploadingSuccessPicture      0x08011c59   Thumb Code   128  drawlcdgui.o(.text)
    DrawEvaluateUploadingFailPicture         0x08011cd9   Thumb Code   126  drawlcdgui.o(.text)
    LCDPictureDisplay                        0x08011d57   Thumb Code   826  drawlcdgui.o(.text)
    DrawRegistingPicture                     0x08012091   Thumb Code    30  drawlcdgui.o(.text)
    DrawRegistFailPicture                    0x080120af   Thumb Code    30  drawlcdgui.o(.text)
    DrawRegistSucPicture                     0x080120cd   Thumb Code    30  drawlcdgui.o(.text)
    PECASelfTestHandle                       0x0801213d   Thumb Code    38  systemalarm.o(.text)
    MechanicalFaultHandle                    0x08012163   Thumb Code   206  systemalarm.o(.text)
    JamFaultHandle                           0x08012231   Thumb Code    86  systemalarm.o(.text)
    MaxFaultHandle                           0x08012287   Thumb Code   112  systemalarm.o(.text)
    BubbleFaultHandle                        0x080122f7   Thumb Code   128  systemalarm.o(.text)
    NonePillCaseHandle                       0x08012377   Thumb Code    90  systemalarm.o(.text)
    BatteryVoltLowHandle                     0x080123d1   Thumb Code   492  systemalarm.o(.text)
    LineLostHandle                           0x080125bd   Thumb Code    84  systemalarm.o(.text)
    InputTotalHandle                         0x08012611   Thumb Code    78  systemalarm.o(.text)
    SystemAlarmJudge                         0x0801265f   Thumb Code   698  systemalarm.o(.text)
    CommandToZigbeeHandle                    0x08012979   Thumb Code    90  zigbeedatahandle.o(.text)
    CommandToZigbeeReadNet                   0x080129d3   Thumb Code    66  zigbeedatahandle.o(.text)
    CommandToZigbeeReadFatherADDR            0x08012a15   Thumb Code    90  zigbeedatahandle.o(.text)
    DataFromZigbeeHandle                     0x08012a6f   Thumb Code     2  zigbeedatahandle.o(.text)
    RTDToZigbeeHandle                        0x08012a71   Thumb Code   800  zigbeedatahandle.o(.text)
    RunToLorawawn                            0x08012d91   Thumb Code   322  zigbeedatahandle.o(.text)
    EvaluateToZigbeeHandle                   0x08012ed3   Thumb Code   478  zigbeedatahandle.o(.text)
    ZigbeeXmitHandle                         0x080130b1   Thumb Code  1020  zigbeedatahandle.o(.text)
    ZigbeeRecvHandle                         0x080134ad   Thumb Code    50  zigbeedatahandle.o(.text)
    Uart2RecvHandle                          0x080134df   Thumb Code   162  zigbeedatahandle.o(.text)
    CalCRC16                                 0x080135d1   Thumb Code    48  crc16.o(.text)
    Power_off                                0x08013609   Thumb Code    40  hostslavehandle.o(.text)
    HostToSlaveHandle                        0x08013631   Thumb Code    68  hostslavehandle.o(.text)
    hex_to_bcd                               0x08013685   Thumb Code    32  fm31256.o(.text)
    bcd_to_hex                               0x080136a5   Thumb Code    22  fm31256.o(.text)
    Read_Reg                                 0x080136bb   Thumb Code   110  fm31256.o(.text)
    Write_Reg                                0x08013729   Thumb Code    86  fm31256.o(.text)
    Read_FM31256RAM                          0x0801377f   Thumb Code   132  fm31256.o(.text)
    Read_Multi31256RAM                       0x08013803   Thumb Code   192  fm31256.o(.text)
    Write_FM31256RAM                         0x080138c3   Thumb Code   116  fm31256.o(.text)
    Write_Multi31256RAM                      0x08013937   Thumb Code   158  fm31256.o(.text)
    InitRtc                                  0x080139d5   Thumb Code   124  fm31256.o(.text)
    GetCurDateTimeFromRTC                    0x08013a51   Thumb Code   192  fm31256.o(.text)
    SetDateTimeToRTC                         0x08013b11   Thumb Code   162  fm31256.o(.text)
    LoraNode_Delay                           0x08013bb9   Thumb Code    26  lorawan.o(.text)
    LoraNode_GPIO_Init                       0x08013bd3   Thumb Code   134  lorawan.o(.text)
    LoraNode_Init_Mode                       0x08013c79   Thumb Code    10  lorawan.o(.text)
    LoraNode_Wake_Sleep                      0x08013c83   Thumb Code    60  lorawan.o(.text)
    transparent_send_data                    0x08013cbf   Thumb Code    66  lorawan.o(.text)
    lorawan_Sleep                            0x08013d01   Thumb Code    62  lorawan.o(.text)
    LoraNode_OTAA_Config                     0x08013d3f   Thumb Code    10  lorawan.o(.text)
    OPB350L_ADCInit                          0x08013d75   Thumb Code   140  bubble_adcsetup.o(.text)
    OPB350L_ADCGet                           0x08013e01   Thumb Code   390  bubble_adcsetup.o(.text)
    Electricity_ADCGet                       0x08013f87   Thumb Code  1160  bubble_adcsetup.o(.text)
    Electricity_WorkOffGet                   0x0801440f   Thumb Code   156  bubble_adcsetup.o(.text)
    SystemInit                               0x080145b9   Thumb Code    78  system_stm32f10x.o(.text)
    SystemCoreClockUpdate                    0x08014607   Thumb Code   142  system_stm32f10x.o(.text)
    NVIC_PriorityGroupConfig                 0x080146b9   Thumb Code    10  misc.o(.text)
    NVIC_Init                                0x080146c3   Thumb Code   100  misc.o(.text)
    NVIC_SetVectorTable                      0x08014727   Thumb Code    14  misc.o(.text)
    NVIC_SystemLPConfig                      0x08014735   Thumb Code    34  misc.o(.text)
    SysTick_CLKSourceConfig                  0x08014757   Thumb Code    40  misc.o(.text)
    EXTI_DeInit                              0x08014795   Thumb Code    28  stm32f10x_exti.o(.text)
    EXTI_Init                                0x080147b1   Thumb Code   142  stm32f10x_exti.o(.text)
    EXTI_StructInit                          0x0801483f   Thumb Code    16  stm32f10x_exti.o(.text)
    EXTI_GenerateSWInterrupt                 0x0801484f   Thumb Code    16  stm32f10x_exti.o(.text)
    EXTI_GetFlagStatus                       0x0801485f   Thumb Code    22  stm32f10x_exti.o(.text)
    EXTI_ClearFlag                           0x08014875   Thumb Code     8  stm32f10x_exti.o(.text)
    EXTI_GetITStatus                         0x0801487d   Thumb Code    34  stm32f10x_exti.o(.text)
    EXTI_ClearITPendingBit                   0x0801489f   Thumb Code     8  stm32f10x_exti.o(.text)
    GPIO_DeInit                              0x080148b1   Thumb Code   172  stm32f10x_gpio.o(.text)
    GPIO_AFIODeInit                          0x0801495d   Thumb Code    20  stm32f10x_gpio.o(.text)
    GPIO_Init                                0x08014971   Thumb Code   278  stm32f10x_gpio.o(.text)
    GPIO_StructInit                          0x08014a87   Thumb Code    16  stm32f10x_gpio.o(.text)
    GPIO_ReadInputDataBit                    0x08014a97   Thumb Code    18  stm32f10x_gpio.o(.text)
    GPIO_ReadInputData                       0x08014aa9   Thumb Code     8  stm32f10x_gpio.o(.text)
    GPIO_ReadOutputDataBit                   0x08014ab1   Thumb Code    18  stm32f10x_gpio.o(.text)
    GPIO_ReadOutputData                      0x08014ac3   Thumb Code     8  stm32f10x_gpio.o(.text)
    GPIO_SetBits                             0x08014acb   Thumb Code     4  stm32f10x_gpio.o(.text)
    GPIO_ResetBits                           0x08014acf   Thumb Code     4  stm32f10x_gpio.o(.text)
    GPIO_WriteBit                            0x08014ad3   Thumb Code    10  stm32f10x_gpio.o(.text)
    GPIO_Write                               0x08014add   Thumb Code     4  stm32f10x_gpio.o(.text)
    GPIO_PinLockConfig                       0x08014ae1   Thumb Code    18  stm32f10x_gpio.o(.text)
    GPIO_EventOutputConfig                   0x08014af3   Thumb Code    26  stm32f10x_gpio.o(.text)
    GPIO_EventOutputCmd                      0x08014b0d   Thumb Code     6  stm32f10x_gpio.o(.text)
    GPIO_PinRemapConfig                      0x08014b13   Thumb Code   138  stm32f10x_gpio.o(.text)
    GPIO_EXTILineConfig                      0x08014b9d   Thumb Code    66  stm32f10x_gpio.o(.text)
    GPIO_ETH_MediaInterfaceConfig            0x08014bdf   Thumb Code     8  stm32f10x_gpio.o(.text)
    RCC_DeInit                               0x08014c0d   Thumb Code    64  stm32f10x_rcc.o(.text)
    RCC_HSEConfig                            0x08014c4d   Thumb Code    70  stm32f10x_rcc.o(.text)
    RCC_GetFlagStatus                        0x08014c93   Thumb Code    56  stm32f10x_rcc.o(.text)
    RCC_WaitForHSEStartUp                    0x08014ccb   Thumb Code    56  stm32f10x_rcc.o(.text)
    RCC_AdjustHSICalibrationValue            0x08014d03   Thumb Code    20  stm32f10x_rcc.o(.text)
    RCC_HSICmd                               0x08014d17   Thumb Code     6  stm32f10x_rcc.o(.text)
    RCC_PLLConfig                            0x08014d1d   Thumb Code    24  stm32f10x_rcc.o(.text)
    RCC_PLLCmd                               0x08014d35   Thumb Code     6  stm32f10x_rcc.o(.text)
    RCC_SYSCLKConfig                         0x08014d3b   Thumb Code    18  stm32f10x_rcc.o(.text)
    RCC_GetSYSCLKSource                      0x08014d4d   Thumb Code    10  stm32f10x_rcc.o(.text)
    RCC_HCLKConfig                           0x08014d57   Thumb Code    18  stm32f10x_rcc.o(.text)
    RCC_PCLK1Config                          0x08014d69   Thumb Code    18  stm32f10x_rcc.o(.text)
    RCC_PCLK2Config                          0x08014d7b   Thumb Code    20  stm32f10x_rcc.o(.text)
    RCC_ITConfig                             0x08014d8f   Thumb Code    26  stm32f10x_rcc.o(.text)
    RCC_USBCLKConfig                         0x08014da9   Thumb Code     8  stm32f10x_rcc.o(.text)
    RCC_ADCCLKConfig                         0x08014db1   Thumb Code    18  stm32f10x_rcc.o(.text)
    RCC_LSEConfig                            0x08014dc3   Thumb Code    50  stm32f10x_rcc.o(.text)
    RCC_LSICmd                               0x08014df5   Thumb Code     6  stm32f10x_rcc.o(.text)
    RCC_RTCCLKConfig                         0x08014dfb   Thumb Code    12  stm32f10x_rcc.o(.text)
    RCC_RTCCLKCmd                            0x08014e07   Thumb Code     8  stm32f10x_rcc.o(.text)
    RCC_GetClocksFreq                        0x08014e0f   Thumb Code   192  stm32f10x_rcc.o(.text)
    RCC_AHBPeriphClockCmd                    0x08014ecf   Thumb Code    26  stm32f10x_rcc.o(.text)
    RCC_APB2PeriphClockCmd                   0x08014ee9   Thumb Code    26  stm32f10x_rcc.o(.text)
    RCC_APB1PeriphClockCmd                   0x08014f03   Thumb Code    26  stm32f10x_rcc.o(.text)
    RCC_APB2PeriphResetCmd                   0x08014f1d   Thumb Code    26  stm32f10x_rcc.o(.text)
    RCC_APB1PeriphResetCmd                   0x08014f37   Thumb Code    26  stm32f10x_rcc.o(.text)
    RCC_BackupResetCmd                       0x08014f51   Thumb Code     8  stm32f10x_rcc.o(.text)
    RCC_ClockSecuritySystemCmd               0x08014f59   Thumb Code     6  stm32f10x_rcc.o(.text)
    RCC_MCOConfig                            0x08014f5f   Thumb Code     6  stm32f10x_rcc.o(.text)
    RCC_ClearFlag                            0x08014f65   Thumb Code    14  stm32f10x_rcc.o(.text)
    RCC_GetITStatus                          0x08014f73   Thumb Code    20  stm32f10x_rcc.o(.text)
    RCC_ClearITPendingBit                    0x08014f87   Thumb Code     6  stm32f10x_rcc.o(.text)
    USART_DeInit                             0x08014fb1   Thumb Code   134  stm32f10x_usart.o(.text)
    USART_Init                               0x08015037   Thumb Code   210  stm32f10x_usart.o(.text)
    USART_StructInit                         0x08015109   Thumb Code    24  stm32f10x_usart.o(.text)
    USART_ClockInit                          0x08015121   Thumb Code    34  stm32f10x_usart.o(.text)
    USART_ClockStructInit                    0x08015143   Thumb Code    12  stm32f10x_usart.o(.text)
    USART_Cmd                                0x0801514f   Thumb Code    24  stm32f10x_usart.o(.text)
    USART_ITConfig                           0x08015167   Thumb Code    74  stm32f10x_usart.o(.text)
    USART_DMACmd                             0x080151b1   Thumb Code    18  stm32f10x_usart.o(.text)
    USART_SetAddress                         0x080151c3   Thumb Code    18  stm32f10x_usart.o(.text)
    USART_WakeUpConfig                       0x080151d5   Thumb Code    18  stm32f10x_usart.o(.text)
    USART_ReceiverWakeUpCmd                  0x080151e7   Thumb Code    24  stm32f10x_usart.o(.text)
    USART_LINBreakDetectLengthConfig         0x080151ff   Thumb Code    18  stm32f10x_usart.o(.text)
    USART_LINCmd                             0x08015211   Thumb Code    24  stm32f10x_usart.o(.text)
    USART_SendData                           0x08015229   Thumb Code     8  stm32f10x_usart.o(.text)
    USART_ReceiveData                        0x08015231   Thumb Code    10  stm32f10x_usart.o(.text)
    USART_SendBreak                          0x0801523b   Thumb Code    10  stm32f10x_usart.o(.text)
    USART_SetGuardTime                       0x08015245   Thumb Code    16  stm32f10x_usart.o(.text)
    USART_SetPrescaler                       0x08015255   Thumb Code    16  stm32f10x_usart.o(.text)
    USART_SmartCardCmd                       0x08015265   Thumb Code    24  stm32f10x_usart.o(.text)
    USART_SmartCardNACKCmd                   0x0801527d   Thumb Code    24  stm32f10x_usart.o(.text)
    USART_HalfDuplexCmd                      0x08015295   Thumb Code    24  stm32f10x_usart.o(.text)
    USART_OverSampling8Cmd                   0x080152ad   Thumb Code    22  stm32f10x_usart.o(.text)
    USART_OneBitMethodCmd                    0x080152c3   Thumb Code    24  stm32f10x_usart.o(.text)
    USART_IrDAConfig                         0x080152db   Thumb Code    18  stm32f10x_usart.o(.text)
    USART_IrDACmd                            0x080152ed   Thumb Code    24  stm32f10x_usart.o(.text)
    USART_GetFlagStatus                      0x08015305   Thumb Code    26  stm32f10x_usart.o(.text)
    USART_ClearFlag                          0x0801531f   Thumb Code    18  stm32f10x_usart.o(.text)
    USART_GetITStatus                        0x08015331   Thumb Code    84  stm32f10x_usart.o(.text)
    USART_ClearITPendingBit                  0x08015385   Thumb Code    52  stm32f10x_usart.o(.text)
    RTC_ITConfig                             0x080153b9   Thumb Code    26  stm32f10x_rtc.o(.text)
    RTC_EnterConfigMode                      0x080153d3   Thumb Code    18  stm32f10x_rtc.o(.text)
    RTC_ExitConfigMode                       0x080153e5   Thumb Code    20  stm32f10x_rtc.o(.text)
    RTC_GetCounter                           0x080153f9   Thumb Code    18  stm32f10x_rtc.o(.text)
    RTC_SetCounter                           0x0801540b   Thumb Code    26  stm32f10x_rtc.o(.text)
    RTC_SetPrescaler                         0x08015425   Thumb Code    28  stm32f10x_rtc.o(.text)
    RTC_SetAlarm                             0x08015441   Thumb Code    26  stm32f10x_rtc.o(.text)
    RTC_GetDivider                           0x0801545b   Thumb Code    22  stm32f10x_rtc.o(.text)
    RTC_WaitForLastTask                      0x08015471   Thumb Code    18  stm32f10x_rtc.o(.text)
    RTC_WaitForSynchro                       0x08015483   Thumb Code    36  stm32f10x_rtc.o(.text)
    RTC_GetFlagStatus                        0x080154a7   Thumb Code    22  stm32f10x_rtc.o(.text)
    RTC_ClearFlag                            0x080154bd   Thumb Code    16  stm32f10x_rtc.o(.text)
    RTC_GetITStatus                          0x080154cd   Thumb Code    32  stm32f10x_rtc.o(.text)
    RTC_ClearITPendingBit                    0x080154ed   Thumb Code    16  stm32f10x_rtc.o(.text)
    TIM_DeInit                               0x08015501   Thumb Code   424  stm32f10x_tim.o(.text)
    TIM_TimeBaseInit                         0x080156a9   Thumb Code   122  stm32f10x_tim.o(.text)
    TIM_OC1Init                              0x08015723   Thumb Code   132  stm32f10x_tim.o(.text)
    TIM_OC2Init                              0x080157a7   Thumb Code   154  stm32f10x_tim.o(.text)
    TIM_OC3Init                              0x08015841   Thumb Code   150  stm32f10x_tim.o(.text)
    TIM_OC4Init                              0x080158d7   Thumb Code   182  stm32f10x_tim.o(.text)
    TIM_SetIC4Prescaler                      0x0801598d   Thumb Code    26  stm32f10x_tim.o(.text)
    TIM_SetIC3Prescaler                      0x08015a29   Thumb Code    18  stm32f10x_tim.o(.text)
    TIM_SetIC2Prescaler                      0x08015ab5   Thumb Code    26  stm32f10x_tim.o(.text)
    TIM_SetIC1Prescaler                      0x08015b51   Thumb Code    18  stm32f10x_tim.o(.text)
    TIM_ICInit                               0x08015bcf   Thumb Code   150  stm32f10x_tim.o(.text)
    TIM_PWMIConfig                           0x08015c65   Thumb Code   124  stm32f10x_tim.o(.text)
    TIM_BDTRConfig                           0x08015ce1   Thumb Code    32  stm32f10x_tim.o(.text)
    TIM_TimeBaseStructInit                   0x08015d01   Thumb Code    18  stm32f10x_tim.o(.text)
    TIM_OCStructInit                         0x08015d13   Thumb Code    20  stm32f10x_tim.o(.text)
    TIM_ICStructInit                         0x08015d27   Thumb Code    18  stm32f10x_tim.o(.text)
    TIM_BDTRStructInit                       0x08015d39   Thumb Code    40  stm32f10x_tim.o(.text)
    TIM_Cmd                                  0x08015d61   Thumb Code    24  stm32f10x_tim.o(.text)
    TIM_CtrlPWMOutputs                       0x08015d79   Thumb Code    30  stm32f10x_tim.o(.text)
    TIM_ITConfig                             0x08015d97   Thumb Code    18  stm32f10x_tim.o(.text)
    TIM_GenerateEvent                        0x08015da9   Thumb Code     4  stm32f10x_tim.o(.text)
    TIM_DMAConfig                            0x08015dad   Thumb Code    10  stm32f10x_tim.o(.text)
    TIM_DMACmd                               0x08015db7   Thumb Code    18  stm32f10x_tim.o(.text)
    TIM_InternalClockConfig                  0x08015dc9   Thumb Code    12  stm32f10x_tim.o(.text)
    TIM_SelectInputTrigger                   0x08015dd5   Thumb Code    18  stm32f10x_tim.o(.text)
    TIM_ITRxExternalClockConfig              0x08015de7   Thumb Code    24  stm32f10x_tim.o(.text)
    TIM_TIxExternalClockConfig               0x08015dff   Thumb Code    62  stm32f10x_tim.o(.text)
    TIM_ETRConfig                            0x08015e3d   Thumb Code    28  stm32f10x_tim.o(.text)
    TIM_ETRClockMode1Config                  0x08015e59   Thumb Code    54  stm32f10x_tim.o(.text)
    TIM_ETRClockMode2Config                  0x08015e8f   Thumb Code    32  stm32f10x_tim.o(.text)
    TIM_PrescalerConfig                      0x08015eaf   Thumb Code     6  stm32f10x_tim.o(.text)
    TIM_CounterModeConfig                    0x08015eb5   Thumb Code    18  stm32f10x_tim.o(.text)
    TIM_EncoderInterfaceConfig               0x08015ec7   Thumb Code    66  stm32f10x_tim.o(.text)
    TIM_ForcedOC1Config                      0x08015f09   Thumb Code    18  stm32f10x_tim.o(.text)
    TIM_ForcedOC2Config                      0x08015f1b   Thumb Code    26  stm32f10x_tim.o(.text)
    TIM_ForcedOC3Config                      0x08015f35   Thumb Code    18  stm32f10x_tim.o(.text)
    TIM_ForcedOC4Config                      0x08015f47   Thumb Code    26  stm32f10x_tim.o(.text)
    TIM_ARRPreloadConfig                     0x08015f61   Thumb Code    24  stm32f10x_tim.o(.text)
    TIM_SelectCOM                            0x08015f79   Thumb Code    24  stm32f10x_tim.o(.text)
    TIM_SelectCCDMA                          0x08015f91   Thumb Code    24  stm32f10x_tim.o(.text)
    TIM_CCPreloadControl                     0x08015fa9   Thumb Code    24  stm32f10x_tim.o(.text)
    TIM_OC1PreloadConfig                     0x08015fc1   Thumb Code    18  stm32f10x_tim.o(.text)
    TIM_OC2PreloadConfig                     0x08015fd3   Thumb Code    26  stm32f10x_tim.o(.text)
    TIM_OC3PreloadConfig                     0x08015fed   Thumb Code    18  stm32f10x_tim.o(.text)
    TIM_OC4PreloadConfig                     0x08015fff   Thumb Code    26  stm32f10x_tim.o(.text)
    TIM_OC1FastConfig                        0x08016019   Thumb Code    18  stm32f10x_tim.o(.text)
    TIM_OC2FastConfig                        0x0801602b   Thumb Code    26  stm32f10x_tim.o(.text)
    TIM_OC3FastConfig                        0x08016045   Thumb Code    18  stm32f10x_tim.o(.text)
    TIM_OC4FastConfig                        0x08016057   Thumb Code    26  stm32f10x_tim.o(.text)
    TIM_ClearOC1Ref                          0x08016071   Thumb Code    18  stm32f10x_tim.o(.text)
    TIM_ClearOC2Ref                          0x08016083   Thumb Code    24  stm32f10x_tim.o(.text)
    TIM_ClearOC3Ref                          0x0801609b   Thumb Code    18  stm32f10x_tim.o(.text)
    TIM_ClearOC4Ref                          0x080160ad   Thumb Code    24  stm32f10x_tim.o(.text)
    TIM_OC1PolarityConfig                    0x080160c5   Thumb Code    18  stm32f10x_tim.o(.text)
    TIM_OC1NPolarityConfig                   0x080160d7   Thumb Code    18  stm32f10x_tim.o(.text)
    TIM_OC2PolarityConfig                    0x080160e9   Thumb Code    26  stm32f10x_tim.o(.text)
    TIM_OC2NPolarityConfig                   0x08016103   Thumb Code    26  stm32f10x_tim.o(.text)
    TIM_OC3PolarityConfig                    0x0801611d   Thumb Code    26  stm32f10x_tim.o(.text)
    TIM_OC3NPolarityConfig                   0x08016137   Thumb Code    26  stm32f10x_tim.o(.text)
    TIM_OC4PolarityConfig                    0x08016151   Thumb Code    26  stm32f10x_tim.o(.text)
    TIM_CCxCmd                               0x0801616b   Thumb Code    30  stm32f10x_tim.o(.text)
    TIM_CCxNCmd                              0x08016189   Thumb Code    30  stm32f10x_tim.o(.text)
    TIM_SelectOCxM                           0x080161a7   Thumb Code    82  stm32f10x_tim.o(.text)
    TIM_UpdateDisableConfig                  0x080161f9   Thumb Code    24  stm32f10x_tim.o(.text)
    TIM_UpdateRequestConfig                  0x08016211   Thumb Code    24  stm32f10x_tim.o(.text)
    TIM_SelectHallSensor                     0x08016229   Thumb Code    24  stm32f10x_tim.o(.text)
    TIM_SelectOnePulseMode                   0x08016241   Thumb Code    18  stm32f10x_tim.o(.text)
    TIM_SelectOutputTrigger                  0x08016253   Thumb Code    18  stm32f10x_tim.o(.text)
    TIM_SelectSlaveMode                      0x08016265   Thumb Code    18  stm32f10x_tim.o(.text)
    TIM_SelectMasterSlaveMode                0x08016277   Thumb Code    18  stm32f10x_tim.o(.text)
    TIM_SetCounter                           0x08016289   Thumb Code     4  stm32f10x_tim.o(.text)
    TIM_SetAutoreload                        0x0801628d   Thumb Code     4  stm32f10x_tim.o(.text)
    TIM_SetCompare1                          0x08016291   Thumb Code     4  stm32f10x_tim.o(.text)
    TIM_SetCompare2                          0x08016295   Thumb Code     4  stm32f10x_tim.o(.text)
    TIM_SetCompare3                          0x08016299   Thumb Code     4  stm32f10x_tim.o(.text)
    TIM_SetCompare4                          0x0801629d   Thumb Code     6  stm32f10x_tim.o(.text)
    TIM_SetClockDivision                     0x080162a3   Thumb Code    18  stm32f10x_tim.o(.text)
    TIM_GetCapture1                          0x080162b5   Thumb Code     6  stm32f10x_tim.o(.text)
    TIM_GetCapture2                          0x080162bb   Thumb Code     6  stm32f10x_tim.o(.text)
    TIM_GetCapture3                          0x080162c1   Thumb Code     6  stm32f10x_tim.o(.text)
    TIM_GetCapture4                          0x080162c7   Thumb Code     8  stm32f10x_tim.o(.text)
    TIM_GetCounter                           0x080162cf   Thumb Code     6  stm32f10x_tim.o(.text)
    TIM_GetPrescaler                         0x080162d5   Thumb Code     6  stm32f10x_tim.o(.text)
    TIM_GetFlagStatus                        0x080162db   Thumb Code    18  stm32f10x_tim.o(.text)
    TIM_ClearFlag                            0x080162ed   Thumb Code     6  stm32f10x_tim.o(.text)
    TIM_GetITStatus                          0x080162f3   Thumb Code    34  stm32f10x_tim.o(.text)
    TIM_ClearITPendingBit                    0x08016315   Thumb Code     6  stm32f10x_tim.o(.text)
    PWR_DeInit                               0x0801631d   Thumb Code    22  stm32f10x_pwr.o(.text)
    PWR_BackupAccessCmd                      0x08016333   Thumb Code     6  stm32f10x_pwr.o(.text)
    PWR_PVDCmd                               0x08016339   Thumb Code     6  stm32f10x_pwr.o(.text)
    PWR_PVDLevelConfig                       0x0801633f   Thumb Code    18  stm32f10x_pwr.o(.text)
    PWR_WakeUpPinCmd                         0x08016351   Thumb Code     8  stm32f10x_pwr.o(.text)
    PWR_EnterSTOPMode                        0x08016359   Thumb Code    54  stm32f10x_pwr.o(.text)
    PWR_EnterSTANDBYMode                     0x0801638f   Thumb Code    42  stm32f10x_pwr.o(.text)
    PWR_GetFlagStatus                        0x080163b9   Thumb Code    20  stm32f10x_pwr.o(.text)
    PWR_ClearFlag                            0x080163cd   Thumb Code    14  stm32f10x_pwr.o(.text)
    BKP_DeInit                               0x080163e9   Thumb Code    16  stm32f10x_bkp.o(.text)
    BKP_TamperPinLevelConfig                 0x080163f9   Thumb Code     6  stm32f10x_bkp.o(.text)
    BKP_TamperPinCmd                         0x080163ff   Thumb Code     8  stm32f10x_bkp.o(.text)
    BKP_ITConfig                             0x08016407   Thumb Code     8  stm32f10x_bkp.o(.text)
    BKP_RTCOutputConfig                      0x0801640f   Thumb Code    22  stm32f10x_bkp.o(.text)
    BKP_SetRTCCalibrationValue               0x08016425   Thumb Code    22  stm32f10x_bkp.o(.text)
    BKP_WriteBackupRegister                  0x0801643b   Thumb Code    24  stm32f10x_bkp.o(.text)
    BKP_ReadBackupRegister                   0x08016453   Thumb Code    26  stm32f10x_bkp.o(.text)
    BKP_GetFlagStatus                        0x0801646d   Thumb Code    10  stm32f10x_bkp.o(.text)
    BKP_ClearFlag                            0x08016477   Thumb Code    18  stm32f10x_bkp.o(.text)
    BKP_GetITStatus                          0x08016489   Thumb Code    10  stm32f10x_bkp.o(.text)
    BKP_ClearITPendingBit                    0x08016493   Thumb Code    18  stm32f10x_bkp.o(.text)
    FLASH_SetLatency                         0x080164ad   Thumb Code    18  stm32f10x_flash.o(.text)
    FLASH_HalfCycleAccessCmd                 0x080164bf   Thumb Code    22  stm32f10x_flash.o(.text)
    FLASH_PrefetchBufferCmd                  0x080164d5   Thumb Code    22  stm32f10x_flash.o(.text)
    FLASH_Unlock                             0x080164eb   Thumb Code    12  stm32f10x_flash.o(.text)
    FLASH_UnlockBank1                        0x080164f7   Thumb Code    12  stm32f10x_flash.o(.text)
    FLASH_Lock                               0x08016503   Thumb Code    14  stm32f10x_flash.o(.text)
    FLASH_LockBank1                          0x08016511   Thumb Code    14  stm32f10x_flash.o(.text)
    FLASH_GetBank1Status                     0x0801651f   Thumb Code    48  stm32f10x_flash.o(.text)
    FLASH_WaitForLastOperation               0x0801654f   Thumb Code    38  stm32f10x_flash.o(.text)
    FLASH_ErasePage                          0x08016575   Thumb Code    72  stm32f10x_flash.o(.text)
    FLASH_EraseAllPages                      0x080165bd   Thumb Code    68  stm32f10x_flash.o(.text)
    FLASH_WaitForLastBank1Operation          0x08016601   Thumb Code    38  stm32f10x_flash.o(.text)
    FLASH_EraseAllBank1Pages                 0x08016627   Thumb Code    68  stm32f10x_flash.o(.text)
    FLASH_GetReadOutProtectionStatus         0x0801666b   Thumb Code    20  stm32f10x_flash.o(.text)
    FLASH_EraseOptionBytes                   0x0801667f   Thumb Code   150  stm32f10x_flash.o(.text)
    FLASH_ProgramWord                        0x08016715   Thumb Code   102  stm32f10x_flash.o(.text)
    FLASH_ProgramHalfWord                    0x0801677b   Thumb Code    60  stm32f10x_flash.o(.text)
    FLASH_ProgramOptionByteData              0x080167b7   Thumb Code    72  stm32f10x_flash.o(.text)
    FLASH_EnableWriteProtection              0x080167ff   Thumb Code   200  stm32f10x_flash.o(.text)
    FLASH_ReadOutProtection                  0x080168c7   Thumb Code   156  stm32f10x_flash.o(.text)
    FLASH_UserOptionByteConfig               0x08016963   Thumb Code    88  stm32f10x_flash.o(.text)
    FLASH_GetUserOptionByte                  0x080169bb   Thumb Code     8  stm32f10x_flash.o(.text)
    FLASH_GetWriteProtectionOptionByte       0x080169c3   Thumb Code     6  stm32f10x_flash.o(.text)
    FLASH_GetPrefetchBufferStatus            0x080169c9   Thumb Code    20  stm32f10x_flash.o(.text)
    FLASH_ITConfig                           0x080169dd   Thumb Code    26  stm32f10x_flash.o(.text)
    FLASH_GetFlagStatus                      0x080169f7   Thumb Code    42  stm32f10x_flash.o(.text)
    FLASH_ClearFlag                          0x08016a21   Thumb Code     6  stm32f10x_flash.o(.text)
    FLASH_GetStatus                          0x08016a27   Thumb Code    48  stm32f10x_flash.o(.text)
    ADC_DeInit                               0x08016a69   Thumb Code    78  stm32f10x_adc.o(.text)
    ADC_Init                                 0x08016ab7   Thumb Code    70  stm32f10x_adc.o(.text)
    ADC_StructInit                           0x08016afd   Thumb Code    18  stm32f10x_adc.o(.text)
    ADC_Cmd                                  0x08016b0f   Thumb Code    22  stm32f10x_adc.o(.text)
    ADC_DMACmd                               0x08016b25   Thumb Code    22  stm32f10x_adc.o(.text)
    ADC_ITConfig                             0x08016b3b   Thumb Code    24  stm32f10x_adc.o(.text)
    ADC_ResetCalibration                     0x08016b53   Thumb Code    10  stm32f10x_adc.o(.text)
    ADC_GetResetCalibrationStatus            0x08016b5d   Thumb Code    20  stm32f10x_adc.o(.text)
    ADC_StartCalibration                     0x08016b71   Thumb Code    10  stm32f10x_adc.o(.text)
    ADC_GetCalibrationStatus                 0x08016b7b   Thumb Code    20  stm32f10x_adc.o(.text)
    ADC_SoftwareStartConvCmd                 0x08016b8f   Thumb Code    22  stm32f10x_adc.o(.text)
    ADC_GetSoftwareStartConvStatus           0x08016ba5   Thumb Code    20  stm32f10x_adc.o(.text)
    ADC_DiscModeChannelCountConfig           0x08016bb9   Thumb Code    24  stm32f10x_adc.o(.text)
    ADC_DiscModeCmd                          0x08016bd1   Thumb Code    22  stm32f10x_adc.o(.text)
    ADC_RegularChannelConfig                 0x08016be7   Thumb Code   184  stm32f10x_adc.o(.text)
    ADC_ExternalTrigConvCmd                  0x08016c9f   Thumb Code    22  stm32f10x_adc.o(.text)
    ADC_GetConversionValue                   0x08016cb5   Thumb Code     8  stm32f10x_adc.o(.text)
    ADC_GetDualModeConversionValue           0x08016cbd   Thumb Code     8  stm32f10x_adc.o(.text)
    ADC_AutoInjectedConvCmd                  0x08016cc5   Thumb Code    22  stm32f10x_adc.o(.text)
    ADC_InjectedDiscModeCmd                  0x08016cdb   Thumb Code    22  stm32f10x_adc.o(.text)
    ADC_ExternalTrigInjectedConvConfig       0x08016cf1   Thumb Code    16  stm32f10x_adc.o(.text)
    ADC_ExternalTrigInjectedConvCmd          0x08016d01   Thumb Code    22  stm32f10x_adc.o(.text)
    ADC_SoftwareStartInjectedConvCmd         0x08016d17   Thumb Code    22  stm32f10x_adc.o(.text)
    ADC_GetSoftwareStartInjectedConvCmdStatus 0x08016d2d   Thumb Code    20  stm32f10x_adc.o(.text)
    ADC_InjectedChannelConfig                0x08016d41   Thumb Code   130  stm32f10x_adc.o(.text)
    ADC_InjectedSequencerLengthConfig        0x08016dc3   Thumb Code    24  stm32f10x_adc.o(.text)
    ADC_SetInjectedOffset                    0x08016ddb   Thumb Code    20  stm32f10x_adc.o(.text)
    ADC_GetInjectedConversionValue           0x08016def   Thumb Code    28  stm32f10x_adc.o(.text)
    ADC_AnalogWatchdogCmd                    0x08016e0b   Thumb Code    16  stm32f10x_adc.o(.text)
    ADC_AnalogWatchdogThresholdsConfig       0x08016e1b   Thumb Code     6  stm32f10x_adc.o(.text)
    ADC_AnalogWatchdogSingleChannelConfig    0x08016e21   Thumb Code    16  stm32f10x_adc.o(.text)
    ADC_TempSensorVrefintCmd                 0x08016e31   Thumb Code    64  stm32f10x_adc.o(.text)
    ADC_GetFlagStatus                        0x08016e71   Thumb Code    18  stm32f10x_adc.o(.text)
    ADC_ClearFlag                            0x08016e83   Thumb Code     6  stm32f10x_adc.o(.text)
    ADC_GetITStatus                          0x08016e89   Thumb Code    36  stm32f10x_adc.o(.text)
    ADC_ClearITPendingBit                    0x08016ead   Thumb Code    10  stm32f10x_adc.o(.text)
    DMA_DeInit                               0x08016eb9   Thumb Code   324  stm32f10x_dma.o(.text)
    DMA_Init                                 0x08016ffd   Thumb Code    60  stm32f10x_dma.o(.text)
    DMA_StructInit                           0x08017039   Thumb Code    26  stm32f10x_dma.o(.text)
    DMA_Cmd                                  0x08017053   Thumb Code    24  stm32f10x_dma.o(.text)
    DMA_ITConfig                             0x0801706b   Thumb Code    18  stm32f10x_dma.o(.text)
    DMA_SetCurrDataCounter                   0x0801707d   Thumb Code     4  stm32f10x_dma.o(.text)
    DMA_GetCurrDataCounter                   0x08017081   Thumb Code     8  stm32f10x_dma.o(.text)
    DMA_GetFlagStatus                        0x08017089   Thumb Code    40  stm32f10x_dma.o(.text)
    DMA_ClearFlag                            0x080170b1   Thumb Code    22  stm32f10x_dma.o(.text)
    DMA_GetITStatus                          0x080170c7   Thumb Code    40  stm32f10x_dma.o(.text)
    DMA_ClearITPendingBit                    0x080170ef   Thumb Code    22  stm32f10x_dma.o(.text)
    Reset_Handler                            0x0801710d   Thumb Code     8  startup_stm32f10x_md.o(.text)
    ADC1_2_IRQHandler                        0x08017127   Thumb Code     0  startup_stm32f10x_md.o(.text)
    CAN1_RX1_IRQHandler                      0x08017127   Thumb Code     0  startup_stm32f10x_md.o(.text)
    CAN1_SCE_IRQHandler                      0x08017127   Thumb Code     0  startup_stm32f10x_md.o(.text)
    DMA1_Channel1_IRQHandler                 0x08017127   Thumb Code     0  startup_stm32f10x_md.o(.text)
    DMA1_Channel2_IRQHandler                 0x08017127   Thumb Code     0  startup_stm32f10x_md.o(.text)
    DMA1_Channel3_IRQHandler                 0x08017127   Thumb Code     0  startup_stm32f10x_md.o(.text)
    DMA1_Channel4_IRQHandler                 0x08017127   Thumb Code     0  startup_stm32f10x_md.o(.text)
    DMA1_Channel5_IRQHandler                 0x08017127   Thumb Code     0  startup_stm32f10x_md.o(.text)
    DMA1_Channel6_IRQHandler                 0x08017127   Thumb Code     0  startup_stm32f10x_md.o(.text)
    DMA1_Channel7_IRQHandler                 0x08017127   Thumb Code     0  startup_stm32f10x_md.o(.text)
    EXTI0_IRQHandler                         0x08017127   Thumb Code     0  startup_stm32f10x_md.o(.text)
    EXTI2_IRQHandler                         0x08017127   Thumb Code     0  startup_stm32f10x_md.o(.text)
    EXTI3_IRQHandler                         0x08017127   Thumb Code     0  startup_stm32f10x_md.o(.text)
    EXTI4_IRQHandler                         0x08017127   Thumb Code     0  startup_stm32f10x_md.o(.text)
    FLASH_IRQHandler                         0x08017127   Thumb Code     0  startup_stm32f10x_md.o(.text)
    I2C1_ER_IRQHandler                       0x08017127   Thumb Code     0  startup_stm32f10x_md.o(.text)
    I2C1_EV_IRQHandler                       0x08017127   Thumb Code     0  startup_stm32f10x_md.o(.text)
    I2C2_ER_IRQHandler                       0x08017127   Thumb Code     0  startup_stm32f10x_md.o(.text)
    I2C2_EV_IRQHandler                       0x08017127   Thumb Code     0  startup_stm32f10x_md.o(.text)
    PVD_IRQHandler                           0x08017127   Thumb Code     0  startup_stm32f10x_md.o(.text)
    RCC_IRQHandler                           0x08017127   Thumb Code     0  startup_stm32f10x_md.o(.text)
    RTCAlarm_IRQHandler                      0x08017127   Thumb Code     0  startup_stm32f10x_md.o(.text)
    RTC_IRQHandler                           0x08017127   Thumb Code     0  startup_stm32f10x_md.o(.text)
    SPI1_IRQHandler                          0x08017127   Thumb Code     0  startup_stm32f10x_md.o(.text)
    SPI2_IRQHandler                          0x08017127   Thumb Code     0  startup_stm32f10x_md.o(.text)
    TAMPER_IRQHandler                        0x08017127   Thumb Code     0  startup_stm32f10x_md.o(.text)
    TIM1_BRK_IRQHandler                      0x08017127   Thumb Code     0  startup_stm32f10x_md.o(.text)
    TIM1_CC_IRQHandler                       0x08017127   Thumb Code     0  startup_stm32f10x_md.o(.text)
    TIM1_TRG_COM_IRQHandler                  0x08017127   Thumb Code     0  startup_stm32f10x_md.o(.text)
    TIM1_UP_IRQHandler                       0x08017127   Thumb Code     0  startup_stm32f10x_md.o(.text)
    TIM2_IRQHandler                          0x08017127   Thumb Code     0  startup_stm32f10x_md.o(.text)
    TIM3_IRQHandler                          0x08017127   Thumb Code     0  startup_stm32f10x_md.o(.text)
    TIM4_IRQHandler                          0x08017127   Thumb Code     0  startup_stm32f10x_md.o(.text)
    USBWakeUp_IRQHandler                     0x08017127   Thumb Code     0  startup_stm32f10x_md.o(.text)
    USB_HP_CAN1_TX_IRQHandler                0x08017127   Thumb Code     0  startup_stm32f10x_md.o(.text)
    USB_LP_CAN1_RX0_IRQHandler               0x08017127   Thumb Code     0  startup_stm32f10x_md.o(.text)
    WWDG_IRQHandler                          0x08017127   Thumb Code     0  startup_stm32f10x_md.o(.text)
    delay_us                                 0x08017131   Thumb Code    46  delay.o(.text)
    TIM3_Int_Init                            0x0801715f   Thumb Code    82  delay.o(.text)
    at_send_simple_cmd                       0x080171b5   Thumb Code    28  at.o(.text)
    at_send_cmd                              0x080171d1   Thumb Code    62  at.o(.text)
    at_send_cmd_back                         0x0801720f   Thumb Code    80  at.o(.text)
    at_send_cmd_match_back                   0x0801725f   Thumb Code    90  at.o(.text)
    at_send_cmd_back_wait                    0x080172b9   Thumb Code    70  at.o(.text)
    at_send_byte                             0x080172ff   Thumb Code    48  at.o(.text)
    bc26_error_event                         0x08017e61   Thumb Code    36  bc26.o(.text)
    bc26_sleep_event                         0x08017e85   Thumb Code    14  bc26.o(.text)
    bc26_sal_init                            0x08017f3b   Thumb Code    46  bc26.o(.text)
    bc26_sal_register                        0x08017f69   Thumb Code    10  bc26.o(.text)
    channel_data_clear                       0x08017fdd   Thumb Code    40  module_wrapper.o(.text)
    at_module_register                       0x08018005   Thumb Code    22  module_wrapper.o(.text)
    at_module_register_default               0x0801801b   Thumb Code     8  module_wrapper.o(.text)
    at_module_start                          0x08018023   Thumb Code    26  module_wrapper.o(.text)
    at_module_init                           0x0801803d   Thumb Code    32  module_wrapper.o(.text)
    at_module_connect                        0x0801805d   Thumb Code    34  module_wrapper.o(.text)
    at_module_udpopen                        0x0801807f   Thumb Code    34  module_wrapper.o(.text)
    at_module_reconnect                      0x080180a1   Thumb Code    34  module_wrapper.o(.text)
    at_module_udpreopen                      0x080180c3   Thumb Code    34  module_wrapper.o(.text)
    at_module_channel_open                   0x080180e5   Thumb Code    48  module_wrapper.o(.text)
    at_module_channel_reopen                 0x08018115   Thumb Code    48  module_wrapper.o(.text)
    at_module_close                          0x08018145   Thumb Code    26  module_wrapper.o(.text)
    at_module_channel_close                  0x0801815f   Thumb Code    30  module_wrapper.o(.text)
    at_module_tcpstate                       0x0801817d   Thumb Code    32  module_wrapper.o(.text)
    at_module_channel_state                  0x0801819d   Thumb Code    36  module_wrapper.o(.text)
    at_module_send                           0x080181c1   Thumb Code    40  module_wrapper.o(.text)
    at_module_send_rai                       0x080181e9   Thumb Code    44  module_wrapper.o(.text)
    at_module_send_ch                        0x08018215   Thumb Code    54  module_wrapper.o(.text)
    at_module_recv_timeout                   0x0801824b   Thumb Code    44  module_wrapper.o(.text)
    at_module_handle_event                   0x08018277   Thumb Code    26  module_wrapper.o(.text)
    at_module_cmd_back                       0x08018291   Thumb Code    38  module_wrapper.o(.text)
    at_module_cmd                            0x080182b7   Thumb Code    30  module_wrapper.o(.text)
    at_module_low_power                      0x080182d5   Thumb Code    26  module_wrapper.o(.text)
    cJSON_GetErrorPtr                        0x080182f9   Thumb Code    12  cjson.o(.text)
    cJSON_IsString                           0x08018305   Thumb Code    22  cjson.o(.text)
    cJSON_GetStringValue                     0x0801831b   Thumb Code    20  cjson.o(.text)
    cJSON_IsNumber                           0x0801832f   Thumb Code    22  cjson.o(.text)
    cJSON_GetNumberValue                     0x08018345   Thumb Code    24  cjson.o(.text)
    cJSON_Version                            0x0801835d   Thumb Code    22  cjson.o(.text)
    cJSON_InitHooks                          0x080183f3   Thumb Code    82  cjson.o(.text)
    cJSON_Delete                             0x0801845f   Thumb Code    84  cjson.o(.text)
    cJSON_SetNumberHelper                    0x080185e1   Thumb Code    72  cjson.o(.text)
    cJSON_free                               0x08018629   Thumb Code    14  cjson.o(.text)
    cJSON_SetValuestring                     0x08018637   Thumb Code    94  cjson.o(.text)
    cJSON_ParseWithLengthOpts                0x080191e5   Thumb Code   204  cjson.o(.text)
    cJSON_ParseWithOpts                      0x080192b1   Thumb Code    40  cjson.o(.text)
    cJSON_Parse                              0x080192d9   Thumb Code    16  cjson.o(.text)
    cJSON_ParseWithLength                    0x080192e9   Thumb Code    20  cjson.o(.text)
    cJSON_Print                              0x080196e1   Thumb Code    16  cjson.o(.text)
    cJSON_PrintUnformatted                   0x080196f1   Thumb Code    16  cjson.o(.text)
    cJSON_PrintBuffered                      0x08019701   Thumb Code    90  cjson.o(.text)
    cJSON_PrintPreallocated                  0x0801975b   Thumb Code    64  cjson.o(.text)
    cJSON_GetArraySize                       0x0801979b   Thumb Code    28  cjson.o(.text)
    cJSON_GetArrayItem                       0x080197d5   Thumb Code    24  cjson.o(.text)
    cJSON_GetObjectItem                      0x0801983f   Thumb Code    18  cjson.o(.text)
    cJSON_GetObjectItemCaseSensitive         0x08019851   Thumb Code    18  cjson.o(.text)
    cJSON_HasObjectItem                      0x08019863   Thumb Code    24  cjson.o(.text)
    cJSON_AddItemToArray                     0x080198f3   Thumb Code    16  cjson.o(.text)
    cJSON_AddItemToObject                    0x0801997f   Thumb Code    26  cjson.o(.text)
    cJSON_AddItemToObjectCS                  0x08019999   Thumb Code    26  cjson.o(.text)
    cJSON_AddItemReferenceToArray            0x080199b3   Thumb Code    32  cjson.o(.text)
    cJSON_AddItemReferenceToObject           0x080199d3   Thumb Code    44  cjson.o(.text)
    cJSON_CreateNull                         0x080199ff   Thumb Code    20  cjson.o(.text)
    cJSON_AddNullToObject                    0x08019a13   Thumb Code    44  cjson.o(.text)
    cJSON_CreateTrue                         0x08019a3f   Thumb Code    20  cjson.o(.text)
    cJSON_AddTrueToObject                    0x08019a53   Thumb Code    44  cjson.o(.text)
    cJSON_CreateFalse                        0x08019a7f   Thumb Code    20  cjson.o(.text)
    cJSON_AddFalseToObject                   0x08019a93   Thumb Code    44  cjson.o(.text)
    cJSON_CreateBool                         0x08019abf   Thumb Code    34  cjson.o(.text)
    cJSON_AddBoolToObject                    0x08019ae1   Thumb Code    48  cjson.o(.text)
    cJSON_CreateNumber                       0x08019b11   Thumb Code    82  cjson.o(.text)
    cJSON_AddNumberToObject                  0x08019b63   Thumb Code    56  cjson.o(.text)
    cJSON_CreateString                       0x08019b9b   Thumb Code    46  cjson.o(.text)
    cJSON_AddStringToObject                  0x08019bc9   Thumb Code    48  cjson.o(.text)
    cJSON_CreateRaw                          0x08019bf9   Thumb Code    46  cjson.o(.text)
    cJSON_AddRawToObject                     0x08019c27   Thumb Code    48  cjson.o(.text)
    cJSON_CreateObject                       0x08019c57   Thumb Code    20  cjson.o(.text)
    cJSON_AddObjectToObject                  0x08019c6b   Thumb Code    44  cjson.o(.text)
    cJSON_CreateArray                        0x08019c97   Thumb Code    20  cjson.o(.text)
    cJSON_AddArrayToObject                   0x08019cab   Thumb Code    44  cjson.o(.text)
    cJSON_DetachItemViaPointer               0x08019cd7   Thumb Code    64  cjson.o(.text)
    cJSON_DetachItemFromArray                0x08019d17   Thumb Code    34  cjson.o(.text)
    cJSON_DeleteItemFromArray                0x08019d39   Thumb Code    22  cjson.o(.text)
    cJSON_DetachItemFromObject               0x08019d4f   Thumb Code    26  cjson.o(.text)
    cJSON_DetachItemFromObjectCaseSensitive  0x08019d69   Thumb Code    26  cjson.o(.text)
    cJSON_DeleteItemFromObject               0x08019d83   Thumb Code    22  cjson.o(.text)
    cJSON_DeleteItemFromObjectCaseSensitive  0x08019d99   Thumb Code    22  cjson.o(.text)
    cJSON_InsertItemInArray                  0x08019daf   Thumb Code    70  cjson.o(.text)
    cJSON_ReplaceItemViaPointer              0x08019df5   Thumb Code    96  cjson.o(.text)
    cJSON_ReplaceItemInArray                 0x08019e55   Thumb Code    42  cjson.o(.text)
    cJSON_ReplaceItemInObject                0x08019ee1   Thumb Code    22  cjson.o(.text)
    cJSON_ReplaceItemInObjectCaseSensitive   0x08019ef7   Thumb Code    22  cjson.o(.text)
    cJSON_CreateStringReference              0x08019f0d   Thumb Code    32  cjson.o(.text)
    cJSON_CreateObjectReference              0x08019f2d   Thumb Code    32  cjson.o(.text)
    cJSON_CreateArrayReference               0x08019f4d   Thumb Code    32  cjson.o(.text)
    cJSON_CreateIntArray                     0x08019f6d   Thumb Code   110  cjson.o(.text)
    cJSON_CreateFloatArray                   0x08019fdb   Thumb Code   110  cjson.o(.text)
    cJSON_CreateDoubleArray                  0x0801a049   Thumb Code   106  cjson.o(.text)
    cJSON_CreateStringArray                  0x0801a0b3   Thumb Code   100  cjson.o(.text)
    cJSON_Duplicate                          0x0801a117   Thumb Code   188  cjson.o(.text)
    cJSON_Minify                             0x0801a2a3   Thumb Code   160  cjson.o(.text)
    cJSON_IsInvalid                          0x0801a343   Thumb Code    20  cjson.o(.text)
    cJSON_IsFalse                            0x0801a357   Thumb Code    20  cjson.o(.text)
    cJSON_IsTrue                             0x0801a36b   Thumb Code    22  cjson.o(.text)
    cJSON_IsBool                             0x0801a381   Thumb Code    24  cjson.o(.text)
    cJSON_IsNull                             0x0801a399   Thumb Code    22  cjson.o(.text)
    cJSON_IsArray                            0x0801a3af   Thumb Code    22  cjson.o(.text)
    cJSON_IsObject                           0x0801a3c5   Thumb Code    22  cjson.o(.text)
    cJSON_IsRaw                              0x0801a3db   Thumb Code    22  cjson.o(.text)
    cJSON_Compare                            0x0801a3f1   Thumb Code   384  cjson.o(.text)
    cJSON_malloc                             0x0801a571   Thumb Code    14  cjson.o(.text)
    InvertUint8                              0x0801a585   Thumb Code    56  crc.o(.text)
    InvertUint16                             0x0801a5bd   Thumb Code    58  crc.o(.text)
    InvertUint32                             0x0801a5f7   Thumb Code    54  crc.o(.text)
    CRC16_CCITT                              0x0801a62d   Thumb Code    72  crc.o(.text)
    ReadProgramData                          0x0801a675   Thumb Code    16  programdata.o(.text)
    WriteProgramData                         0x0801a685   Thumb Code    16  programdata.o(.text)
    WriteInitProgramData                     0x0801a695   Thumb Code    26  programdata.o(.text)
    byteToHexStr                             0x0801a6b9   Thumb Code    78  sys.o(.text)
    letterSwitch                             0x0801a707   Thumb Code    52  sys.o(.text)
    inttohex                                 0x0801a73b   Thumb Code   104  sys.o(.text)
    my_atoi                                  0x0801a7a3   Thumb Code    54  sys.o(.text)
    my_atoui64                               0x0801a7d9   Thumb Code    76  sys.o(.text)
    my_atoabs                                0x0801a825   Thumb Code    42  sys.o(.text)
    my_itoa                                  0x0801a84f   Thumb Code   150  sys.o(.text)
    split                                    0x0801a8e5   Thumb Code    84  sys.o(.text)
    splitCharLimit                           0x0801a939   Thumb Code    92  sys.o(.text)
    delay_ms                                 0x0801a995   Thumb Code    26  sys.o(.text)
    Usart_SendString                         0x0801a9af   Thumb Code    50  sys.o(.text)
    UsartPrintf                              0x0801a9e1   Thumb Code    76  sys.o(.text)
    uart_recv_clear                          0x0801aa2d   Thumb Code    26  sys.o(.text)
    valid_data_clear                         0x0801aa47   Thumb Code    22  sys.o(.text)
    uart_recv_wait                           0x0801aa5d   Thumb Code    92  sys.o(.text)
    uart_recv_match_wait                     0x0801aab9   Thumb Code    80  sys.o(.text)
    AesEncrypt                               0x0801ade9   Thumb Code    86  aes.o(.text)
    AesDecrypt                               0x0801ae3f   Thumb Code    84  aes.o(.text)
    ScheduleKey                              0x0801ae93   Thumb Code   200  aes.o(.text)
    fillSrcData                              0x0801af5b   Thumb Code    70  aes.o(.text)
    ECBAesEncrypt                            0x0801afa1   Thumb Code    58  aes.o(.text)
    cutSrcData                               0x0801afdb   Thumb Code    38  aes.o(.text)
    ECBAesDecrypt                            0x0801b001   Thumb Code    56  aes.o(.text)
    utils_hmac_sha1_str                      0x0801b0b5   Thumb Code   202  mbedtls_util.o(.text)
    utils_sha256                             0x0801b17f   Thumb Code    46  mbedtls_util.o(.text)
    utils_sha256_str                         0x0801b1ad   Thumb Code    34  mbedtls_util.o(.text)
    utils_aes128_cbc_enc                     0x0801b1cf   Thumb Code   140  mbedtls_util.o(.text)
    utils_aes128_cbc_dec                     0x0801b25b   Thumb Code   114  mbedtls_util.o(.text)
    utils_aes128_cbc_base64_enc              0x0801b2cd   Thumb Code   104  mbedtls_util.o(.text)
    utils_aes128_cbc_base64_dec              0x0801b335   Thumb Code   110  mbedtls_util.o(.text)
    coap_parseHeader                         0x0801b3fd   Thumb Code    60  coap.o(.text)
    coap_parseToken                          0x0801b439   Thumb Code    50  coap.o(.text)
    coap_parseOption                         0x0801b46b   Thumb Code   222  coap.o(.text)
    coap_parseOptionsAndPayload              0x0801b549   Thumb Code   146  coap.o(.text)
    coap_parse                               0x0801b5db   Thumb Code    84  coap.o(.text)
    coap_findOptions                         0x0801b62f   Thumb Code    70  coap.o(.text)
    coap_buffer_to_string                    0x0801b675   Thumb Code    40  coap.o(.text)
    coap_option_nibble                       0x0801b69d   Thumb Code    32  coap.o(.text)
    coap_build                               0x0801b6bd   Thumb Code   484  coap.o(.text)
    coap_make_response                       0x0801b8a1   Thumb Code   118  coap.o(.text)
    coap_handle_req                          0x0801b917   Thumb Code   204  coap.o(.text)
    coap_setup                               0x0801b9e3   Thumb Code     2  coap.o(.text)
    endpoint_setup                           0x0801b9ed   Thumb Code     2  coaphandle.o(.text)
    CoapPublish                              0x0801ba69   Thumb Code   604  coaphandle.o(.text)
    CoapConnect                              0x0801c2d5   Thumb Code   444  coaphandle.o(.text)
    freshSignal                              0x0801c491   Thumb Code   146  coaphandle.o(.text)
    CoapHandleEvent                          0x0801c991   Thumb Code    22  coaphandle.o(.text)
    CoapHandle                               0x0801ca39   Thumb Code    92  coaphandle.o(.text)
    ModelRegister                            0x0801ca95   Thumb Code    50  coaphandle.o(.text)
    GetModeldBm                              0x0801cac7   Thumb Code    86  coaphandle.o(.text)
    GetModelCSQ                              0x0801cb1d   Thumb Code    62  coaphandle.o(.text)
    GetSignalDetail                          0x0801cb5b   Thumb Code   568  coaphandle.o(.text)
    ModuleKeepLine                           0x0801ce05   Thumb Code    78  regist.o(.text)
    DeviceRegist                             0x0801d03d   Thumb Code   228  regist.o(.text)
    remoteHandle                             0x0801d505   Thumb Code   148  remote.o(.text)
    mbedtls_aes_init                         0x0801d73d   Thumb Code    20  aes_1.o(.text)
    mbedtls_aes_free                         0x0801d751   Thumb Code    22  aes_1.o(.text)
    mbedtls_aes_setkey_enc                   0x0801d767   Thumb Code   504  aes_1.o(.text)
    mbedtls_aes_setkey_dec                   0x0801d95f   Thumb Code   210  aes_1.o(.text)
    mbedtls_internal_aes_encrypt             0x0801da31   Thumb Code  1186  aes_1.o(.text)
    mbedtls_aes_encrypt                      0x0801ded3   Thumb Code    20  aes_1.o(.text)
    mbedtls_internal_aes_decrypt             0x0801dee7   Thumb Code  1182  aes_1.o(.text)
    mbedtls_aes_decrypt                      0x0801e385   Thumb Code    20  aes_1.o(.text)
    mbedtls_aes_crypt_ecb                    0x0801e399   Thumb Code    58  aes_1.o(.text)
    mbedtls_aes_crypt_cbc                    0x0801e3d3   Thumb Code   234  aes_1.o(.text)
    mbedtls_base64_encode                    0x0801e4bd   Thumb Code   316  base64.o(.text)
    mbedtls_base64_decode                    0x0801e5f9   Thumb Code   364  base64.o(.text)
    mbedtls_ct_memcmp                        0x0801e765   Thumb Code    54  constant_time.o(.text)
    mbedtls_ct_uint_mask                     0x0801e79b   Thumb Code    12  constant_time.o(.text)
    mbedtls_ct_size_bool_eq                  0x0801e7bd   Thumb Code    22  constant_time.o(.text)
    mbedtls_ct_uint_if                       0x0801e7d3   Thumb Code    26  constant_time.o(.text)
    mbedtls_ct_base64_enc_char               0x0801e7ed   Thumb Code    94  constant_time.o(.text)
    mbedtls_ct_base64_dec_value              0x0801e84b   Thumb Code   100  constant_time.o(.text)
    mbedtls_platform_zeroize                 0x0801e8b1   Thumb Code    26  platform_util.o(.text)
    mbedtls_sha1_init                        0x0801e8d1   Thumb Code    18  sha1.o(.text)
    mbedtls_sha1_free                        0x0801e8e3   Thumb Code    20  sha1.o(.text)
    mbedtls_sha1_clone                       0x0801e8f7   Thumb Code    26  sha1.o(.text)
    mbedtls_sha1_starts_ret                  0x0801e911   Thumb Code    38  sha1.o(.text)
    mbedtls_sha1_starts                      0x0801e937   Thumb Code    12  sha1.o(.text)
    mbedtls_internal_sha1_process            0x0801e943   Thumb Code  6632  sha1.o(.text)
    mbedtls_sha1_process                     0x0802032b   Thumb Code    16  sha1.o(.text)
    mbedtls_sha1_update_ret                  0x0802033b   Thumb Code   158  sha1.o(.text)
    mbedtls_sha1_update                      0x080203d9   Thumb Code    20  sha1.o(.text)
    mbedtls_sha1_finish_ret                  0x080203ed   Thumb Code   304  sha1.o(.text)
    mbedtls_sha1_finish                      0x0802051d   Thumb Code    16  sha1.o(.text)
    mbedtls_sha1_ret                         0x0802052d   Thumb Code    84  sha1.o(.text)
    mbedtls_sha1                             0x08020581   Thumb Code    20  sha1.o(.text)
    mbedtls_sha256_init                      0x08020599   Thumb Code    18  sha256.o(.text)
    mbedtls_sha256_free                      0x080205ab   Thumb Code    20  sha256.o(.text)
    mbedtls_sha256_clone                     0x080205bf   Thumb Code    26  sha256.o(.text)
    mbedtls_sha256_starts_ret                0x080205d9   Thumb Code    90  sha256.o(.text)
    mbedtls_sha256_starts                    0x08020633   Thumb Code    16  sha256.o(.text)
    mbedtls_internal_sha256_process          0x08020643   Thumb Code  3834  sha256.o(.text)
    mbedtls_sha256_process                   0x0802153d   Thumb Code    16  sha256.o(.text)
    mbedtls_sha256_update_ret                0x0802154d   Thumb Code   158  sha256.o(.text)
    mbedtls_sha256_update                    0x080215eb   Thumb Code    20  sha256.o(.text)
    mbedtls_sha256_finish_ret                0x080215ff   Thumb Code   382  sha256.o(.text)
    mbedtls_sha256_finish                    0x0802177d   Thumb Code    16  sha256.o(.text)
    mbedtls_sha256_ret                       0x0802178d   Thumb Code   102  sha256.o(.text)
    mbedtls_sha256                           0x080217f3   Thumb Code    28  sha256.o(.text)
    __aeabi_uldivmod                         0x0802180f   Thumb Code    98  uldiv.o(.text)
    tolower                                  0x08021871   Thumb Code    12  tolower.o(.text)
    rand                                     0x0802187d   Thumb Code    20  rand.o(.text)
    srand                                    0x08021891   Thumb Code     6  rand.o(.text)
    __aeabi_memcpy                           0x080218a1   Thumb Code    36  memcpya.o(.text)
    __aeabi_memcpy4                          0x080218a1   Thumb Code     0  memcpya.o(.text)
    __aeabi_memcpy8                          0x080218a1   Thumb Code     0  memcpya.o(.text)
    __aeabi_memset                           0x080218c5   Thumb Code    14  memseta.o(.text)
    __aeabi_memset4                          0x080218c5   Thumb Code     0  memseta.o(.text)
    __aeabi_memset8                          0x080218c5   Thumb Code     0  memseta.o(.text)
    __aeabi_memclr                           0x080218d3   Thumb Code     4  memseta.o(.text)
    __aeabi_memclr4                          0x080218d3   Thumb Code     0  memseta.o(.text)
    __aeabi_memclr8                          0x080218d3   Thumb Code     0  memseta.o(.text)
    memset                                   0x080218d7   Thumb Code    18  memseta.o(.text)
    strstr                                   0x080218e9   Thumb Code    36  strstr.o(.text)
    strlen                                   0x0802190d   Thumb Code    14  strlen.o(.text)
    strcmp                                   0x0802191b   Thumb Code    28  strcmp.o(.text)
    memcmp                                   0x08021937   Thumb Code    26  memcmp.o(.text)
    strcpy                                   0x08021951   Thumb Code    18  strcpy.o(.text)
    strncmp                                  0x08021963   Thumb Code    30  strncmp.o(.text)
    strtok                                   0x08021981   Thumb Code    62  strtok.o(.text)
    __0sscanf                                0x080219c5   Thumb Code    48  __0sscanf.o(.text)
    _scanf_real                              0x08021afd   Thumb Code     0  scanf_fp.o(.text)
    _scanf_really_real                       0x08021afd   Thumb Code   556  scanf_fp.o(.text)
    __aeabi_dadd                             0x08021d35   Thumb Code   322  dadd.o(.text)
    __aeabi_dsub                             0x08021e77   Thumb Code     6  dadd.o(.text)
    __aeabi_drsub                            0x08021e7d   Thumb Code     6  dadd.o(.text)
    __aeabi_dmul                             0x08021e83   Thumb Code   228  dmul.o(.text)
    __aeabi_i2d                              0x08021f67   Thumb Code    34  dflti.o(.text)
    __aeabi_d2iz                             0x08021f89   Thumb Code    62  dfixi.o(.text)
    __aeabi_f2d                              0x08021fc7   Thumb Code    38  f2d.o(.text)
    __aeabi_cdcmpeq                          0x08021fed   Thumb Code     0  cdcmple.o(.text)
    __aeabi_cdcmple                          0x08021fed   Thumb Code    48  cdcmple.o(.text)
    __aeabi_cdrcmple                         0x0802201d   Thumb Code    48  cdrcmple.o(.text)
    __aeabi_uidiv                            0x0802204d   Thumb Code     0  uidiv.o(.text)
    __aeabi_uidivmod                         0x0802204d   Thumb Code    44  uidiv.o(.text)
    __aeabi_llsl                             0x08022079   Thumb Code    30  llshl.o(.text)
    _ll_shift_l                              0x08022079   Thumb Code     0  llshl.o(.text)
    __aeabi_llsr                             0x08022097   Thumb Code    32  llushr.o(.text)
    _ll_ushift_r                             0x08022097   Thumb Code     0  llushr.o(.text)
    __aeabi_lasr                             0x080220b7   Thumb Code    36  llsshr.o(.text)
    _ll_sshift_r                             0x080220b7   Thumb Code     0  llsshr.o(.text)
    __vfscanf_char                           0x080220e9   Thumb Code    20  scanf_char.o(.text)
    _sgetc                                   0x08022105   Thumb Code    30  _sgetc.o(.text)
    _sbackspace                              0x08022123   Thumb Code    34  _sgetc.o(.text)
    __strtod_int                             0x0802217b   Thumb Code    90  strtod.o(.text)
    __I$use$fp                               0x080221e1   Thumb Code     0  iusefp.o(.text)
    _double_round                            0x080221e1   Thumb Code    30  depilogue.o(.text)
    _double_epilogue                         0x080221ff   Thumb Code   156  depilogue.o(.text)
    __aeabi_ddiv                             0x0802229b   Thumb Code   222  ddiv.o(.text)
    __aeabi_ul2d                             0x08022379   Thumb Code    24  dfltul.o(.text)
    __aeabi_d2ulz                            0x08022391   Thumb Code    48  dfixul.o(.text)
    __aeabi_d2f                              0x080223c1   Thumb Code    56  d2f.o(.text)
    __scatterload                            0x080223f9   Thumb Code    28  init.o(.text)
    __scatterload_rt2                        0x080223f9   Thumb Code     0  init.o(.text)
    isspace                                  0x0802241d   Thumb Code    10  isspace_c.o(.text)
    __vfscanf                                0x08022429   Thumb Code   808  _scanf.o(.text)
    _float_round                             0x08022755   Thumb Code    18  fepilogue.o(.text)
    _float_epilogue                          0x08022767   Thumb Code    92  fepilogue.o(.text)
    __ctype_lookup                           0x080227c5   Thumb Code    34  ctype_c.o(.text)
    __decompress                             0x080227ed   Thumb Code     0  __dczerorl2.o(.text)
    __decompress1                            0x080227ed   Thumb Code    86  __dczerorl2.o(.text)
    __0printf                                0x08022845   Thumb Code    22  printfa.o(i.__0printf)
    __1printf                                0x08022845   Thumb Code     0  printfa.o(i.__0printf)
    __2printf                                0x08022845   Thumb Code     0  printfa.o(i.__0printf)
    __c89printf                              0x08022845   Thumb Code     0  printfa.o(i.__0printf)
    printf                                   0x08022845   Thumb Code     0  printfa.o(i.__0printf)
    __0snprintf                              0x08022865   Thumb Code    44  printfa.o(i.__0snprintf)
    __1snprintf                              0x08022865   Thumb Code     0  printfa.o(i.__0snprintf)
    __2snprintf                              0x08022865   Thumb Code     0  printfa.o(i.__0snprintf)
    __c89snprintf                            0x08022865   Thumb Code     0  printfa.o(i.__0snprintf)
    snprintf                                 0x08022865   Thumb Code     0  printfa.o(i.__0snprintf)
    __0sprintf                               0x08022895   Thumb Code    34  printfa.o(i.__0sprintf)
    __1sprintf                               0x08022895   Thumb Code     0  printfa.o(i.__0sprintf)
    __2sprintf                               0x08022895   Thumb Code     0  printfa.o(i.__0sprintf)
    __c89sprintf                             0x08022895   Thumb Code     0  printfa.o(i.__0sprintf)
    sprintf                                  0x08022895   Thumb Code     0  printfa.o(i.__0sprintf)
    __0vsnprintf                             0x080228bd   Thumb Code    40  printfa.o(i.__0vsnprintf)
    __1vsnprintf                             0x080228bd   Thumb Code     0  printfa.o(i.__0vsnprintf)
    __2vsnprintf                             0x080228bd   Thumb Code     0  printfa.o(i.__0vsnprintf)
    __c89vsnprintf                           0x080228bd   Thumb Code     0  printfa.o(i.__0vsnprintf)
    vsnprintf                                0x080228bd   Thumb Code     0  printfa.o(i.__0vsnprintf)
    free                                     0x080228e9   Thumb Code    88  mallocr.o(i.__free$realloc)
    malloc                                   0x08022945   Thumb Code    64  mallocr.o(i.__malloc$realloc)
    __scatterload_copy                       0x08022995   Thumb Code    14  handlers.o(i.__scatterload_copy)
    __scatterload_null                       0x080229a3   Thumb Code     2  handlers.o(i.__scatterload_null)
    __scatterload_zeroinit                   0x080229a5   Thumb Code    14  handlers.o(i.__scatterload_zeroinit)
    _is_digit                                0x08022b39   Thumb Code    14  scanf_fp.o(i._is_digit)
    realloc                                  0x080232e9   Thumb Code   102  mallocr.o(i.realloc)
    strtod                                   0x08023355   Thumb Code    28  strtod.o(i.strtod)
    table_week                               0x08023370   Data          12  rtcsetup.o(.constdata)
    mon_table                                0x0802337c   Data          12  rtcsetup.o(.constdata)
    asc8                                     0x08023388   Data         576  drawlcdgui.o(.constdata)
    asc12                                    0x080235c8   Data        1248  drawlcdgui.o(.constdata)
    asc16                                    0x08023aa8   Data        1632  drawlcdgui.o(.constdata)
    hz12                                     0x08024108   Data        3888  drawlcdgui.o(.constdata)
    hz16                                     0x08025038   Data        1890  drawlcdgui.o(.constdata)
    hz24                                     0x0802579a   Data         300  drawlcdgui.o(.constdata)
    auchCRCHi                                0x080258c6   Data         256  crc16.o(.constdata)
    auchCRCLo                                0x080259c6   Data         256  crc16.o(.constdata)
    __ctype_categories                       0x08028018   Data          64  ctype_c.o(.constdata)
    Region$$Table$$Base                      0x08028170   Number         0  anon$$obj.o(Region$$Table)
    Region$$Table$$Limit                     0x08028190   Number         0  anon$$obj.o(Region$$Table)
    mcu_id                                   0x20000000   Data           8  driver.o(.data)
    KeyScanStatus                            0x20000008   Data           8  typedefine.o(.data)
    KeyActionFlag                            0x20000010   Data           8  typedefine.o(.data)
    KeyScanQty                               0x20000018   Data           8  typedefine.o(.data)
    MoreKeyActionFlag                        0x20000020   Data           8  typedefine.o(.data)
    motorWorkState                           0x20000028   Data           1  typedefine.o(.data)
    displayTimeBuf                           0x2000002a   Data           8  typedefine.o(.data)
    dateLimit                                0x20000032   Data           1  typedefine.o(.data)
    alarmRecord                              0x20000033   Data           5  typedefine.o(.data)
    emSetTimeChoose                          0x20000038   Data           1  typedefine.o(.data)
    setTimeBuf                               0x2000003a   Data           8  typedefine.o(.data)
    setPasswordBuf                           0x20000042   Data           3  typedefine.o(.data)
    verifyPasswordBuf                        0x20000045   Data           3  typedefine.o(.data)
    emEvaluateTransfuseChoose                0x20000048   Data           1  typedefine.o(.data)
    emEngineeringMode1Choose                 0x20000049   Data           1  typedefine.o(.data)
    emEngineeringMode3Choose                 0x2000004a   Data           1  typedefine.o(.data)
    emPictureRunState                        0x2000004b   Data           1  typedefine.o(.data)
    HornWorkStep                             0x2000004c   Data           1  typedefine.o(.data)
    speakerWorkStep                          0x2000004d   Data           1  typedefine.o(.data)
    sysPromptToneType                        0x2000004e   Data           1  typedefine.o(.data)
    SysHornToneType                          0x2000004f   Data           1  typedefine.o(.data)
    sysPromptToneCounts                      0x20000050   Data           1  typedefine.o(.data)
    testDispCounts                           0x20000051   Data           1  typedefine.o(.data)
    FirstSurplusDose                         0x20000052   Data           1  typedefine.o(.data)
    PCASurplusDose                           0x20000053   Data           1  typedefine.o(.data)
    IC2Value                                 0x20000054   Data           2  stm32f10x_it.o(.data)
    DutyCycle                                0x20000056   Data           2  stm32f10x_it.o(.data)
    Frequency                                0x20000058   Data           4  stm32f10x_it.o(.data)
    EXPCA_flag                               0x2000005c   Data           1  stm32f10x_it.o(.data)
    Quiet_Timedata                           0x2000005e   Data           2  stm32f10x_it.o(.data)
    Quiet_Timedata_flag                      0x20000060   Data           1  stm32f10x_it.o(.data)
    lorawan_overtime                         0x20000062   Data           2  stm32f10x_it.o(.data)
    lorawan_overtime_flag                    0x20000064   Data           1  stm32f10x_it.o(.data)
    time_1sflag                              0x20000065   Data           1  stm32f10x_it.o(.data)
    time_3sflag                              0x20000066   Data           1  stm32f10x_it.o(.data)
    time_3s                                  0x20000068   Data           2  stm32f10x_it.o(.data)
    lorawan_time_5s                          0x2000006a   Data           2  stm32f10x_it.o(.data)
    lorawan_time_5sflag                      0x2000006c   Data           1  stm32f10x_it.o(.data)
    test_flag                                0x2000006d   Data           1  stm32f10x_it.o(.data)
    self_check_finish                        0x2000006e   Data           1  stm32f10x_it.o(.data)
    random_time                              0x20000070   Data           4  stm32f10x_it.o(.data)
    random_cont                              0x20000074   Data           2  stm32f10x_it.o(.data)
    random_data                              0x20000078   Data           4  stm32f10x_it.o(.data)
    lorawan_send_finish_flag                 0x2000007c   Data           1  stm32f10x_it.o(.data)
    pressureFZero                            0x20000082   Data           2  ads1110setup.o(.data)
    pressureFZero2                           0x20000084   Data           2  ads1110setup.o(.data)
    pressureCounts                           0x20000086   Data           2  ads1110setup.o(.data)
    Pressurebf_Cont                          0x20000088   Data           1  ads1110setup.o(.data)
    average_Pressure                         0x2000008a   Data           2  ads1110setup.o(.data)
    average_Pressure_bf                      0x2000008c   Data           2  ads1110setup.o(.data)
    self_adaption_Pressure                   0x2000008e   Data           2  ads1110setup.o(.data)
    self_adaption_cont                       0x20000090   Data           1  ads1110setup.o(.data)
    self_adaption_flag                       0x20000091   Data           1  ads1110setup.o(.data)
    ces_cong                                 0x20000092   Data           2  ads1110setup.o(.data)
    tempPressure                             0x20000094   Data           2  ads1110setup.o(.data)
    tempPressure_2                           0x20000096   Data           2  ads1110setup.o(.data)
    ces_flag1                                0x20000098   Data           1  ads1110setup.o(.data)
    usart1RecvCnt                            0x20000099   Data           1  usartsetup.o(.data)
    usart2RecvCnt                            0x2000009a   Data           1  usartsetup.o(.data)
    usart3RecvCnt                            0x2000009b   Data           1  usartsetup.o(.data)
    historyRecordQTY                         0x2000009c   Data           2  history.o(.data)
    historyRecordPointer                     0x2000009e   Data           2  history.o(.data)
    historyRefreshFlag                       0x200000a0   Data           1  history.o(.data)
    FackhistoryRecordQTY                     0x200000a2   Data           2  history.o(.data)
    ADC_ConvertedValue                       0x200000a4   Data           8  adcsetup.o(.data)
    batteryVolt                              0x200000ac   Data          14  adcsetup.o(.data)
    batteryAverage                           0x200000ba   Data           2  adcsetup.o(.data)
    batteryCounts                            0x200000bc   Data           1  adcsetup.o(.data)
    ADC_Voit_Done                            0x200000bd   Data           1  adcsetup.o(.data)
    emSysWorkStep                            0x200000c0   Data           1  controlsystem.o(.data)
    infusionMode                             0x200000c1   Data           1  controlsystem.o(.data)
    controlTimerCounts                       0x200000c2   Data           1  controlsystem.o(.data)
    InfusionStopTimer                        0x200000c4   Data           4  controlsystem.o(.data)
    InfusionXmitTimer                        0x200000c8   Data           4  controlsystem.o(.data)
    lockTimeCountDown                        0x200000cc   Data           2  controlsystem.o(.data)
    G_Led_Time                               0x200000ce   Data           2  controlsystem.o(.data)
    Y_Led_Time                               0x200000d0   Data           2  controlsystem.o(.data)
    emLockPasswordStep                       0x200000d2   Data           1  controlsystem.o(.data)
    emLockPasswordFailStep                   0x200000d3   Data           1  controlsystem.o(.data)
    emAlarmRecordStep                        0x200000d4   Data           1  controlsystem.o(.data)
    emAlarmRememberStep                      0x200000d5   Data           1  controlsystem.o(.data)
    inputDose_bf                             0x200000d6   Data           2  controlsystem.o(.data)
    Input_End                                0x200000d8   Data           1  controlsystem.o(.data)
    start_flag                               0x200000d9   Data           1  controlsystem.o(.data)
    Key_Quiet_Cont                           0x200000da   Data           1  controlsystem.o(.data)
    LimitBeginsTime                          0x200000db   Data           1  controlsystem.o(.data)
    LcdFlicker_Flag                          0x200000dc   Data           1  controlsystem.o(.data)
    PCADontRun_Flag                          0x200000dd   Data           1  controlsystem.o(.data)
    AppendComplete                           0x200000de   Data           1  controlsystem.o(.data)
    Sound_prepore_flag                       0x200000df   Data           1  controlsystem.o(.data)
    pca_count                                0x200000e0   Data           1  controlsystem.o(.data)
    sysPromptToneTypebf                      0x200000e1   Data           1  controlsystem.o(.data)
    TotalDoesChange0                         0x200000e2   Data           1  controlsystem.o(.data)
    TotalDoesChange1                         0x200000e3   Data           1  controlsystem.o(.data)
    Start_send                               0x200000e4   Data           1  controlsystem.o(.data)
    ran                                      0x200000e5   Data           1  controlsystem.o(.data)
    SetParametersAgain                       0x200000e6   Data           1  controlsystem.o(.data)
    InpudingComplete                         0x200000e7   Data           1  controlsystem.o(.data)
    FackreadIndex                            0x200000e8   Data           1  controlsystem.o(.data)
    KEY_Enter_action                         0x200000e9   Data           1  controlsystem.o(.data)
    TurnOffACKTone                           0x200000ea   Data           1  controlsystem.o(.data)
    LCDBlackFlashCount                       0x200000eb   Data           1  controlsystem.o(.data)
    emDisplayPicture                         0x200000ec   Data           1  drawlcdgui.o(.data)
    emCurrentPicture                         0x200000ed   Data           1  drawlcdgui.o(.data)
    emLockPassowrdPicture                    0x200000ee   Data           1  drawlcdgui.o(.data)
    emLockPassowrdFailPicture                0x200000ef   Data           1  drawlcdgui.o(.data)
    emAlarmRecordPicture                     0x200000f0   Data           1  drawlcdgui.o(.data)
    emAlarmRememberPicture                   0x200000f1   Data           1  drawlcdgui.o(.data)
    modifyStep                               0x200000f2   Data           1  drawlcdgui.o(.data)
    Version_data                             0x200000f4   Data           2  drawlcdgui.o(.data)
    SysAlarmJudge                            0x200000f8   Data           8  systemalarm.o(.data)
    sysPromptToneType_bf                     0x20000100   Data           1  systemalarm.o(.data)
    VoltLowest_cont                          0x20000101   Data           1  systemalarm.o(.data)
    VoltLowest_cont2                         0x20000102   Data           1  systemalarm.o(.data)
    Timer_VoltLowes                          0x20000104   Data           4  systemalarm.o(.data)
    VoltLowest_Alarm_Flag                    0x20000108   Data           1  systemalarm.o(.data)
    Alarm_flag                               0x20000109   Data           1  systemalarm.o(.data)
    ADC_LowVoletCount                        0x2000010a   Data           1  systemalarm.o(.data)
    JamSelfcheckCycle                        0x2000010b   Data           1  systemalarm.o(.data)
    self_adaption_Alarmcont                  0x2000010c   Data           1  systemalarm.o(.data)
    JamSelfcheckThroughCycle                 0x2000010d   Data           1  systemalarm.o(.data)
    zigbeeXmitCounts                         0x2000010e   Data           1  zigbeedatahandle.o(.data)
    RunToLorawawn_flag                       0x2000010f   Data           1  zigbeedatahandle.o(.data)
    StartToRun_flag                          0x20000110   Data           1  zigbeedatahandle.o(.data)
    Running_flag                             0x20000111   Data           1  zigbeedatahandle.o(.data)
    check_succeed                            0x20000112   Data           1  zigbeedatahandle.o(.data)
    send_number                              0x20000113   Data           1  zigbeedatahandle.o(.data)
    FailureSendNumber                        0x20000114   Data           2  zigbeedatahandle.o(.data)
    lorawan_to_sleep                         0x20000116   Data           1  zigbeedatahandle.o(.data)
    StartToRunSend_flag                      0x20000117   Data           1  zigbeedatahandle.o(.data)
    PauseSend_flag                           0x20000118   Data           1  zigbeedatahandle.o(.data)
    Recive_lorawanID_flag                    0x2000011a   Data           1  lorawan.o(.data)
    send_cont                                0x2000011c   Data           2  lorawan.o(.data)
    init_sent                                0x2000011e   Data           1  lorawan.o(.data)
    lorawan_init_flag                        0x2000011f   Data           1  lorawan.o(.data)
    lorawan_send_data_flag                   0x20000120   Data           1  lorawan.o(.data)
    BubbleVolt                               0x20000122   Data          40  bubble_adcsetup.o(.data)
    BubbleCounts                             0x2000014a   Data           2  bubble_adcsetup.o(.data)
    BubbleData                               0x2000014c   Data           2  bubble_adcsetup.o(.data)
    BoxData                                  0x2000014e   Data           2  bubble_adcsetup.o(.data)
    BoxCont                                  0x20000150   Data           2  bubble_adcsetup.o(.data)
    BubbleCheckTime                          0x20000152   Data           2  bubble_adcsetup.o(.data)
    BubbleCheckFlag                          0x20000154   Data           2  bubble_adcsetup.o(.data)
    CheckDoneFlag                            0x20000156   Data           2  bubble_adcsetup.o(.data)
    BubbleCountFlag                          0x20000158   Data           1  bubble_adcsetup.o(.data)
    BlockageRecovery                         0x20000159   Data           1  bubble_adcsetup.o(.data)
    AnotherAlarm                             0x2000015a   Data           1  bubble_adcsetup.o(.data)
    ElectricityCheckFlag                     0x2000015c   Data           2  bubble_adcsetup.o(.data)
    ElectricityCheckTime                     0x2000015e   Data           2  bubble_adcsetup.o(.data)
    ElectDoneFlag                            0x20000160   Data           2  bubble_adcsetup.o(.data)
    ElectricityCounts                        0x20000162   Data           2  bubble_adcsetup.o(.data)
    ElectricityData                          0x20000164   Data           2  bubble_adcsetup.o(.data)
    ElectricityDatabf                        0x20000166   Data           2  bubble_adcsetup.o(.data)
    ElectCountFlag                           0x20000168   Data           1  bubble_adcsetup.o(.data)
    ElectStartCount                          0x20000169   Data           1  bubble_adcsetup.o(.data)
    ElectLargeCount                          0x2000016a   Data           1  bubble_adcsetup.o(.data)
    ElectSmallCount                          0x2000016b   Data           1  bubble_adcsetup.o(.data)
    ElectRunCount                            0x2000016c   Data           1  bubble_adcsetup.o(.data)
    ElectBlockingCount                       0x2000016d   Data           1  bubble_adcsetup.o(.data)
    ElectricityCountsOff                     0x2000016e   Data           1  bubble_adcsetup.o(.data)
    ElectricityOffTime                       0x20000170   Data           2  bubble_adcsetup.o(.data)
    ElectricityOFFflag                       0x20000172   Data           2  bubble_adcsetup.o(.data)
    ElectricityOffData                       0x20000174   Data           2  bubble_adcsetup.o(.data)
    SystemCoreClock                          0x20000178   Data           4  system_stm32f10x.o(.data)
    AHBPrescTable                            0x2000017c   Data          16  system_stm32f10x.o(.data)
    err_cout                                 0x200001a0   Data           1  bc26.o(.data)
    bc26_at_event                            0x200001a8   Data          48  bc26.o(.data)
    at_module_bc26                           0x200001d8   Data          80  bc26.o(.data)
    tcp_connect_status                       0x2000022c   Data           1  module_wrapper.o(.data)
    module_start_status                      0x2000022d   Data           1  module_wrapper.o(.data)
    module_init_status                       0x2000022e   Data           1  module_wrapper.o(.data)
    registInfo                               0x20000244   Data           4  programdata.o(.data)
    classification                           0x20000248   Data           4  programdata.o(.data)
    module_check_status                      0x2000026c   Data           4  coaphandle.o(.data)
    coap_send_pkt                            0x20000274   Data         220  coaphandle.o(.data)
    PumpType_Normal                          0x20000350   Data           1  coaphandle.o(.data)
    send_fall_num                            0x20000356   Data           2  coaphandle.o(.data)
    repeat_send_switch                       0x2000035c   Data           1  coaphandle.o(.data)
    registModuleStartCou                     0x20000388   Data           4  regist.o(.data)
    key                                      0x2000038c   Data          17  regist.o(.data)
    remote_flag                              0x200003a0   Data           1  remote.o(.data)
    __stdout                                 0x200003b8   Data           4  stdout.o(.data)
    __microlib_freelist                      0x200003bc   Data           4  mvars.o(.data)
    __microlib_freelist_initialised          0x200003c0   Data           4  mvars.o(.data)
    TaskSchedulerFlag                        0x200003c8   Data          62  typedefine.o(.bss)
    TaskSchedulerTimer                       0x20000408   Data         116  typedefine.o(.bss)
    realTimeData                             0x20000480   Data          64  typedefine.o(.bss)
    verifyInfo                               0x200004c0   Data          16  typedefine.o(.bss)
    setParamInfo                             0x200004d0   Data          60  typedefine.o(.bss)
    runParamInfo                             0x2000050c   Data          14  typedefine.o(.bss)
    evaluateTransfuseValue                   0x2000051a   Data          11  typedefine.o(.bss)
    EngineeringModeValue                     0x20000526   Data          18  typedefine.o(.bss)
    pressureF1                               0x20000538   Data         800  ads1110setup.o(.bss)
    PressureF1_bf                            0x20000858   Data          20  ads1110setup.o(.bss)
    PressureF1_bf2                           0x2000086c   Data          20  ads1110setup.o(.bss)
    self_adaption_buf                        0x20000880   Data          10  ads1110setup.o(.bss)
    usart1XmitBuffer                         0x2000088a   Data          64  usartsetup.o(.bss)
    usart1RecvBuffer                         0x200008ca   Data          32  usartsetup.o(.bss)
    usart2XmitBuffer                         0x200008ea   Data          34  usartsetup.o(.bss)
    usart2RecvBuffer                         0x2000090c   Data          80  usartsetup.o(.bss)
    usart3XmitBuffer                         0x2000095c   Data          64  usartsetup.o(.bss)
    usart3RecvBuffer                         0x2000099c   Data          32  usartsetup.o(.bss)
    historyRecord                            0x200009bc   Data          28  history.o(.bss)
    historyRecordBuf                         0x200009d8   Data        2048  history.o(.bss)
    paramRecordBuf                           0x200011d8   Data         128  parameterset.o(.bss)
    paramTransferBuf                         0x20001258   Data         128  parameterset.o(.bss)
    sysAlarmFlag                             0x200012d8   Data          15  systemalarm.o(.bss)
    AlarmRecord                              0x200012e7   Data          15  systemalarm.o(.bss)
    ElectricityVolt                          0x200012f6   Data         100  bubble_adcsetup.o(.bss)
    ElectricityVolt2                         0x2000135a   Data          40  bubble_adcsetup.o(.bss)
    Elect_adaption_buf                       0x20001382   Data          10  bubble_adcsetup.o(.bss)
    Elect_adaption_buf1                      0x2000138c   Data          10  bubble_adcsetup.o(.bss)
    Elect_adaption_buf2                      0x20001396   Data          10  bubble_adcsetup.o(.bss)
    module_channel                           0x200013a0   Data        2464  module_wrapper.o(.bss)
    PROGRAM_INFO_DATA                        0x20001d4f   Data         600  programdata.o(.bss)
    uart_recv                                0x20001fa8   Data        1036  sys.o(.bss)
    valid_data                               0x200023b4   Data        1228  sys.o(.bss)
    endpoints                                0x20002880   Data          16  coaphandle.o(.bss)
    coap_rec_pkt                             0x20002ce8   Data         220  coaphandle.o(.bss)
    registData                               0x20002df4   Data         200  regist.o(.bss)
    expansionkey                             0x20002ebc   Data         240  regist.o(.bss)
    __heap_base                              0x20003078   Data           0  startup_stm32f10x_md.o(HEAP)
    __heap_limit                             0x20003878   Data           0  startup_stm32f10x_md.o(HEAP)
    __initial_sp                             0x20005c78   Data           0  startup_stm32f10x_md.o(STACK)



==============================================================================

Memory Map of the image

  Image Entry point : 0x080000ed

  Load Region LR_IROM1 (Base: 0x08000000, Size: 0x00028554, Max: 0x00080000, ABSOLUTE, COMPRESSED[0x000282a0])

    Execution Region ER_IROM1 (Base: 0x08000000, Size: 0x00028190, Max: 0x00080000, ABSOLUTE)

    Base Addr    Size         Type   Attr      Idx    E Section Name        Object

    0x08000000   0x000000ec   Data   RO          797    RESET               startup_stm32f10x_md.o
    0x080000ec   0x00000000   Code   RO         1995  * .ARM.Collect$$$$00000000  mc_w.l(entry.o)
    0x080000ec   0x00000004   Code   RO         2346    .ARM.Collect$$$$00000001  mc_w.l(entry2.o)
    0x080000f0   0x00000004   Code   RO         2349    .ARM.Collect$$$$00000004  mc_w.l(entry5.o)
    0x080000f4   0x00000000   Code   RO         2351    .ARM.Collect$$$$00000008  mc_w.l(entry7b.o)
    0x080000f4   0x00000000   Code   RO         2353    .ARM.Collect$$$$0000000A  mc_w.l(entry8b.o)
    0x080000f4   0x00000008   Code   RO         2354    .ARM.Collect$$$$0000000B  mc_w.l(entry9a.o)
    0x080000fc   0x00000000   Code   RO         2356    .ARM.Collect$$$$0000000D  mc_w.l(entry10a.o)
    0x080000fc   0x00000000   Code   RO         2358    .ARM.Collect$$$$0000000F  mc_w.l(entry11a.o)
    0x080000fc   0x00000004   Code   RO         2347    .ARM.Collect$$$$00002712  mc_w.l(entry2.o)
    0x08000100   0x000000c8   Code   RO            1    .text               main.o
    0x080001c8   0x00000728   Code   RO          133    .text               driver.o
    0x080008f0   0x00000494   Code   RO          184    .text               typedefine.o
    0x08000d84   0x00000dd0   Code   RO          215    .text               stm32f10x_it.o
    0x08001b54   0x000004c8   Code   RO          256    .text               rtcsetup.o
    0x0800201c   0x00000074   Code   RO          272    .text               spisetup.o
    0x08002090   0x00000260   Code   RO          284    .text               ads1110setup.o
    0x080022f0   0x00000434   Code   RO          304    .text               iicsetup.o
    0x08002724   0x000002d0   Code   RO          316    .text               usartsetup.o
    0x080029f4   0x00000482   Code   RO          335    .text               lcdsetup.o
    0x08002e76   0x00000002   PAD
    0x08002e78   0x00000b30   Code   RO          347    .text               history.o
    0x080039a8   0x0000009e   Code   RO          370    .text               flashsetup.o
    0x08003a46   0x00000002   PAD
    0x08003a48   0x00000d34   Code   RO          385    .text               parameterset.o
    0x0800477c   0x00000288   Code   RO          403    .text               adcsetup.o
    0x08004a04   0x00005678   Code   RO          421    .text               controlsystem.o
    0x0800a07c   0x000080c0   Code   RO          448    .text               drawlcdgui.o
    0x0801213c   0x0000083c   Code   RO          471    .text               systemalarm.o
    0x08012978   0x00000c58   Code   RO          491    .text               zigbeedatahandle.o
    0x080135d0   0x00000038   Code   RO          511    .text               crc16.o
    0x08013608   0x0000007c   Code   RO          526    .text               hostslavehandle.o
    0x08013684   0x00000534   Code   RO          538    .text               fm31256.o
    0x08013bb8   0x000001bc   Code   RO          574    .text               lorawan.o
    0x08013d74   0x0000079c   Code   RO          597    .text               bubble_adcsetup.o
    0x08014510   0x000001a8   Code   RO          631    .text               system_stm32f10x.o
    0x080146b8   0x000000dc   Code   RO          649    .text               misc.o
    0x08014794   0x0000011c   Code   RO          661    .text               stm32f10x_exti.o
    0x080148b0   0x0000035c   Code   RO          673    .text               stm32f10x_gpio.o
    0x08014c0c   0x000003a4   Code   RO          685    .text               stm32f10x_rcc.o
    0x08014fb0   0x00000408   Code   RO          699    .text               stm32f10x_usart.o
    0x080153b8   0x00000148   Code   RO          711    .text               stm32f10x_rtc.o
    0x08015500   0x00000e1a   Code   RO          723    .text               stm32f10x_tim.o
    0x0801631a   0x00000002   PAD
    0x0801631c   0x000000cc   Code   RO          735    .text               stm32f10x_pwr.o
    0x080163e8   0x000000c4   Code   RO          747    .text               stm32f10x_bkp.o
    0x080164ac   0x000005bc   Code   RO          759    .text               stm32f10x_flash.o
    0x08016a68   0x0000044e   Code   RO          771    .text               stm32f10x_adc.o
    0x08016eb6   0x00000002   PAD
    0x08016eb8   0x00000254   Code   RO          783    .text               stm32f10x_dma.o
    0x0801710c   0x00000024   Code   RO          798    .text               startup_stm32f10x_md.o
    0x08017130   0x00000084   Code   RO          802    .text               delay.o
    0x080171b4   0x00000188   Code   RO          814    .text               at.o
    0x0801733c   0x00000ca0   Code   RO          840    .text               bc26.o
    0x08017fdc   0x0000031c   Code   RO          884    .text               module_wrapper.o
    0x080182f8   0x0000228c   Code   RO          906    .text               cjson.o
    0x0801a584   0x000000f0   Code   RO          959    .text               crc.o
    0x0801a674   0x00000044   Code   RO          974    .text               programdata.o
    0x0801a6b8   0x00000480   Code   RO          993    .text               sys.o
    0x0801ab38   0x0000050c   Code   RO         1015    .text               aes.o
    0x0801b044   0x000003b8   Code   RO         1032    .text               mbedtls_util.o
    0x0801b3fc   0x000005f0   Code   RO         1080    .text               coap.o
    0x0801b9ec   0x00001418   Code   RO         1105    .text               coaphandle.o
    0x0801ce04   0x00000464   Code   RO         1150    .text               regist.o
    0x0801d268   0x000004d4   Code   RO         1173    .text               remote.o
    0x0801d73c   0x00000d80   Code   RO         1193    .text               aes_1.o
    0x0801e4bc   0x000002a8   Code   RO         1252    .text               base64.o
    0x0801e764   0x0000014a   Code   RO         1374    .text               constant_time.o
    0x0801e8ae   0x00000002   PAD
    0x0801e8b0   0x00000020   Code   RO         1608    .text               platform_util.o
    0x0801e8d0   0x00001cc8   Code   RO         1833    .text               sha1.o
    0x08020598   0x00001276   Code   RO         1845    .text               sha256.o
    0x0802180e   0x00000062   Code   RO         1998    .text               mc_w.l(uldiv.o)
    0x08021870   0x0000000c   Code   RO         2000    .text               mc_w.l(tolower.o)
    0x0802187c   0x00000024   Code   RO         2002    .text               mc_w.l(rand.o)
    0x080218a0   0x00000024   Code   RO         2005    .text               mc_w.l(memcpya.o)
    0x080218c4   0x00000024   Code   RO         2009    .text               mc_w.l(memseta.o)
    0x080218e8   0x00000024   Code   RO         2013    .text               mc_w.l(strstr.o)
    0x0802190c   0x0000000e   Code   RO         2015    .text               mc_w.l(strlen.o)
    0x0802191a   0x0000001c   Code   RO         2017    .text               mc_w.l(strcmp.o)
    0x08021936   0x0000001a   Code   RO         2019    .text               mc_w.l(memcmp.o)
    0x08021950   0x00000012   Code   RO         2021    .text               mc_w.l(strcpy.o)
    0x08021962   0x0000001e   Code   RO         2023    .text               mc_w.l(strncmp.o)
    0x08021980   0x00000044   Code   RO         2025    .text               mc_w.l(strtok.o)
    0x080219c4   0x00000038   Code   RO         2326    .text               mc_w.l(__0sscanf.o)
    0x080219fc   0x00000338   Code   RO         2328    .text               mc_w.l(scanf_fp.o)
    0x08021d34   0x0000014e   Code   RO         2332    .text               mf_w.l(dadd.o)
    0x08021e82   0x000000e4   Code   RO         2334    .text               mf_w.l(dmul.o)
    0x08021f66   0x00000022   Code   RO         2336    .text               mf_w.l(dflti.o)
    0x08021f88   0x0000003e   Code   RO         2338    .text               mf_w.l(dfixi.o)
    0x08021fc6   0x00000026   Code   RO         2340    .text               mf_w.l(f2d.o)
    0x08021fec   0x00000030   Code   RO         2342    .text               mf_w.l(cdcmple.o)
    0x0802201c   0x00000030   Code   RO         2344    .text               mf_w.l(cdrcmple.o)
    0x0802204c   0x0000002c   Code   RO         2361    .text               mc_w.l(uidiv.o)
    0x08022078   0x0000001e   Code   RO         2363    .text               mc_w.l(llshl.o)
    0x08022096   0x00000020   Code   RO         2365    .text               mc_w.l(llushr.o)
    0x080220b6   0x00000024   Code   RO         2367    .text               mc_w.l(llsshr.o)
    0x080220da   0x00000002   PAD
    0x080220dc   0x00000028   Code   RO         2371    .text               mc_w.l(scanf_char.o)
    0x08022104   0x00000040   Code   RO         2373    .text               mc_w.l(_sgetc.o)
    0x08022144   0x0000009c   Code   RO         2375    .text               mc_w.l(strtod.o)
    0x080221e0   0x00000000   Code   RO         2377    .text               mc_w.l(iusefp.o)
    0x080221e0   0x000000ba   Code   RO         2378    .text               mf_w.l(depilogue.o)
    0x0802229a   0x000000de   Code   RO         2380    .text               mf_w.l(ddiv.o)
    0x08022378   0x00000018   Code   RO         2382    .text               mf_w.l(dfltul.o)
    0x08022390   0x00000030   Code   RO         2384    .text               mf_w.l(dfixul.o)
    0x080223c0   0x00000038   Code   RO         2386    .text               mf_w.l(d2f.o)
    0x080223f8   0x00000024   Code   RO         2388    .text               mc_w.l(init.o)
    0x0802241c   0x0000000a   Code   RO         2390    .text               mc_w.l(isspace_c.o)
    0x08022426   0x00000002   PAD
    0x08022428   0x0000032c   Code   RO         2392    .text               mc_w.l(_scanf.o)
    0x08022754   0x0000006e   Code   RO         2394    .text               mf_w.l(fepilogue.o)
    0x080227c2   0x00000002   PAD
    0x080227c4   0x00000028   Code   RO         2396    .text               mc_w.l(ctype_c.o)
    0x080227ec   0x00000056   Code   RO         2407    .text               mc_w.l(__dczerorl2.o)
    0x08022842   0x00000002   PAD
    0x08022844   0x00000020   Code   RO         2268    i.__0printf         mc_w.l(printfa.o)
    0x08022864   0x00000030   Code   RO         2269    i.__0snprintf       mc_w.l(printfa.o)
    0x08022894   0x00000028   Code   RO         2270    i.__0sprintf        mc_w.l(printfa.o)
    0x080228bc   0x0000002c   Code   RO         2273    i.__0vsnprintf      mc_w.l(printfa.o)
    0x080228e8   0x0000005c   Code   RO         2300    i.__free$realloc    mc_w.l(mallocr.o)
    0x08022944   0x00000050   Code   RO         2301    i.__malloc$realloc  mc_w.l(mallocr.o)
    0x08022994   0x0000000e   Code   RO         2401    i.__scatterload_copy  mc_w.l(handlers.o)
    0x080229a2   0x00000002   Code   RO         2402    i.__scatterload_null  mc_w.l(handlers.o)
    0x080229a4   0x0000000e   Code   RO         2403    i.__scatterload_zeroinit  mc_w.l(handlers.o)
    0x080229b2   0x00000002   PAD
    0x080229b4   0x00000184   Code   RO         2275    i._fp_digits        mc_w.l(printfa.o)
    0x08022b38   0x0000000e   Code   RO         2330    i._is_digit         mc_w.l(scanf_fp.o)
    0x08022b46   0x00000002   PAD
    0x08022b48   0x000006dc   Code   RO         2276    i._printf_core      mc_w.l(printfa.o)
    0x08023224   0x00000024   Code   RO         2277    i._printf_post_padding  mc_w.l(printfa.o)
    0x08023248   0x0000002e   Code   RO         2278    i._printf_pre_padding  mc_w.l(printfa.o)
    0x08023276   0x00000016   Code   RO         2279    i._snputc           mc_w.l(printfa.o)
    0x0802328c   0x0000000a   Code   RO         2280    i._sputc            mc_w.l(printfa.o)
    0x08023296   0x00000002   PAD
    0x08023298   0x00000050   Code   RO         2302    i.internal_alloc    mc_w.l(mallocr.o)
    0x080232e8   0x0000006c   Code   RO         2303    i.realloc           mc_w.l(mallocr.o)
    0x08023354   0x0000001c   Code   RO         1992    i.strtod            m_ws.l(strtod.o)
    0x08023370   0x00000018   Data   RO          257    .constdata          rtcsetup.o
    0x08023388   0x0000253e   Data   RO          449    .constdata          drawlcdgui.o
    0x080258c6   0x00000200   Data   RO          512    .constdata          crc16.o
    0x08025ac6   0x0000020a   Data   RO         1016    .constdata          aes.o
    0x08025cd0   0x00000020   Data   RO         1107    .constdata          coaphandle.o
    0x08025cf0   0x00002228   Data   RO         1194    .constdata          aes_1.o
    0x08027f18   0x00000100   Data   RO         1846    .constdata          sha256.o
    0x08028018   0x00000040   Data   RO         2397    .constdata          mc_w.l(ctype_c.o)
    0x08028058   0x0000005e   Data   RO          841    .conststring        bc26.o
    0x080280b6   0x00000002   PAD
    0x080280b8   0x000000b8   Data   RO         1108    .conststring        coaphandle.o
    0x08028170   0x00000020   Data   RO         2399    Region$$Table       anon$$obj.o


    Execution Region RW_IRAM1 (Base: 0x20000000, Size: 0x00005c78, Max: 0x00010000, ABSOLUTE, COMPRESSED[0x00000110])

    Base Addr    Size         Type   Attr      Idx    E Section Name        Object

    0x20000000   0x00000008   Data   RW          134    .data               driver.o
    0x20000008   0x0000004c   Data   RW          186    .data               typedefine.o
    0x20000054   0x00000029   Data   RW          216    .data               stm32f10x_it.o
    0x2000007d   0x00000001   PAD
    0x2000007e   0x00000004   Data   RW          258    .data               rtcsetup.o
    0x20000082   0x00000017   Data   RW          286    .data               ads1110setup.o
    0x20000099   0x00000003   Data   RW          318    .data               usartsetup.o
    0x2000009c   0x00000008   Data   RW          349    .data               history.o
    0x200000a4   0x0000001a   Data   RW          404    .data               adcsetup.o
    0x200000be   0x00000002   PAD
    0x200000c0   0x0000002c   Data   RW          422    .data               controlsystem.o
    0x200000ec   0x0000000a   Data   RW          450    .data               drawlcdgui.o
    0x200000f6   0x00000002   PAD
    0x200000f8   0x00000016   Data   RW          473    .data               systemalarm.o
    0x2000010e   0x0000000b   Data   RW          492    .data               zigbeedatahandle.o
    0x20000119   0x00000001   PAD
    0x2000011a   0x00000007   Data   RW          575    .data               lorawan.o
    0x20000121   0x00000001   PAD
    0x20000122   0x00000054   Data   RW          599    .data               bubble_adcsetup.o
    0x20000176   0x00000002   PAD
    0x20000178   0x00000014   Data   RW          632    .data               system_stm32f10x.o
    0x2000018c   0x00000014   Data   RW          686    .data               stm32f10x_rcc.o
    0x200001a0   0x00000088   Data   RW          842    .data               bc26.o
    0x20000228   0x00000007   Data   RW          886    .data               module_wrapper.o
    0x2000022f   0x00000001   PAD
    0x20000230   0x00000014   Data   RW          908    .data               cjson.o
    0x20000244   0x00000008   Data   RW          976    .data               programdata.o
    0x2000024c   0x0000013b   Data   RW         1109    .data               coaphandle.o
    0x20000387   0x00000001   PAD
    0x20000388   0x00000015   Data   RW         1152    .data               regist.o
    0x2000039d   0x00000003   PAD
    0x200003a0   0x0000000a   Data   RW         1175    .data               remote.o
    0x200003aa   0x00000002   PAD
    0x200003ac   0x00000004   Data   RW         1609    .data               platform_util.o
    0x200003b0   0x00000004   Data   RW         2003    .data               mc_w.l(rand.o)
    0x200003b4   0x00000004   Data   RW         2026    .data               mc_w.l(strtok.o)
    0x200003b8   0x00000004   Data   RW         2360    .data               mc_w.l(stdout.o)
    0x200003bc   0x00000004   Data   RW         2369    .data               mc_w.l(mvars.o)
    0x200003c0   0x00000004   Data   RW         2370    .data               mc_w.l(mvars.o)
    0x200003c4   0x00000004   PAD
    0x200003c8   0x00000170   Zero   RW          185    .bss                typedefine.o
    0x20000538   0x00000352   Zero   RW          285    .bss                ads1110setup.o
    0x2000088a   0x00000132   Zero   RW          317    .bss                usartsetup.o
    0x200009bc   0x0000081c   Zero   RW          348    .bss                history.o
    0x200011d8   0x00000100   Zero   RW          386    .bss                parameterset.o
    0x200012d8   0x0000001e   Zero   RW          472    .bss                systemalarm.o
    0x200012f6   0x000000aa   Zero   RW          598    .bss                bubble_adcsetup.o
    0x200013a0   0x000009a0   Zero   RW          885    .bss                module_wrapper.o
    0x20001d40   0x0000000f   Zero   RW          907    .bss                cjson.o
    0x20001d4f   0x00000258   Zero   RW          975    .bss                programdata.o
    0x20001fa7   0x00000001   PAD
    0x20001fa8   0x000008d8   Zero   RW          994    .bss                sys.o
    0x20002880   0x00000574   Zero   RW         1106    .bss                coaphandle.o
    0x20002df4   0x000001b8   Zero   RW         1151    .bss                regist.o
    0x20002fac   0x000000c8   Zero   RW         1174    .bss                remote.o
    0x20003074   0x00000004   PAD
    0x20003078   0x00000800   Zero   RW          796    HEAP                startup_stm32f10x_md.o
    0x20003878   0x00002400   Zero   RW          795    STACK               startup_stm32f10x_md.o


==============================================================================

Image component sizes


      Code (inc. data)   RO Data    RW Data    ZI Data      Debug   Object Name

       648         54          0         26          0       2265   adcsetup.o
       608         62          0         23        850       3037   ads1110setup.o
      1292         12        522          0          0       6107   aes.o
      3456        102       8744          0          0      16280   aes_1.o
       392         14          0          0          0       4456   at.o
       680          0          0          0          0       2970   base64.o
      3232        964         94        136          0      10866   bc26.o
      1948        222          0         84        170       5074   bubble_adcsetup.o
      8844        180          0         20         15      46711   cjson.o
      1520          8          0          0          0       9010   coap.o
      5144        956        216        315       1396      16457   coaphandle.o
       330          0          0          0          0       3291   constant_time.o
     22136       1998          0         44          0      24372   controlsystem.o
         0          0          0          0          0         32   core_cm3.o
       240          0          0          0          0       1596   crc.o
        56          8        512          0          0       1357   crc16.o
       132          4          0          0          0        853   delay.o
     32960       2212       9534         10          0      26326   drawlcdgui.o
      1832         68          0          8          0      63200   driver.o
       158          0          0          0          0       7909   flashsetup.o
      1332          6          0          0          0       4874   fm31256.o
      2864        116          0          8       2076       4243   history.o
       124         16          0          0          0        694   hostslavehandle.o
      1076          8          0          0          0       3676   iicsetup.o
      1154          6          0          0          0       5489   lcdsetup.o
       444         44          0          7          0       3116   lorawan.o
       200         18          0          0          0     238499   main.o
       952         90          0          0          0       7734   mbedtls_util.o
       220         22          0          0          0       1849   misc.o
       796         10          0          7       2464       8399   module_wrapper.o
      3380         72          0          0        256       3402   parameterset.o
        32          6          0          4          0       1535   platform_util.o
        68         10          0          8        600       2278   programdata.o
      1124        328          0         21        440       4244   regist.o
      1236        420          0         10        200       3144   remote.o
      1224         52         24          4          0       4357   rtcsetup.o
      7368         54          0          0          0       6938   sha1.o
      4726         82        256          0          0       6804   sha256.o
       116          4          0          0          0        783   spisetup.o
        36          8        236          0      11264        836   startup_stm32f10x_md.o
      1102         26          0          0          0      11093   stm32f10x_adc.o
       196          8          0          0          0       3552   stm32f10x_bkp.o
       596          8          0          0          0       4418   stm32f10x_dma.o
       284         10          0          0          0       2311   stm32f10x_exti.o
      1468         34          0          0          0       8262   stm32f10x_flash.o
       860         38          0          0          0       5785   stm32f10x_gpio.o
      3536        308          0         41          0       5305   stm32f10x_it.o
       204         14          0          0          0       1979   stm32f10x_pwr.o
       932         36          0         20          0       9000   stm32f10x_rcc.o
       328          4          0          0          0       2754   stm32f10x_rtc.o
      3610         88          0          0          0      22896   stm32f10x_tim.o
      1032         22          0          0          0       8508   stm32f10x_usart.o
      1152         48          0          0       2264       6637   sys.o
       424         36          0         20          0       2079   system_stm32f10x.o
      2108        208          0         22         30       4933   systemalarm.o
      1172        156          0         76        368      14991   typedefine.o
       720         20          0          3        306       3612   usartsetup.o
      3160        180          0         11          0       5359   zigbeedatahandle.o

    ----------------------------------------------------------------------
    136974       9480      20172        944      22704     688537   Object Totals
         0          0         32          0          0          0   (incl. Generated)
        10          0          2         16          5          0   (incl. Padding)

    ----------------------------------------------------------------------

      Code (inc. data)   RO Data    RW Data    ZI Data      Debug   Library Member Name

        28          0          0          0          0         80   strtod.o
        56          8          0          0          0         84   __0sscanf.o
        86          0          0          0          0          0   __dczerorl2.o
       812          4          0          0          0        112   _scanf.o
        64          0          0          0          0         84   _sgetc.o
        40          6         64          0          0         68   ctype_c.o
         0          0          0          0          0          0   entry.o
         0          0          0          0          0          0   entry10a.o
         0          0          0          0          0          0   entry11a.o
         8          4          0          0          0          0   entry2.o
         4          0          0          0          0          0   entry5.o
         0          0          0          0          0          0   entry7b.o
         0          0          0          0          0          0   entry8b.o
         8          4          0          0          0          0   entry9a.o
        30          0          0          0          0          0   handlers.o
        36          8          0          0          0         68   init.o
        10          0          0          0          0         68   isspace_c.o
         0          0          0          0          0          0   iusefp.o
        30          0          0          0          0         68   llshl.o
        36          0          0          0          0         68   llsshr.o
        32          0          0          0          0         68   llushr.o
       360         30          0          0          0        356   mallocr.o
        26          0          0          0          0         80   memcmp.o
        36          0          0          0          0         68   memcpya.o
        36          0          0          0          0        108   memseta.o
         0          0          0          8          0          0   mvars.o
      2422        104          0          0          0        836   printfa.o
        36         10          0          4          0        136   rand.o
        40          8          0          0          0         84   scanf_char.o
       838         12          0          0          0        216   scanf_fp.o
         0          0          0          4          0          0   stdout.o
        28          0          0          0          0         76   strcmp.o
        18          0          0          0          0         68   strcpy.o
        14          0          0          0          0         68   strlen.o
        30          0          0          0          0         80   strncmp.o
        36          0          0          0          0         80   strstr.o
       156         12          0          0          0        120   strtod.o
        68          6          0          4          0         80   strtok.o
        12          0          0          0          0         68   tolower.o
        44          0          0          0          0         80   uidiv.o
        98          0          0          0          0         92   uldiv.o
        48          0          0          0          0         68   cdcmple.o
        48          0          0          0          0         68   cdrcmple.o
        56          0          0          0          0         88   d2f.o
       334          0          0          0          0        148   dadd.o
       222          0          0          0          0        100   ddiv.o
       186          0          0          0          0        176   depilogue.o
        62          0          0          0          0         80   dfixi.o
        48          0          0          0          0         68   dfixul.o
        34          0          0          0          0         76   dflti.o
        24          0          0          0          0         76   dfltul.o
       228          0          0          0          0         96   dmul.o
        38          0          0          0          0         68   f2d.o
       110          0          0          0          0        168   fepilogue.o

    ----------------------------------------------------------------------
      7030        216         64         20          4       4744   Library Totals
        14          0          0          0          4          0   (incl. Padding)

    ----------------------------------------------------------------------

      Code (inc. data)   RO Data    RW Data    ZI Data      Debug   Library Name

        28          0          0          0          0         80   m_ws.l
      5550        216         64         20          0       3384   mc_w.l
      1438          0          0          0          0       1280   mf_w.l

    ----------------------------------------------------------------------
      7030        216         64         20          4       4744   Library Totals

    ----------------------------------------------------------------------

==============================================================================


      Code (inc. data)   RO Data    RW Data    ZI Data      Debug   

    144004       9696      20236        964      22708     685609   Grand Totals
    144004       9696      20236        272      22708     685609   ELF Image Totals (compressed)
    144004       9696      20236        272          0          0   ROM Totals

==============================================================================

    Total RO  Size (Code + RO Data)               164240 ( 160.39kB)
    Total RW  Size (RW Data + ZI Data)             23672 (  23.12kB)
    Total ROM Size (Code + RO Data + RW Data)     164512 ( 160.66kB)

==============================================================================

